:0200000480007A
:100000009705000093850528732560026B10B500E5
:10001000EF000027130510006B00050013858126F3
:10002000138601323306A64093050000EF00D06628
:1000300017150000130505D7EF005052EF00105CB4
:08004000EF0080006F00D052B8
:10004800130101F3130510002326110C2322910C30
:100058002324810C2320210D232E310B232C410B2B
:10006800232A510B2328610BEF00005437550180D8
:1000780013050598EF00405A930401021387040002
:1000880093070000930640022320F7009387170088
:1000980013074700E39AD7FE130400001307100064
:1000A800B75901801309400283A70400930504008F
:1000B8001385C99A63868700EF0040641307000020
:1000C8001304140093844400E31024FF631E0716EE
:1000D800375501801305059EEF000054EF005013BB
:1000E800375501801305059FEF00005313054000A5
:1000F800EF00804BEF00501B13051000EF00C04AC3
:1001080037550180130545A0EF000051EF009027F7
:1001180037550180130545A13704FFFFEF00C04F95
:1001280093040000375B0180B75A0180375A018079
:10013800B759018013094401232094009305040052
:1001480013058BA2EF00805B9385040013850AA337
:10015800EF00C05A9385040013054AA4EF00005A23
:10016800138549A513044400EF00004B9384140041
:10017800E31424FD375501801305C5A6EF00C049D7
:10018800B76701809387C7003716008013074000C0
:10019800138807049306C10013068694930540004C
:1001A80013054000138941292326F1002328010162
:1001B800232CE100232EE100232A2101EF00006611
:1001C800375501801305C5A8EF00004593040000CA
:1001D800375A0180B75A0180930940001304000080
:1001E80083278101B387F402B38787009397270099
:1001F800B307F90003A5070013041400EF00004635
:100208001305CAA2EF004041E31C34FD9384140097
:1002180013858A9AEF004040E39284FC8320C10C46
:100228000324810C8324410C0329010C8329C10B6D
:10023800032A810B832A410B032B010B13050000B2
:100248001301010D67800000375501801305859B58
:10025800EF00803C6FF0DFE793070000638807003A
:1002680037150080130505DA6F00D02E678000006F
:10027800130500006B000500732550026B00050094
:100288009761010093810158F32520029395A500F9
:10029800732600021316260037F1FF6F3301B140B1
:1002A8003301C100F326100263860600130500001F
:1002B8006B0005006780000083270500135886003F
:1002C80093560601135786012380C700A3800701B0
:1002D8002381D700A381E700938847006352C00AAF
:1002E8001388870033B80501B3B6B7001307F6FFC4
:1002F8001348180093C6160013379700B366D80042
:10030800134717003377D7006304070833E7B800AB
:1003180013773700631E07061378C6FF9387050017
:10032800138708003308B80083A60700938747009F
:1003380013074700232ED7FEE39807FF9377C6FFDE
:10034800B386F800630CF6023387F500034807000C
:1003580013871700238006016352C7023387E5001D
:100368000347070093872700A380E60063D8C700E8
:10037800B387F50083C707002381F600B388C80058
:1003880093F73800B3881701232015016780000010
:1003980013074600B387E7001387080083C60500E4
:1003A8001307170093851500A30FD7FEE318F7FE70
:1003B8006FF0DFFC83270500130101FF03C8070066
:1003C80003C6170083C6270003C7370023060101A9
:1003D800A306C1002307D100A307E1008328C100B9
:1003E800138847006352100B1386870033B6C50085
:1003F800B3B6B7001387F8FF1346160093C6160066
:1004080013379700B366D600134717003377D70022
:100418006306070833E705011377370063100708F9
:1004280013F6C8FF13070800938705003306B600C4
:1004380083260700938747001307470023AED7FE9C
:10044800E398C7FE93F7C8FFB306F800638CF80279
:1004580003C306003386F5001387170023006600E0
:100468006352170303C616003387E50093872700F6
:100478002300C70063D8170103C72600B387F50018
:100488002380E70033081801937738003388070181
:10049800232005011301010167800000138748002C
:1004A800B387E70013070800834607001307170000
:1004B80093851500A38FD5FEE318F7FE6FF09FFC18
:1004C80067800000B727000023A2F500130500008D
:1004D8006780000013051000678000001305000006
:1004E8006780000013050000678000001305060000
:1004F800635EC000B386C5003707010083C70500E7
:10050800938515002320F700E39AD5FE6780000045
:10051800130101FF232481001304050037550180CE
:100528001305058723261100EF00000F1355F4412A
:10053800B3478500B7360000B387A7409386068087
:1005480003A5412563D4F600938706008320C100E4
:1005580003248100B387A70023AAF1241301010112
:100568006780000013050000678000001305000085
:100578006F0080036F0040063755018013054588DA
:100588006F00800903A581261307150023A4E1261F
:1005980067800000375501801305858A6F00C00702
:1005A8006B10B500678000006B00050067800000D5
:1005B8006B40B500678000006B2005006780000075
:1005C8006B30000067800000732510026780000010
:1005D80073253002678000007325000267800000E1
:1005E80073252002678000007325400267800000A1
:1005F8007325500267800000732560026780000041
:100608007325700267800000732500C067800000B2
:10061800732520C067800000130141FF23201100CB
:100628002322B1008345050063880500EF00C0015F
:10063800130515006FF01FFF83200100832541007B
:100648001301C10067800000976201009382829BBA
:1006580083A2020023A0B20067800000130101FFFB
:100668002322910023261100232481002320210125
:100678009307F0009304050063FCA7043759018031
:1006880093060000130400021309C9901304C4FF61
:10069800B3D7840093F7F700139727003307E900CF
:1006A800639407006388060003250700EFF0DFF670
:1006B80093061000E31C04FC8320C100032481007E
:1006C8008324410003290100130101016780000010
:1006D800B7570180931425009387C790032481009E
:1006E800B384970003A504008320C100832441003C
:1006F80003290100130101016FF01FF2130101FF2B
:100708002324810023261100232291002320210184
:1007180013840500EFF05FF09307F00063F087069D
:100728003759018093060000930400021309C99009
:100738009384C4FFB357940093F7F70013972700E7
:100748003307E90063940700638806000325070060
:10075800EFF09FEC93061000E39C04FC0324810057
:100768008320C100832441000329010037550180FB
:100778001305859A130101016FF01FEAB75701802D
:100788009387C7901314240033848700032504003B
:10079800EFF09FE86FF09FFC03A5C127130101FF4D
:1007A80023261100EFF05FE003A5012883A7412865
:1007B800E7800700EFF05FE18320C10013351500E3
:1007C800130101016FF05FDE03A58127130101FF0B
:1007D8002326110023248100EFF01FDDEFF0DFDF77
:1007E80013040500EFF0DFDE83A54127930605001B
:1007F80003A5C12683A701271306040013070000D9
:10080800E7800700EFF05FDC032481008320C1004C
:1008180013351500130101016FF01FD9130101FFF2
:100828002324810023229100232021012326110063
:1008380023A2C12823A0D12823AEB12693071000F4
:1008480063FAA700B70500809385057AEFF05FD5B6
:1008580083A5C12713850500EFF01FD503A501283F
:1008680083A74128E7800700EFF01FD60324810003
:100878008320C1008324410003290100133515009A
:10088800130101016FF05FD2832685001307100062
:100898006362D70A9307050003250500130101FECB
:1008A80083A64700232C8100232A910023282101B5
:1008B80023263101232E110023ACA12623AAF126D9
:1008C80023A8B12623A6C126636AD704EFF0DFCD9B
:1008D800EFF09FD013040500EFF09FCF83A54127C9
:1008E80083A701279306050003A5C1261306040064
:1008F80013070000E7800700EFF01FCD03248101F4
:100908008320C10183244101032901018329C100F6
:1009180013351500130101026FF01FC9B7050080D8
:10092800138506009385057DEFF09FC703A58127F2
:100938006FF0DFF9375501801305C5946F00006724
:10094800130101FF23261100232481002322910093
:1009580093040500EFF05FC713040500EFF0DFC74D
:1009680083A7C40083A6040003A744003304F40249
:1009780083A784008320C100832441003304A4009A
:10098800131524003386A600B306A70083A6060025
:1009980003270600032481003385A700B307D70087
:1009A8002320F5001301010167800000130101FFF6
:1009B80023261100EFF05FC1131725009387412DFF
:1009C800B387E70023A0A700631805008320C100B0
:1009D80013010101678000008320C1001305000096
:1009E800130101016FF05FBC130101FF2326110001
:1009F800EFF09FBE8320C10013172500938741881D
:100A0800B387E70023A0A700130101016780000056
:100A180037550180130101FF130585AC232611000A
:100A28002324810023229100EFF01FBF130540000B
:100A3800EFF09FB7EFF05FBA1384418813172500D2
:100A4800930705003307E400130510002320F7007F
:100A5800EFF09FB503250400B7540180EFF01FC0E5
:100A68001385849AEFF05FBB03254400EFF01FBFA6
:100A78001385849AEFF05FBA03258400EFF01FBE58
:100A88001385849AEFF05FB90325C400EFF01FBD0A
:100A9800032481008320C1001385849A83244100A4
:100AA800130101016FF05FB7130101FF2326110045
:100AB8002324810023229100EFF01FB213040500C4
:100AC80013352500EFF05FAF9307100063F8870830
:100AD80013353400EFF05FAE930720009384412D67
:100AE8006308F40613142400338484009307D000A9
:100AF8002328F400EFF0DFACEFF09FAC03A504016E
:100B080037540180EFF09FB51305849AEFF0DFB0FA
:100B180003A54401EFF09FB41305849AEFF0DFAF0B
:100B280003A58401EFF09FB31305849AEFF0DFAEBD
:100B380003A5C401EFF09FB21305849A0324810032
:100B48008320C10083244100130101016FF0DFAC51
:100B58009307C00023ACF4006FF0DFF913451400CD
:100B6800EFF09FA59384412D631804009307A0001C
:100B780023A8F4006FF01FF89307B00023AAF4002D
:100B88006FF05FF7B7150080130101FF9385459B50
:100B980013054000232611002324810023229100FD
:100BA800EFF01FA0EFF05FA21384412D93172500EB
:100BB800B307F40023A0A700631C05040325040061
:100BC800B7540180EFF09FA91385849AEFF0DFA452
:100BD80003254400EFF09FA81385849AEFF0DFA364
:100BE80003258400EFF09FA71385849AEFF0DFA216
:100BF8000325C400EFF09FA6032481008320C100D1
:100C08001385849A83244100130101016FF0DFA04A
:100C180013050000EFF05F996FF05FFA3755018018
:100C2800130101FF130585AC23261100232481003D
:100C380023229100EFF05F9E13054000EFF0DF964E
:100C4800EFF09F99938441881317250093070500B7
:100C58003387E400130510002320F700EFF0DF943A
:100C680003A5040037540180EFF05F9F1305849AB1
:100C7800EFF09F9A03A54400EFF05F9E1305849A56
:100C8800EFF09F9903A58400EFF05F9D1305849A08
:100C9800EFF09F9803A5C4009384412DEFF01F9CAB
:100CA8001305849AEFF05F97375501801305059F68
:100CB800EFF09F9613054000EFF01F8FEFF0DFDE97
:100CC80013051000EFF05F8E37550180130585ADD1
:100CD800EFF09F94B71500809385459B130540005E
:100CE800EFF01F8CEFF05F8E93172500B387F400A9
:100CF80023A0A700631A050403A50400EFF01F96BC
:100D08001305849AEFF05F9103A54400EFF01F9557
:100D18001305849AEFF05F9003A58400EFF01F9409
:100D28001305849AEFF05F8F03A5C400EFF01F93BB
:100D38001305849A032481008320C1008324410081
:100D4800130101016FF05F8D13050000EFF0DF85DF
:100D58006FF09FFA93050500930600001306000044
:100D6800130500006F209075130101FF9305000023
:100D7800232481002326110013040500EF20907D11
:100D880003A501258327C50363840700E7800700BF
:100D980013050400EFF0CFCD130101FF23248100D8
:100DA800B7670180376401801304440093874700C4
:100DB800B3878740232291002326110093D427402C
:100DC800638004029387C7FF338487008327040066
:100DD8009384F4FF1304C4FFE7800700E39804FE3C
:100DE8008320C100032481008324410013010101F1
:100DF80067800000130101FF2324810023202101C3
:100E080037640180376901809307040013090900DA
:100E18003309F94023261100232291001359294050
:100E280063000902130404009304000083270400EC
:100E38009384140013044400E7800700E31899FE24
:100E4800376401803769018093070400130949005A
:100E58003309F940135929406300090213040400B7
:100E680093040000832704009384140013044400AF
:100E7800E7800700E31899FE8320C100032481005E
:100E88008324410003290100130101016780000048
:100E98001303F00013070500637EC3029377F7007E
:100EA8006390070A63920508937606FF1376F600A7
:100EB800B386E6002320B7002322B7002324B70017
:100EC8002326B70013070701E366D7FE631406005D
:100ED80067800000B306C34093962600970200007F
:100EE800B38656006780C6002307B700A306B7007D
:100EF8002306B700A305B7002305B700A304B7006E
:100F08002304B700A303B7002303B700A302B70065
:100F18002302B700A301B7002301B700A300B7005D
:100F28002300B7006780000093F5F50F93968500BE
:100F3800B3E5D50093960501B3E5D5006FF0DFF66C
:100F48009396270097020000B3865600938200000C
:100F5800E78006FA93800200938707FF3307F7407C
:100F68003306F600E378C3F66FF0DFF3130101FCF4
:100F78002324C1022326D1022328E102232AF102D5
:100F8800232C0103232E11031386050083258500D6
:100F980093068102232E11002326D100EF00C005FD
:100FA8008320C101130101046780000003A3C12548
:100FB800130101FC2324C1022326D1022322B102FA
:100FC8002328E102232AF102232C0103232E1103F3
:100FD80083258300930641021306050013050300C9
:100FE800232E11002326D100EF0000018320C10128
:100FF8001301010467800000130101E12326111E7B
:101008002320211F2324811D2320A11D138C0500CB
:1010180013090600232AD1002324811E2322911EAE
:10102800232E311D232C411D232A511D2328611DE8
:101038002326711D2322911D232EB11B130D05009C
:10104800EF60005783270500138507002328F10266
:10105800EF8040512326A1022328010E232A010EE6
:10106800232C010E232E010E63060D0003278D038A
:10107800E308070A8316CC00139706019397260105
:101088001357070163CA07023727000003264C06D7
:1010980033E7E60013170701B7E6FFFF13570741C9
:1010A8009386F6FFB376D6002316EC0013170701D4
:1010B8002322DC0613570701937687006388062EE0
:1010C80083260C016384062E1377A7019306A000DC
:1010D8006300D7309307C110375701802322F10EE0
:1010E80093880700930747B237570180232CF100F4
:1010F800130B0900930707CA2324F10083470B0049
:101108002326010E2324010E23200102232A010293
:10111800232C0102232E0102232401042326010487
:10112800232601006386072213040B00930650024E
:10113800638AD7308347140013041400E39A07FE28
:10114800B3046441630664218326C10E8327810E9C
:1011580023A06801B38696009387170023A29800FE
:101168002326D10E2324F10E93067000938888005D
:1011780063C2F62E0327C100834704003307970094
:101188002326E1006386071C83441400A303010C93
:1011980013041400930DF0FF93090000130A0000D4
:1011A8001309A005930A9000930BA002938C0800E2
:1011B80013041400938704FE6364F9040327810170
:1011C80093972700B387E70083A707006780070086
:1011D80093090000938604FD834404009397290033
:1011E800B387370193971700B389F600938604FDF8
:1011F80013041400E3F2DAFE938704FEE370F9FCAB
:1012080093880C006386041423069114A303010C2D
:10121800930A1000930C1000130BC114232801002B
:10122800930D00002324010223220102232E010032
:10123800937B2A0063840B00938A2A0013794A0857
:101248008327C10E6316090033885941E3460071AC
:101258008346710C638A06028326810E1306710C7D
:1012680023A0C80093871700130610009386160062
:1012780023A2C8002326F10E2324D10E13067000E2
:10128800938888006342D652638C0B028326810EB2
:101298001306810C23A0C80093872700130620009B
:1012A8009386160023A2C8002326F10E2324D10E0C
:1012B80013067000938888006354D6006F00D078B6
:1012C80093060008E30ED93CB38D9D41E34AB0492B
:1012D80093760A10E39806280327810EB3879701AF
:1012E80023A068011307170023A298012326F10EF3
:1012F8002324E10E9306700063C8E654938888009F
:10130800137A4A0063060A00B3845941634E905425
:1013180063D4590193890A000327C10033073701B1
:101328002326E100E398074E832701012324010EB9
:10133800638807008325010113050D00EF30002A9B
:101348009308C110130B040083470B00E39E07DCCE
:101358008327C10E638407006F1050328357CC0077
:1013680093F70704638407006F2000238320C11EBE
:101378000324811E0325C1008324411E0329011E65
:101388008329C11D032A811D832A411D032B011DA9
:10139800832BC11C032C811C832C411C032D011C95
:1013A800832DC11B1301011F6780000093050C00EA
:1013B80013050D00EF20C07A630405006F20C01DDF
:1013C8000357CC009306A0001377A701E314D7D0E6
:1013D8000317EC00E34007D08326410113060900F8
:1013E80093050C0013050D00EF20806B2326A10048
:1013F8006FF0DFF713050D00EF60801B83274500B2
:10140800138507002326F104EF80C0159307050014
:1014180013050D00938407002324F104EF6040199D
:1014280083278500232EF102638404006F10C01205
:10143800834404006FF0DFD783440400136A0A0270
:101448006FF01FD7B3046441E31064D183470400ED
:101458006FF05FD31306410E93050C0013050D00C2
:10146800EFA0D053E31C05EE9308C1106FF09FD096
:1014780093778A0093880C00638407006F10C0126A
:10148800832741011305010B2328910193877700D6
:1014980093F787FF83A5070003A647009387870074
:1014A800232AF100EF2091638327010B8328010190
:1014B8002328F10E8327410B232AF10E8327810B62
:1014C800232CF10E8327C10B232EF10E1305010FD8
:1014D80023281101EF6000072326A10C93072000A1
:1014E800832801016314F5006F10C04F93071000A3
:1014F8006314F5006F104064930710066394F400BA
:101508006F20401C930710046394F4006F101019A7
:1015180093FBF4FD9307F0FF232271056394FD000C
:101528006F200028930770046394FB006F20001E4F
:101538000323C10F23244103032E010F832E410FE0
:10154800032F810F93670A10635403006F20003E36
:10155800232C0104138A0700232801009307600441
:101568006394FB006F1090699307500423281105BA
:101578006384FB006F10906013891D00930A010BB0
:10158800930609001308C10D9307010D1307C10C39
:101598001306200093850A0013050D002328C10BAC
:1015A8002320C105232AD10B2322D103232CE10BAD
:1015B8002320E103232E610A232E6100EF40104F00
:1015C8000323C101032F0102832E4102032E0104CC
:1015D80083280105130B050033092501930C010A23
:1015E80093850C0013850A00232E11012328C10BB3
:1015F800232AD10B232CE10B232E610A2320010A75
:101608002322010A2324010A2326010AEF00411F8D
:101618008328C10113070900630205020327C10DCE
:10162800637E27019306000393071700232EF10C0E
:101638002300D7000327C10DE36827FFB3076741DD
:101648002320F1020327C10C93077004232EE10025
:10165800032741046314F7006F10D04303274104A4
:10166800930760046314F7006F10D0678327C101E4
:1016780003274104930510049387F7FF2326F10CF1
:1016880093F6F40F130600006318B7009386F6006C
:1016980093F6F60F13061000230AD10C9306B00236
:1016A80063DA07000327C101930710009306D002ED
:1016B800B387E740A30AD10C9306900063C4F600F1
:1016C8006F20C0281308310E130508001306A00068
:1016D800130E300633E7C70293050500938607000B
:1016E8001305F5FF13070703A38FE5FEB3C7C7026A
:1016F800E342DEFE9387070313F6F70FA30FC5FE39
:101708009387E5FF63E407016F2040379306610D77
:101718006F00800003C607002380C6009387170068
:1017280093861600E39807FF9307510EB387B740D7
:101738001307610DB307F7009306410DB387D74030
:10174800232CF1020327010283268103930710004B
:10175800B30CD70063C4E7006F2040298327C10278
:10176800B38CFC008327810293CAFCFF93DAFA4109
:1017780013FAF7BF136A0A10B3FA5C0123240102B3
:1017880023220102232E0100832781056394070089
:101798006F1090379307D002A303F10C930D00004C
:1017A800938A1A006FF0DFA81306410E93050C0008
:1017B80013050D00EFA0901EE31805068327C10E40
:1017C8009308C1106FF05FAC832601030327C102A1
:1017D8001306700023A0D8008326810EB307F700F4
:1017E80023A2E800938616002326F10E2324D10EA7
:1017F800938888006354D6021306410E93050C00A3
:1018080013050D00EFA09019E31005028325C10C04
:101818008327C10E8326810E9308C11063D4050067
:101828006F105058032701029386160023A0680101
:10183800B307F70023A2E8002326F10E2324D10ED4
:1018480013077000E35CD7AA1306410E93050C003A
:1018580013050D00EFA090146318057C8327C10EB3
:101868009308C1106FF0DFA9930600010327810ECA
:1018780063C496006F109051B7560180938E06C9C5
:1018880013090001130A7000138B0E006F00C000CB
:10189800938404FF6356990493870701130717007D
:1018A80023A0680123A228012326F10E2324E10E98
:1018B80093888800E35EEAFC1306410E93050C004A
:1018C80013050D00EFA0900D63100576938404FFB7
:1018D8008327C10E0327810E9308C110E34E99FA9E
:1018E800930E0B00B38797001307170023A0D801A6
:1018F80023A298002326F10E2324E10E93067000FC
:10190800E3D8E6A01306410E93050C0013050D005D
:10191800EFA0D008631A05708327C10E6FF05F9F90
:1019280013050D00EF2090346FF0CFF40327410129
:1019380093880C00A303010C8327070013074700B3
:10194800232AE1002306F114930A1000930C1000D7
:10195800130BC1146FF09F8C83274101A303010C63
:1019680093880C0003AB070013894700E30E0B5A5A
:101978009307F0FF6394FD006F10001013860D00AD
:101988009305000013050B00232A9101EF60C05B4B
:101998002328A10083284101631405006F10D0316A
:1019A80083270101232A210123280100B38C6741E1
:1019B8008347710C93CAFCFF93DAFA41232401028E
:1019C80023220102232E0100B3FA5C01930D0000CB
:1019D800E3800786938A1A006FF09F85834404008A
:1019E800136A4A006FF0CFFC8326410193770A02FD
:1019F80093880C0003A7060093864600232AD1008B
:101A0800E39E073693770A01638407006F10C005C9
:101A180093770A04638407006F10C03F137A0A2083
:101A280063140A006F1040048327C100130B0400DD
:101A38002300F7006FF05F91834404009307C0060A
:101A4800E384F44C136A0A016FF08FF6032741010F
:101A5800B787FFFF93C707832314F10C9307470049
:101A6800232AF10003290700B7570180938747AF5E
:101A780093880C00232AF102930C0000936B2A0030
:101A88009307200093048007A303010C1307F0FFBA
:101A98006386ED203367990113FAFBF7631E071E6F
:101AA80063940D266390071C93FC1B00130B011B0A
:101AB800E39C0C28938A0C0063D4BC01938A0D0024
:101AC8008347710C232801002324010223220102E9
:101AD800232E0100E39007F06FF08FF58344040094
:101AE80093078006E38AF442136A0A046FF04FEC06
:101AF8009307B00283440400A303F10C6FF04FEB8B
:101B080083440400136A0A086FF08FEA83440400D0
:101B180013071400639474016F105072938604FDC8
:101B280013040700930D000063E6DAE88344040019
:101B380093972D00B387B70193971700B38DD700FC
:101B4800938604FD13041400E3F2DAFE6FF08FE6C7
:101B5800832741018344040083A907009387470032
:101B6800232AF10063D609E4B3093041136A4A0015
:101B78006FF00FE483440400136A1A006FF04FE318
:101B88008347710C83440400639407E293070002BF
:101B9800A303F10C6FF0CFE193880C00136A0A01DC
:101BA80093770A02E38E070C83274101138B770092
:101BB800137B8BFF03290B00832C4B0093078B00AF
:101BC800232AF100937BFABF930700006FF0DFEB45
:101BD80093880C00936B0A0193F70B02E388070CB8
:101BE80083274101138B7700137B8BFF93078B00AF
:101BF800232AF10003290B00832C4B0093071000C4
:101C08006FF09FE883440400136A8A006FF04FDA8C
:101C180093880C00136A0A0193770A02E380070C81
:101C280083274101138B7700137B8BFF83274B009E
:101C380003290B0013078B00232AE100938C07006C
:101C4800E3C6070C9307F0FF930B0A006384FD02B9
:101C5800B3679901937BFAF7639E070063920D02BD
:101C6800138A0B00930D0000930C0000130B011B4B
:101C78006FF05FE4E3920C3A93079000E3EE2739A4
:101C880013090903A307211B138A0B00930C1000E7
:101C9800130BF11A6FF01FE2930B0A0013071000E1
:101CA800E38AE7FC13072000638CE706130B011B8C
:101CB8001397DC0193777900135939009387070349
:101CC8003369270193DC3C00A30FFBFE33679901BE
:101CD80013060B00130BFBFFE31C07FC93F61B001A
:101CE800638A0606930600036386D7061306E6FF93
:101CF8009307011BA30FDBFEB38CC740138A0B00AD
:101D0800130B06006FF01FDB130710006394E70046
:101D18006F10D01413072000930B0A00E398E7F81C
:101D280083264103130B011B9377F900B387F60051
:101D380003C70700135949009397CC0133E92701DA
:101D480093DC4C00A30FEBFEB3679901130BFBFF69
:101D5800E39C07FC9307011BB38C6741138A0B00B4
:101D68006FF05FD59306500663DC962C8326010F2F
:101D78009305010A1305010B2328D10A8326410F75
:101D8800232211052320F104232AD10A8326810F57
:101D98002320010A2322010A232CD10A8326C10FFA
:101DA8002324010A2326010A232ED10AEFF0502505
:101DB80083270104832841046318054A0327810EF9
:101DC800B75601809386C68C23A0D8009387170046
:101DD800930610001307170023A2D8002326F10E3C
:101DE8002324E10E9306700093888800E3C6E63A40
:101DF8000327C10C83260102635CD7720327010302
:101E08008326C1029388880023ACE8FE0327810E4D
:101E1800B387D70023AED8FE130717002326F10E89
:101E28002324E10E93067000E3C0E60C03270102A9
:101E38009304F7FF635690CC930600010327810EA5
:101E4800E3DC963613090001930C70006F00C000A4
:101E5800938404FFE3529936832681009387070110
:101E68001307170023A0D80023A228012326F10E68
:101E78002324E10E93888800E3DCECFC1306410E72
:101E880093050C0013050D00EFA04031631E0518E3
:101E98008327C10E0327810E9308C1106FF05FFBE3
:101EA80033895941635220C3130600018326810EEA
:101EB80063542607130E0001930B70006F00C000D7
:101EC800130909FF635A2E05032781009387070129
:101ED8009386160023A0E80023A2C8012326F10E4A
:101EE8002324D10E93888800E3DCDBFC1306410E23
:101EF80093050C0013050D00EFA0402A6316051288
:101F0800130E0001130909FF8327C10E8326810ED2
:101F18009308C110E34A2EFB03278100B3872701EA
:101F28009386160023A0E80023A228012326F10E99
:101F38002324D10E13067000938888006356D6B800
:101F48001306410E93050C0013050D00EFA00025A4
:101F5800631C050C8327C10E9308C1106FF0CFB620
:101F6800130600018326810E6352B607930B000106
:101F7800130970006F00C000938D0DFF63D8BB0577
:101F880003278100938707019386160023A0E800A2
:101F980023A278012326F10E2324D10E93888800EA
:101FA800E35CD9FC1306410E93050C0013050D00E4
:101FB800EFA0C01E631A0506938D0DFF8327C10E7F
:101FC8008326810E9308C110E3CCBBFB0327810055
:101FD800B387B7019386160023A0E80023A2B801AF
:101FE8002326F10E2324D10E13067000938888004F
:101FF8006350D6AE1306410E93050C0013050D0071
:10200800EFA0C019631205028327C10E9308C110FF
:102018006FF00FAC1306410E93050C0013050D006D
:10202800EFA0C017630205B0832B010163880BB2D0
:1020380093850B0013050D00EF20405A6FF00FB287
:102048008326810E938C1700832701021306100044
:1020580023A0680193841600138988006356F63814
:102068009307100023A2F8002326910F2324910E32
:102078009307700063CE97748327C1020327010377
:1020880093841400B38CFC002322F9002320E90078
:102098002326910F2324910E9307700013098900BA
:1020A80063CA97748327010F138614009305010AE6
:1020B8002328F10A8327410F1305010B232EC100A2
:1020C800232AF10A8327810F2320010A2322010AE8
:1020D800232CF10A8327C10F2324010A2326010A8E
:1020E800232EF10AEFF0C0710326C10183270102F4
:1020F8009308890093060600938DF7FF630A05305D
:1021080013071B00B38CBC012320E9002322B9016B
:102118002326910F2324C10E9307700063CCC75068
:102128009307090193862400138908009388070000
:10213800032681031307410D2320E900B307960105
:102148002322C9002326F10E2324D10E1307700081
:102158006358D79A6FF04FEF375701801306000185
:102168008326810E930E07C9635C06092320810428
:102178002322910413040D0093040C00130E000194
:1021880093027000130C0800138D0E006F00C0003E
:10219800130C0CFF635A8E0593870701938616006C
:1021A80023A0A80123A2C8012326F10E2324D10EBF
:1021B80093888800E3DED2FC1306410E9385040061
:1021C80013050400EF90907D6312057A130E000149
:1021D800130C0CFF8327C10E8326810E9308C110B0
:1021E80093027000E34A8EFB13080C00930E0D0057
:1021F800138C0400130D04008324410403240104F8
:10220800B38707019386160023A0D80123A20801EB
:102218002326F10E2324D10E13067000938888001C
:102228006344D6006FF0CF821306410E93050C006D
:1022380013050D00EF909076E31805DE8327C10E95
:102248009308C1106FF0CF801306410E93050C0060
:1022580013050D00EF909074E31805DC8327C10E79
:102268009308C1106FF0CF858325C10C635CB066FD
:102278000327C101832601029304070063C2E638DD
:10228800635690028326810EB387970023A06801C6
:102298009386160023A298002326F10E2324D10E3C
:1022A8001306700093888800E342D63293C6F4FF81
:1022B8000327C10193D6F641B3F4D400B304974081
:1022C800634490480327C10193760A40B30DEB009D
:1022D800E398060C8324C10C0327010263C6E400BB
:1022E80093761A00E3880630832601030327C10288
:1022F8001306700023A0D8008326810EB387E70059
:1023080023A2E800938616002326F10E2324D10E7B
:10231800938888006354D6006F10801783260102C3
:102328003307DB00B38496403307B74113890400B1
:102338006354970013090700635820030327810E8D
:10234800B387270123A0B8011307170023A2280188
:102358002326F10E2324E10E93067000938888004B
:1023680063D4E6006F10801C1347F9FF1357F74139
:102378003377E900B384E440634490006FE05FF88A
:10238800930600010327810E63D8966213090001A2
:10239800930C70006F00C000938404FF635E996023
:1023A80083268100938707011307170023A0D8000D
:1023B80023A228012326F10E2324E10E9388880006
:1023C800E3DCECFC1306410E93050C0013050D002D
:1023D800EF90D05CE31A05C48327C10E0327810E52
:1023E8009308C1106FF05FFB93771A00E39A07C652
:1023F80023A2C8002326910F2324910E930770006F
:1024080063CA972293862600938808016FF05FD2EB
:10241800E350B0D3130700016344B7016F10806124
:10242800130B7000930406006F000001938D0DFFDD
:10243800635EB71D9384140083278100938C0C017D
:102448002322E9002320F9002326910F2324910E4B
:1024580013098900E35C9BFC1306410E93050C00ED
:1024680013050D00EF909053E31005BC832CC10EAB
:102478008324810E1309C110130700016FF01FFB9D
:102488008326410193770A01138746006392071652
:1024980093770A046384076883274101930C00003B
:1024A800232AE10003D907006FF0CFF18326410109
:1024B80093F70B0113874600639E070C93F70B04F1
:1024C800638E076083274101930C0000232AE100F3
:1024D80003D90700930710006FF00FDB8326410133
:1024E80093770A0113874600639A070E93770A04C5
:1024F8006386076083274101232AE10003990700C7
:10250800935CF94193870C0063DE07F2B33720012F
:10251800B30C9041B38CFC409307D002A303F10C99
:1025280033092041930B0A00930710006FF00FD670
:1025380013771A00631407006FE09FDC6FF01F8C9D
:1025480093880C006FF04FED93070003A307F11A6F
:10255800130BF11A6FF00FD68327C10383440400CD
:10256800639407006FE0DFC483C707006394070024
:102578006FE01FC4136A0A406FE09FC38326C1003F
:10258800130B040093D7F6412320D7002322F7002A
:102598006FE09FDB03A90600930C0000232AE100EB
:1025A800930710006FF04FCE0327410183270700E0
:1025B80013074700232AE10083A5070003A6470065
:1025C80083A6870083A7C7002328B10E232AC10E3C
:1025D800232CD10E232EF10E6FE05FEF03A9060026
:1025E800232AE100935CF94193870C006FF04FE5D3
:1025F80003A90600930C0000232AE1006FF08FDC8A
:1026080093840600E34090C86FF05FCA9386140075
:102618001307890083278100B38CBC012322B901E9
:102628002320F9002326910F2324D10E930770004D
:1026380063DED7741306410E93050C0013050D00D5
:10264800EF90D035E312059E8326810E832CC10EB0
:1026580093084111938616001309C1106FF05FADFE
:1026680093880C00930B0A006FF00FD7B7570180BF
:10267800938747AF93880C00232AF10293770A02C5
:102688006388071283274101138B7700137B8BFF25
:1026980003290B00832C4B0093078B00232AF1009E
:1026A80093771A00638E0700B3679901638A07005E
:1026B800930700032304F10CA304910C136A2A0066
:1026C800937BFABF930720006FF00FBCB7570180C8
:1026D800938787B093880C00232AF1026FF01FFAC2
:1026E80093880C006FF0CFCB1306410E93050C00B6
:1026F80013050D00EF90902AE31805928327C10E69
:102708009308C1106FF08FF283441400136A0A0211
:10271800130414006FE0DFA983441400136A0A202D
:10272800130414006FE0DFA893076000938C0D007A
:1027380063EEB76B37570180938A0C00232A210177
:10274800130BC7B16FE09FAD130600018326810EFE
:1027580063549640930C0001930D70006F00C00005
:10276800938404FF63DA9C3E032781009387070163
:102778009386160023A0E80023A298012326F10ED1
:102788002324D10E93888800E3DCDDFC1306410E78
:1027980093050C0013050D00EF905020E3160588F3
:1027A8008327C10E8326810E9308C1106FF05FFB4B
:1027B8008326410193770A01138746006380071C2B
:1027C80003A90600930C0000232AE1006FF05FEDD7
:1027D8001306410E93050C0013050D00EF90101C15
:1027E800E3140584832CC10E8324810E1309C110C0
:1027F8006FF09F881306410E93050C0013050D001A
:10280800EF90D019E3120582832CC10E8324810E28
:102818001309C1106FF01F89130B011B93070000E8
:1028280023288100232E910013040B002322310357
:10283800130B0C009304090093890C0013FA0B4046
:10284800832CC103930AF00F138C08001389070027
:102858006F0040021306A0009306000013850400D1
:1028680093850900EFD0502BE38A092A93040500C9
:10287800938905001306A000930600001385040041
:1028880093850900EFD0906C13050503A30FA4FEF0
:10289800130919001304F4FFE30E0AFA83C60C00A7
:1028A800E31AD9FAE30859FB6392094A930790009F
:1028B80063EE974893080C009307011B130C0B0059
:1028C800130B0400232E91038324C10183294102A1
:1028D8000324010123202103B38C6741138A0B00D1
:1028E8006FF04F9D8326810E375601801306C68CE4
:1028F80023A0C800938717001306100093861600BC
:1029080023A2C8002326F10E2324D10E130670003B
:10291800938888006344D648638405006FE0DFEA43
:102928000327010293761A00B3E6E60063940600D3
:102938006FE01F9D832601030327C1021306700061
:1029480023A0D8008326810EB307F70023A2E8004E
:10295800938616002326F10E2324D10E6354D60045
:102968006FE09FE9938888006FE0DFEB832B01011C
:10297800130D0400138C04006FF04FEB93770A04D7
:102988006380071483274101930C0000232AE10088
:1029980003D907006FF0DFD01306410E93050C0032
:1029A80013050D00EF90807F631005E88327C10EA3
:1029B8009308C1106FF0CFC383268100B3879700B7
:1029C80023A2980023A0D800130717002326F10E8E
:1029D8002324E10E9306700063C4E6006FE01F92A3
:1029E8006FE09FE68327010F9305010A1305010B8A
:1029F8002328F10A8327410F2320010A2322010AF1
:102A0800232AF10A8327810F2324010A2326010A96
:102A1800232CF10A8327C10F232EF10AEFE0507F00
:102A280083280101E34005268347710C13077004CE
:102A38006358973837570180130B87AE2328010056
:102A48002324010223220102232E0100137AFAF71C
:102A5800930A3000930C3000930D00006384070044
:102A68006FE05FF76FE0CFFC8327C100130B040012
:102A78002320F7006FE05F8D13050B0023209105DD
:102A8800EF60502E8347710C934AF5FF93DAFA41B1
:102A9800232A2101232801002324010223220102E1
:102AA800232E010083280104930C0500B37A5501F5
:102AB800930D0000638407006FE0DFF16FE04FF7CC
:102AC80093770A206382073A83274101930C000019
:102AD800232AE10003C907006FF09FBC93F70B207E
:102AE8006388073683274101930C0000232AE100FD
:102AF80003C90700930710006FE01FF993770A20B6
:102B0800638C073283274101232AE10003890700E8
:102B1800935CF94193870C006FF08F9293770A20AA
:102B28006382073083274101930C0000232AE100C8
:102B380003C907006FF00F898327C10F63CA0734E1
:102B48008347710C13077004E35C971C37570180A7
:102B5800130B07AF6FF09FEE03278100B387970031
:102B68009386160023A0E80023A298002326F10EDE
:102B78002324D10E13067000938888006354D6F47A
:102B88001306410E93050C0013050D00EF9000612C
:102B9800631C05C88327C10E9308C1106FF08FF21C
:102BA80003270102832C4102232E410123208104A3
:102BB800232231052322510383298102232461031F
:102BC800B30BEB000324C103032A8104832AC10445
:102BD8009304700013090001130B0C0063880C08A0
:102BE800639809081304F4FF938CFCFF0327810EF4
:102BF800B387470123A058011307170023A24801F0
:102C08002326F10E2324E10E9388880063CEE40E78
:102C1800834604003386BB41138C06006354D600F8
:102C2800130C0600635680038326810EB387870141
:102C380023A0B8019386160023A288012326F10E4B
:102C48002324D10E63C2D40E8346040093888800DF
:102C58001346FCFF1356F6413377CC00338CE6401D
:102C6800634C8001B38DDD00E39C0CF6638A095E3A
:102C78009389F9FF6FF09FF78326810E63488901D6
:102C88006F008005130C0CFF63588905032781002A
:102C9800938707019386160023A0E80023A2280142
:102CA8002326F10E2324D10E93888800E3DCD4FC7C
:102CB8001306410E93050B0013050D00EF90004E0F
:102CC80063140566130C0CFF8327C10E8326810E3F
:102CD8009308C110E34C89FB03278100B387870160
:102CE8009386160023A0E80023A288012326F10E6C
:102CF8002324D10E63C0D4668346040093888800D9
:102D0800B38DDD006FF05FF61306410E93050B00DF
:102D180013050D00EF908048631805608327C10EE6
:102D28009308C1106FF0DFEE1306410E93050B00F8
:102D380013050D00EF9080466318055E8346040076
:102D48008327C10E9308C1106FF09FF08327810479
:102D58008325C104130900003304F44013860700D7
:102D680013050400EF60D00883C51C001306A000FB
:102D7800930600003338B0001385040093850900DA
:102D8800B38C0C01EFD040596FF05FAE93861600FC
:102D980093088700130907006FF08FB91306410ED7
:102DA80093050C0013050D00EF90403F631E05A628
:102DB8008325C10C8327C10E9308C1106FF0DFB5BE
:102DC80037570180130B47AE6FF05FC71306410EEC
:102DD80093050C0013050D00EF90403C631605A405
:102DE8008327C10E9308C1106FF04FCC930C60007D
:102DF8006FF05F94832601023307DB00B3849640AB
:102E08003308B74113890400635098D613090800A2
:102E18006FF08FD58327C100130B04002310F70030
:102E28006FE08FD283274101930C0000232AE10031
:102E380003A907006FE01FD983274101232AE10076
:102E480003A90700935CF94193870C006FE05FDFEB
:102E580083274101930C0000232AE10003A90700FE
:102E6800930710006FE05FC283274101930C0000B5
:102E7800232AE10003A907006FF09F821306410E81
:102E880093050C0013050D00EF9040316FE00FCD56
:102E98009307D002A303F10C6FF0DFCA9307000376
:102EA8002304F10C9307800513672A00A304F10C8F
:102EB8002324E1029307300623280100130BC114D1
:102EC800E3C4B7030323C10F93FBF4FD2322710569
:102ED800232C0104032E010F832E410F032F810F92
:102EE800136A2A10634E034493071006E38EF40A0C
:102EF800930710046384F4006FE04FE6930A010B14
:102F080013850A00232A11052328C10B232AD10B74
:102F1800232CE10B232E610AEF10815B1306C10CF1
:102F2800EF600025138605009305050013850A0048
:102F3800EF10C13A8327010B930C010A1309010909
:102F48002328F1088327410B13060108930509007C
:102F5800232AF1088327810B13850C002320C10441
:102F6800232CF1088327C10B232001082322010801
:102F7800232EF108B707FC3F2326F1082324010874
:102F8800EFE0503D0328010A032E410A832E810AEF
:102F9800032FC10A93850C0013850A002328010B0F
:102FA80023280105232AC10B2322C103232CD10B7B
:102FB8002320D103232EE10B232EE1012320010A34
:102FC8002322010A2324010A2326010AEFE05003E1
:102FD800032FC101832E0102032E4102032801059C
:102FE8008328410563160500930710002326F10C7A
:102FF800B7570180938787B02322F1029386FDFF9C
:10300800232E4105232291062326B107232AA1074F
:10301800232C810723208106232431072328110725
:10302800130C0B00938B0600232E6107130D080069
:10303800930D0E0093840E00130A0F006F00800496
:1030480093850C0013850A002320C102232EF10169
:10305800232CF10B232EC10A2328610B232A310BC1
:103068002320010A2322010A2324010A2326010A14
:10307800EFE00079832FC10103260102938BFBFF48
:103088006302050EB70703401306090093850C0079
:1030980013850A00232EF1082320A10B2322B10B4C
:1030A8002324910A2326410B23280108232A0108F7
:1030B800232C0108EFE0102A13850A00EF00D17BCA
:1030C800930505001304050013850A008329010BE5
:1030D8008324410B032B810B032AC10BEF10010B37
:1030E8000327010B03260104930509002320E108A7
:1030F8000327410B13850C00232831092322E108FB
:103108000327810B232A9108232C61092324E10832
:103118000327C10B232E41092326E108EFF0D02312
:1031280083274102032B010A8329410A3387870039
:1031380003470700832F810A0326C10A232A810532
:103148002300EC00232871059307F0FF130C1C00E3
:10315800130D0B00938D090093840F00130A0600CA
:10316800E390FBEE8328010793030B009382090089
:103178003709FE3F93850C0013850A0023201103AD
:10318800232E8100032AC105832441060324010656
:103198002328710A23227106232A510A2320510663
:1031A800232CF10B232EF105232EC10A2320C10461
:1031B8002320010A2322010A2324010A2326210BA2
:1031C800EFE0C070930B0C00832DC106032D41075F
:1031D800032C8107032BC107832981068328010259
:1031E8006342A0488323410683220106832FC10539
:1031F8000326010493850C0013850A002328710A0D
:10320800232A510A232CF10B232EC10A2320010A59
:103218002322010A2324010A2326210BEFE0405E22
:1032280083280102631805008327C10193FC170056
:10323800639A0C428327010513060003938617003F
:10324800B386DB0063C80700938B1B00A38FCBFEFC
:10325800E39C76FFB3876B412320F1026FE08FBEBA
:1032680003270102130C0B00032B8102232E81027A
:10327800032AC101B306EB00032401048329410496
:10328800832A410263E4B6016FF0CF84938D060070
:103298006FF04F840327C1019307D0FF6344F70001
:1032A80063DAED009384E4FF93F7F4FD2322F1043D
:1032B8006FE0CFBB832701020327C1016340F72AD0
:1032C80083278102930C070093F717006386070092
:1032D8008327C102B30CF7008327810293F70740C5
:1032E800638607008327C1016342F05C93CAFCFF31
:1032F80093DAFA41B3FA5C019304700623240102BD
:10330800232201026FE04FC88347710C930D000020
:10331800638407006FE00FEC6FD09FF19307900074
:1033280063E697D46FF00FD9832B0101130C0B00C0
:103338006FE0DFCF2324410323280100130A09008B
:10334800B707008033C367009307D002232CF1042A
:103358006FF09FB91306410E93050B0013050D007E
:10336800EF80D063E31205FC834604008327C10E77
:103378009308C110B38DDD006FF01F8F930A010B06
:103388009307010D1308C10D1307C10C93860D0097
:103398001306200093850A0013050D002328C10B8E
:1033A8002320C105232AD10B2322D103232CE10B8F
:1033B8002320E103232E610A232E6100EF20106FE2
:1033C800930770040323C101032F0102832E4102D6
:1033D800032E010483280105130B05006390FB08E5
:1033E8008327810293F717006396072E93077004CB
:1033F8000327C10D2322F1046FE04FA4930A010BA8
:103408001308C10D9307010D1307C10C93860D0016
:103418001306300093850A0013050D0023281105B3
:103428002328C10B2320C105232AD10B2322D10332
:10343800232CE10B2320E103232E610A232E6100B4
:10344800EF20D0660323C101032F0102832E41021E
:10345800032E010483280105130B0500930760045C
:103468003309BB01639EFB2683460B0093070003C9
:103478006386F650930C010A8327C10C3309F900BF
:103488006FE00F969307D002A303F10C6FF00FDAE9
:103498001306410E93050C0013050D00EF80105024
:1034A800630405006FE05FB88324C10C8327C10E55
:1034B8009308C1106FE09FE68347710C232A21010E
:1034C8002324010223220102232E0100938A0D00E6
:1034D800938C0D00930D0000638407006FE08FCF7D
:1034E8006FD01FD5832781020327C10193F71700E7
:1034F800B3E7B7016356E05063900744832CC101DA
:10350800930460068327810293F707406392073A82
:1035180093CAFCFF93DAFA41B3FA5C016FF01FDE3D
:1035280037570180130BC7AE6FF04FD11306410E0A
:1035380093050C0013050D00EF8050466304050049
:103548006FE09FAE8324C10C032701028327C10EBD
:103558009308C110B30497406FE01FE1832701026D
:103568000327C10293047006B38CE7008327C101C7
:10357800E34AF0F8B38CFC40938C1C0093CAFCFF20
:1035880093DAFA41B3FA5C016FF05FD7B75601805E
:10359800938E06C96FE00FB59307F0FF2326F1005D
:1035A8006FD0DFDC130600FFB304B04063D2C5065A
:1035B80013090001930C70006F00C000938404FF8E
:1035C800635899040327810093870701938616009F
:1035D80023A0E80023A228012326F10E2324D10EDC
:1035E80093888800E3DCDCFC1306410E93050C008D
:1035F80013050D00EF80903A630405006FE0DFA229
:103608008327C10E8326810E9308C1106FF01FFB1C
:1036180003278100B38797009386160023A0E8004C
:1036280023A298002326F10E2324D10E130670003E
:10363800635AD6B21306410E93050C0013050D000C
:10364800EF80D035630405006FE01F9E8327C10E0D
:103658008326810E9308C1106FE0CF9C930B0A005C
:103668006FE00FE28327410593860B00232EF10CB0
:103678008327410203C6FBFF83C5F7006310B60228
:1036880013050003A38FA6FE8326C10D9387F6FFBB
:10369800232EF10C03C6F6FFE386C5FE930516003C
:1036A8001305900393F5F50F6306A600A38FB6FEE6
:1036B8006FF05FBA8327410283C5A700A38FB6FEC8
:1036C8006FF05FB9930700032304F10C9307800799
:1036D8006FF08FFD930770043309BB012322F104B7
:1036E800930C010A6FD0DFEF93851D0013050D00C1
:1036F80023281101EF40C00B83280101130B05009B
:10370800630005362328A1006FF0CFFB63940D00FA
:10371800930D10000323C10F032E010F832E410FB9
:10372800032F810F13690A10E34603C0930A010BA4
:103738001308C10D9307010D1307C10C93860D00E3
:103748001306200093850A0013050D002322110596
:103758002328C10B2320C105232AD10B2322D103FF
:10376800232CE10B2320E103232E610A232E610081
:10377800EF20D0330323C10123244103032F010287
:10378800832E4102032E010483284104130B0500F4
:10379800130A0900232C0104232801006FF05FC4D9
:1037A800930D60006FD0DFD8930A010B13850A00D0
:1037B800232A11052328C10B232AD10B232CE10B23
:1037C800232E610AEF00D1501306C10CEF50501A96
:1037D800138605009305050013850A00EF001130D4
:1037E8008327010B930C010A130901092328F10807
:1037F8008327410B1306010893050900232AF108C2
:103808008327810B13850C002320C104232CF10886
:103818008327C10B2320010823220108232EF10846
:10382800B707FC3F2326F10823240108EFE0803284
:103838000328010A032E410A832E810A032FC10A95
:1038480093850C0013850A002328010B2328010502
:10385800232AC10B2322C103232CD10B2320D103FC
:10386800232EE10B232EE1012320010A2322010A42
:103878002324010A2326010AEFD09078032FC101DF
:10388800832E0102032E41020328010583284105E6
:1038980063160500930710002326F10CB757018023
:1038A800938747AF2322F1026FF04FF59304700618
:1038B8000326C1039306F00F83470600638AD71ACD
:1038C8000327C101130500009305000063DEE7002C
:1038D8003307F74083471600638407049385150070
:1038E80013061600E394D7FE232EC102232EE1000F
:1038F8002322B1022324A102032781028327410244
:10390800B387E70003278104B387E702B38C9701E5
:1039180093CAFCFF93DAFA41B3FA5C016FD0DFE691
:1039280083470600130515006FF0DFFB232801000D
:10393800138A07006FF0DFA08327C1029304600693
:10394800B30CF700B38CBC016FF0DFBB9306610DBD
:103958006318060093060003230BD10C9306710D20
:103968001307011B938707033386E6402380F6007D
:103978009307D60D232CF1026FD0DFDC930C010ADC
:1039880093850C0013850A00232811052328C10BF1
:103998002320C105232AD10B2322D103232CE10B99
:1039A8002320E103232E610A232E61002320010A2C
:1039B8002322010A2324010A2326010AEFD0506496
:1039C8000323C101032F0102832E4102032E0104A8
:1039D80083280105E30205AA93071000B387B741BE
:1039E8002326F10C3309F9006FD09FBF832781028A
:1039F80093F71700639407006FD0DFD66FD01FD6F8
:103A0800639A0700930A100093046006930C100051
:103A18006FF0DF8E8327C10293046006938C170032
:103A2800B38CBC0193CAFCFF93DAFA41B3FA5C0188
:103A38006FF0DF8C138708006FE0DFBD832741013B
:103A480083AD07009387470063D40D00930DF0FF03
:103A580083441400232AF100130407006FD04FF5A4
:103A68008357CC0093E707042316FC006FD01F8F01
:103A780023240102232201026FF01FE8930720008C
:103A8800232CF1026FD01FCC9307050003A5C12595
:103A98009306060013860500938507006FD0CFD5DF
:103AA80083D7C50003AE450603D3E50083A8C50147
:103AB80003A84502130101B893F7D7FF1307004085
:103AC800232C8146231AF10013840500930701076C
:103AD80093058100232A914623282147232E114646
:103AE800130905002326C107231B610023221103A4
:103AF800232601032324F100232CF1002328E100CD
:103B0800232EE10023200102EFD00FCF93040500FC
:103B1800635C05028357410193F707046388070034
:103B28008357C40093E707042316F4008320C14792
:103B3800032481470329014713850400832441474F
:103B480013010148678000009305810013050900EF
:103B5800EF000058E30005FC9304F0FF6FF09FFBB3
:103B680083A7C125130101FF23248100232291008B
:103B780023261100930405001384050063860700BB
:103B880003A787036300070E0317C40093170701F1
:103B98009376870093D70701638006048326040180
:103BA8006380060613F6170063040608032644011B
:103BB80023240400130500003306C040232CC4004E
:103BC800638606088320C100032481008324410002
:103BD800130101016780000093F607016384060C56
:103BE80093F7470063960708832604011367870045
:103BF800931707012316E40093D70701E39406FA05
:103C080013F6072893050020E30EB6F89305040081
:103C180013850400EF30D0270317C400832604015E
:103C28009317070193D7070113F61700E31006F857
:103C380013F627009305000063140600832544014A
:103C48002324B40013050000E39E06F693F7070843
:103C5800E38A07F6136707042316E4001305F0FF49
:103C68006FF05FF613850700EF0050006FF0DFF18B
:103C780083250403638E0500930704046388F50015
:103C880013850400EF0090150317C40023280402CD
:103C9800832604011377B7FD232204002320D400D0
:103CA8006FF0DFF49307900023A0F4001367070474
:103CB8002316E4001305F0FF6FF0DFF003A70125DA
:103CC80083278714638C070403A747001308F001B0
:103CD800634EE806131827006306050233830701BD
:103CE8002324C30883A88718130610003316E60098
:103CF800B3E8C80023A417192324D310930620007F
:103D08006304D5021307170023A2E700B38707014E
:103D180023A4B70013050000678000009307C714A9
:103D28002324F7146FF05FFA83A6C7181307170048
:103D380023A2E70033E6C60023A6C718B387070106
:103D480023A4B70013050000678000001305F0FFE7
:103D580067800000130101FD232C410103AA0125FE
:103D6800232021032326110203298A1423248102F4
:103D780023229102232E3101232A51012328610194
:103D8800232671012324810163000904130B050014
:103D9800938B0500930A10009309F0FF83244900D0
:103DA8001384F4FF6342040293942400B30499003B
:103DB80063840B0483A74410638077051304F4FF1E
:103DC8009384C4FFE31634FF8320C10203248102D5
:103DD80083244102032901028329C101032A8101A5
:103DE800832A4101032B0101832BC100032C81008D
:103DF80013010103678000008327490083A644005C
:103E08009387F7FF638E870423A20400E38806FAEA
:103E18008327891833978A00032C4900B377F70062
:103E280063920702E78006000327490083278A1464
:103E380063148701E304F9F8E38807F81389070096
:103E48006FF0DFF58327C91883A544083377F70097
:103E5800631C070013050B00E78006006FF0DFFC0A
:103E6800232289006FF09FFA13850500E78006007A
:103E78006FF09FFB8397C500130101FE232C81007F
:103E880023263101232E1100232A91002328210102
:103E980093F687001384050093090500639A0610BA
:103EA800371700001307078083A64500B3E7E7002C
:103EB8002396F5006354D01803278402630A070C7D
:103EC80083A409009396070123A0090013963701DC
:103ED8008325C40193D6060163480616930610008D
:103EE8001306000013850900E70007009307F0FF99
:103EF800630CF5188356C400032784028325C40184
:103F080093F64600638E0600832644008327040345
:103F18003305D540638607008327C4033305F5407E
:103F2800130605009306000013850900E700070043
:103F38009307F0FF631EF51003A709008317C40059
:103F4800630807169306D0016306D700930660013D
:103F58006314D70C8326040137F7FFFF1307F77F95
:103F6800B3F7E7002316F400232204002320D4002B
:103F78008325040323A09900638C05009307040498
:103F88006386F50013850900EF00406523280402C5
:103F9800130500008320C10103248101832441010A
:103FA800032901018329C100130101026780000070
:103FB80003A90501E30E09FC83A405001397070173
:103FC800135707011377370023A02501B384244131
:103FD800930700006314070083A745012324F40016
:103FE800634890006FF0DFFA3309A900E35290FAB2
:103FF800832744028325C40193860400130609001D
:1040080013850900E7800700B384A440E34EA0FCB1
:104018008357C4001305F0FF93E707048320C10109
:104028002316F4000324810183244101032901019B
:104038008329C100130101026780000003A7C5039B
:10404800E34CE0E66FF0DFF4032504056FF05FEB67
:104058008357C40037F7FFFF1307F77FB3F7E7006D
:10406800832604019397070193D707412316F40089
:10407800232204002320D40013973701E35A07EEC4
:104088002328A4046FF0DFEE83A70900E38407E682
:104098001307D0016388E702130760016384E7020E
:1040A8008357C40093E707042316F4006FF09FEECC
:1040B80037F7FFFF1307F77F83260401B3F7E700FD
:1040C8006FF0DFFA23A09900130500006FF09FEC52
:1040D800130101FE232C8100232E11001304050077
:1040E8006306050083278503638007028397C5005D
:1040F800639607028320C101032481011305000090
:1041080013010102678000002326B100EF0000368A
:104118008325C1008397C500E38E07FC13050400BF
:10412800032481018320C101130101026FF09FD490
:10413800930505006306050003A5C1256FF05FF927
:1041480003A50125B74500809385850D6F005003B1
:104158001305000067800000B7D500809385456B84
:104168006F001002130101FEB7470080232E1100D3
:10417800232C8100232A91002328210123263101A1
:1041880023244101232251012320610103244500F6
:1041980093870716232EF5021307C52E93073000C1
:1041A8002324E52E2322F52E2320052E93074000F5
:1041B800130905002326F400130680009305000068
:1041C80023220406232004002322040023240400BD
:1041D80023280400232A0400232C04001305C40503
:1041E800EFC01FCB379B008083248900B79A0080DB
:1041F800379A0080B7990080130B0B36938A4A3C94
:10420800130ACA449389494BB70701002320640362
:10421800232254032324440323263403232E840017
:104228009387970023A6F4001306800093050000E7
:1042380023A2040623A0040023A2040023A404004C
:1042480023A8040023AA040023AC04001385C40592
:10425800EFC01FC40324C900B707020023A06403EA
:1042680023A2540323A4440323A6340323AE9400B7
:10427800938727012326F400232204062320040021
:10428800232204002324040023280400232A0400F2
:10429800232C04001305C4051306800093050000B1
:1042A800EFC01FBF8320C1012320640323225403CE
:1042B8002324440323263403232E8400032481016A
:1042C80093071000232CF9028324410103290101DB
:1042D8008329C100032A8100832A4100032B01009E
:1042E80013010102678000001305000067800000C9
:1042F800130101FF23229100130680069384F5FF22
:10430800B384C402232021011389050023248100DA
:104318002326110093854407EF30804913040500D4
:10432800630005021305C50023200400232224018D
:104338002324A4001386840693050000EFC05FB50C
:104348008320C10013050400032481008324410055
:10435800032901001301010167800000130101FE18
:104368002328210103A9012523263101232E110029
:1043780083278903232C8100232A910093090500B0
:104388006386070A1309092E9304F0FF832749005F
:10439800032489009387F7FF63D807006F0000089C
:1043A80013048406638C97060317C4009387F7FFEA
:1043B800E31807FEB707FFFF9387170023220406B9
:1043C8002320040023220400232404002326F400CD
:1043D80023280400232A0400232C04001306800049
:1043E800930500001305C405EFC09FAA2328040203
:1043F800232A040223220404232404048320C10161
:1044080013050400032481018324410103290101C8
:104418008329C100130101026780000003240900F9
:10442800630C0400130904006FF05FF6130509001C
:10443800EFF05FD36FF01FF5930540001385090077
:10444800EFF01FEB2320A90013040500E31C05FC73
:104458009307C00023A0F9006FF05FFA03A50125B8
:10446800B7D500809385456B6F00805183278503FE
:1044780063840700678000006FF0DFCE678000006C
:1044880067800000678000006780000003A5C125E1
:10449800B7450080938585156F00404403A5C12565
:1044A800B74500809385052F6F004043130101FE37
:1044B80023263101232C8100232A9100232821015E
:1044C80023244101232E1100138A05001309050036
:1044D800938901CCEF30903403A78900B717000007
:1044E8001384F7FE832447003304444193F4C4FF44
:1044F800330494001354C4001304F4FF1314C400C9
:10450800634EF4009305000013050900EF40D050F6
:1045180083A78900B38797006308F502130509008C
:10452800EF3010308320C10103248101832441012D
:10453800032901018329C100032A81001305000012
:104548001301010267800000B305804013050900CC
:10455800EF40904C9307F0FF6308F5049387412FD1
:1045680003A7070083A68900B384844093E414005A
:10457800330487401305090023A2960023A087006F
:10458800EF30102A8320C1010324810183244101D3
:10459800032901018329C100032A810013051000A2
:1045A800130101026780000093050000130509004C
:1045B800EF40904603A789009306F000B307E54053
:1045C800E3DEF6F483A6012693E717002322F7001B
:1045D8003305D54023AAA12E6FF05FF4638405123A
:1045E800130101FF23248100232291001384050075
:1045F8009304050023261100EF3050220328C4FF3E
:10460800130784FF9377E8FF3306F700938501CCFF
:104618008326460003A5850093F6C6FF6306C51AE0
:104628002322D600137818003305D600631E080825
:10463800032384FF03284500330767408328870046
:10464800138581CCB387670013781800638EA8128E
:104658000323C70023A6680023241301630E081C44
:1046680093E617002322D7002320F6009306F01FB5
:1046780063E6F60A93F687FF9386860003A545004E
:10468800B386D50003A6060013D857009307100079
:10469800B3970701B3E7A700138586FF2326A70072
:1046A8002324C70023A2F50023A0E6002326E60062
:1046B800032481008320C100138504008324410062
:1046C800130101016F30D01503254500137515003E
:1046D800631C0502B387D700138581CC8326860027
:1046E80093E817003308F7006384A6160326C6006C
:1046F80023A6C6002324D600232217012320F8006E
:104708006FF0DFF66780000093E61700232ED4FED3
:104718002320F6009306F01FE3FEF6F493D69700E5
:10472800130640006368D60E93D667001388960375
:10473800138686031318380033880501832608007A
:10474800130888FF6304D81203A646001376C6FF31
:1047580063F6C70083A68600E318D8FE03A8C60040
:10476800232607012324D700032481008320C100C6
:104778002324E800138504008324410023A6E600CF
:10478800130101016F30D009631208148325C60094
:1047980003268600B387F600032481002326B6008B
:1047A80023A4C50093E617008320C1002322D70065
:1047B800138504003307F700832441002320F70002
:1047C800130101016F30D00513781800B387D700A3
:1047D80063100802032584FF3307A7408326C70018
:1047E80003268700B387A7002326D60023A4C60084
:1047F80013E6170083A641262322C70023A4E50059
:10480800E3E8D7EA83A5012913850400EFF01FCA5E
:104818006FF01FEA130640016374D60213064005C1
:104828006364D60693D6C7001388F6061386E60691
:10483800131838006FF05FF0B387D7006FF01FEAE6
:104848001388C6051386B605131838006FF0DFEE17
:1048580023AAE50023A8E5002326A7002324A70010
:10486800232217012320F8006FF09FE403A54500D9
:1048780013562640930710003396C7003366A600E8
:1048880023A2C5006FF0DFED13064015636CD60058
:1048980093D6F7001388860713867607131838000F
:1048A8006FF09FE913064055636CD60093D6270135
:1048B8001388D6071386C607131838006FF0DFE78A
:1048C8001308803F1306E0076FF01FE793E6170011
:1048D8002322D7002320F6006FF09FDD130101FE8D
:1048E80023282101232631012324410123225101B8
:1048F80023206101232E1100232C8100232A9100FB
:10490800138B0500930A052E130A00009309100063
:104918001309F0FF83A44A0003A48A009384F4FFD8
:1049280063C604028357C4009384F4FF63FCF90050
:104938008317E4001305040063862701E7000B00D2
:10494800336AAA0013048406E39E24FD83AA0A009E
:10495800E3920AFC8320C1010324810183244101DD
:10496800032901018329C100832A4100032B010087
:1049780013050A00032A8100130101026780000061
:10498800130101FD23202103232E3101232C410192
:10499800232A5101232861012326710123261102AC
:1049A8002324810223229102930A0500938B050098
:1049B800130B052E130A0000930910001309F0FFCA
:1049C80083244B0003248B009384F4FF63C8040200
:1049D8008357C4009384F4FF63FEF9008317E4004F
:1049E8009305040013850A0063862701E7800B00FE
:1049F800336AAA0013048406E39C24FD032B0B00EE
:104A0800E3100BFC8320C1020324810283244102AA
:104A1800032901028329C101832A4101032B0101D2
:104A2800832BC10013050A00032A81011301010326
:104A38006780000093064500930700001305A50151
:104A48003788FFFF6F00C001939717002390E60097
:104A5800939707019386260093D70701630ED50223
:104A680003D70600137617006304060093E71700C0
:104A78001357170013F62700B3650701E30606FC72
:104A8800939717002390B600939707019386260003
:104A980093D70701E316D5FC6780000093068501CC
:104AA80013070000130525006F00C0011317170036
:104AB8002390F600131707019386E6FF13570701A3
:104AC8006304D50483D706001396070113560641DD
:104AD800939717006354060013671700939707010D
:104AE80093D707011376270093E51700E30006FC28
:104AF800131717002390B600131707019386E6FFD4
:104B080013570701E310D5FC67800000130101FE6D
:104B1800370E0100231D0100231E01009385850126
:104B28009307C10113088100130EFEFF03D7050088
:104B38009387E7FF9385E5FF63180702239F07FE26
:104B4800E39607FF130646009306E10103D7070023
:104B58009387270013062600231FE6FEE398D7FE57
:104B680013010102678000003307A70283D82700DA
:104B780003D30700B376C701B3861601135707019D
:104B880093D80601330767003307170193580701C5
:104B98002391D7002390E700239F17FFE39807F995
:104BA8006FF05FFA130725018357050013052500E9
:104BB80063980700E31AE5FE13050000678000000C
:104BC8001305100067800000130101FF23229100E4
:104BD80083542501232481002326110093C7F4FF61
:104BE800139717011304050063160700EFF09FFBE6
:104BF80063180500B787FFFFB3C4F40023199400B6
:104C08008320C10003248100832441001301010192
:104C180067800000130101FF23248100035425014C
:104C2800232611009347F4FF13971701631A07000F
:104C3800EFF05FF793070500130500006394070082
:104C48001355F4008320C1000324810013010101DE
:104C58006780000083572501130101FD2324810289
:104C680093D7F70023229102232611022320210340
:104C7800232E3101B307F0402390F5008357250117
:104C8800378700001307F7FFB377F7002391F50084
:104C980093040500130405016382E7049387650004
:104CA800239205001305E5FF035704001304E4FFEE
:104CB80093872700239FE7FEE31885FE239C0500C2
:104CC8008320C102032481028324410203290102B3
:104CD8008329C101130101036780000003572501DF
:104CE8001389450033F7E700631CF7022326B10058
:104CF800EFF05FEB8325C10063040502938765002D
:104D0800239205001385C4FF035704001304E4FF2E
:104D180093872700239FE7FEE31885FE6FF05FFA6D
:104D28009389A50113092900231F09FEE39C29FF84
:104D38008320C10203248102832441020329010242
:104D48008329C101130101036780000083572501EE
:104D5800130101FB2324810493C7F7FF2322910445
:104D680023261104139717019304050013840500E3
:104D780063160700EFF01FE3631205088357240149
:104D880093C7F7FF1397170163040706930581007C
:104D980013850400EFF01FEC93054102130504008E
:104DA800EFF05FEB8355810003554102630CB504B6
:104DB8009307A100130761021306010283D60700B7
:104DC80093872700639A060883560700130727006E
:104DD80063940608E394C7FE130500008320C1040A
:104DE8000324810483244104130101056780000022
:104DF80013050400EFF01FDBE30A05F81305E0FFD5
:104E08006FF0DFFD133515000356A10083566102CC
:104E18003305A0401307A10093076102137525000D
:104E28001305F5FF9305C103938727001307270090
:104E3800631ED600E382B7FA0356070083D607003D
:104E48001307270093872700E306D6FEE3E8C6F892
:104E58003305A0406FF09FF813051000E38005F8B4
:104E68001305F0FF6FF09FF7130101FF23261100D0
:104E7800EFF05FD38320C100133515001301010142
:104E880067800000130101FE232C8100232A910072
:104E9800232E1100232821012326310193840500A4
:104EA8001304050063C4050A9307F0001386050080
:104EB80013054500930684019305F00063D4970217
:104EC8009307050003D7270093872700239FE7FE52
:104ED800E39AD7FE231C0400130606FFE3C2C5FEAF
:104EE80093F4F4009307700063D8970213078401C2
:104EF8009305240093070000835607001307E7FF74
:104F080013968600B3E7C7002311F70093D78600EE
:104F1800E314B7FE938484FF638A04009384F4FF48
:104F280013050400EFF09FB7E39A04FE1305000091
:104F38008320C10103248101832441010329010144
:104F48008329C1001301010267800000930710FF45
:104F58003309B04063DCF51293058501930900001D
:104F6800930645001306F000035784019387050054
:104F7800B3E9E90003D7E7FF9387E7FF2391E70049
:104F8800E39AD7FE23120400130909FFE34E26FD16
:104F9800930700FF130710FFB3879740130900001A
:104FA80063C4E40A3309F9009307700063D6270540
:104FB8009399090193D90941834784019305A40171
:104FC800B3E9F9009399090193D9090193070000FE
:104FD80003D60600938626001357860033E7E700BA
:104FE8009317860093970701239FE6FE93D707013F
:104FF800E390B6FE130989FF630C09068357840101
:105008001309F9FF1305040093F71700B3E93701F3
:10501800EFF05FA2E31409FE9397090193D70741C4
:105028006390070413950901135505018320C101F5
:105038000324810183244101032901018329C1003B
:10504800130101026780000013F907FF33092041AB
:105058003309F90093077000E3D027FB6FF05FF581
:105068009309100013950901135505016FF01FFCF2
:1050780013850900639809001315050113550501E7
:105088006FF01FEB130510006FF01FFF930790FFE1
:1050980093090000E3D4F5F6930644006FF0DFF1BE
:1050A80083574500130101FF232291002326110095
:1050B800232481002320210193040500639C070C0D
:1050C80003576500130400009317070193D707419E
:1050D80063C4070A9306A5011306000A63180702AA
:1050E800938764006F00800003D707009387270029
:1050F800239EE7FEE39AF6FE239C040013040401B2
:10510800630CC40603D76400E30C07FC937707F02D
:105118006390070413858401938524009307000096
:1051280013070500835607001307E7FF1396860049
:10513800B3E7C7002311F70093D78600E394E5FE91
:1051480003D7640013048400937707F0E38807FC0F
:105158001309000A6F00400113041400EFF01F94B4
:10516800634C890003D764001317070113570741DD
:1051780013850400E35207FE8320C10013050400D1
:105188000324810083244100032901001301010144
:105198006780000013F707F013040000631007048A
:1051A8001309F0F66F0040011304F4FFEFF09F8835
:1051B800E30424FD83D7440013850400E39607FE27
:1051C8008320C100130504000324810083244100C7
:1051D80003290100130101016780000093064500BF
:1051E8009305A501130700006F00800083D7060010
:1051F80013D687003367C700939787002390E6008C
:10520800139707019386260013570701E390B6FE0C
:1052180083D74400130480FF6FF09FF8130101FE49
:10522800232C8100232A91002328210123263101E0
:105238002324410123225101138906009384070086
:10524800232E11001304050093890500130A060094
:10525800930A0700EFF0DFE4930700093309A94038
:1052680063DCA716B78700009387E7FF63DA271F79
:1052780063840A1C03A5440083A70400630AF50697
:105288001387A4019387440313072700231F07FEEE
:10529800E31CF7FE93078003630CF53263D0A7166F
:1052A80093070004630CF52E930710076318F53471
:1052B800B78700409387F7FF1307A00023AAF400DD
:1052C800B787FFFF23A4E400239CF40023A6E4008F
:1052D8009307A000378700009387870093971700EC
:1052E800B387F4002395E70023A0A4006358201B8C
:1052F80083A5840083D744011308F008139615008A
:105308003306C40003570600B376F700634AA802C1
:105318001308B0006346B80293070600930584019A
:1053280003D727006304070093E6160023910700BC
:1053380093872700E396F5FE0357060083D74401B9
:1053480093C7F7FFB3F7E7002310F60083D764018C
:1053580033F7D700630007046384D71A138624033E
:10536800930684019384C401130700008357060041
:1053780083D506009386E6FF1306E6FFB387B700DA
:10538800B387E70013D707012391F60013771700B7
:10539800E31E96FC6358201983574400639E071246
:1053A800B7870000231C04009387E7FF63C8270919
:1053B800231124018320C101032481018324410195
:1053C800032901018329C100032A8100832A41009E
:1053D80013010102678000006354090E930700F768
:1053E800635CF908930724001304A401938727003A
:1053F800239F07FEE39C87FE6FF0DFFB9307800186
:105408006308F51693075003631AF51E3717000053
:10541800B7070004930660009387F77F1307078098
:1054280023AAF40023A4D400239CE40023A6D400D8
:10543800930760006FF05FEA231C0400B787FFFF43
:1054480093C7F7FF2311F400930744001304840162
:105458002390070093872700E31CF4FE6FF09FF565
:10546800930724001304A40193872700239F07FEB2
:10547800E39C87FE6FF01FF49305090013050400F1
:10548800EFF05FA06304050093091000638C0A0C19
:1054980003A5440083A70400E314F5DE930700097D
:1054A8006304F50A835784011305040093F7170072
:1054B800B3E9F900EFF00FD803A544006FF05FE3FC
:1054C800E3800AEE03A5440083A70400E31AF5DA93
:1054D800E34020E36FF09FFC13050400EFF08FD545
:1054E800B787000013091900231C04009387E7FFFE
:1054F800E3C627F5E35E09EA231104006FF09FEB8A
:105508006394090C83A7C40003D7840193971700F9
:10551800B307F40083D70700B3F7E700E39007E485
:10552800E34C20E7930700096306F5001305040020
:10553800EFF0CFD683574400E39007FA231C04000A
:10554800E34C09FA6FF0DFE603A6840083D7440131
:10555800131616003306C40003570600B3F6E70017
:105568006FF01FDE231C0400231104006FF09FE47A
:10557800B70780009387F70F1307400023AAF400AA
:105588009307001023A4E400239CF40023A6E4005E
:1055980093074000130700106FF01FD493077000A3
:1055A80023A4F400B70701809387F7FF23AAF40028
:1055B80093071000239CF4009307600023A6F400CF
:1055C800130710006FF05FD1E30A0AD86FF09FDC71
:1055D800B70780009387F70F1307600023AAF4002A
:1055E8009307001023A4E400239CF40023A6E400FE
:1055F80093076000130700106FF01FCE9307C000D9
:1056080023A4F400B70701809387F7FF23AAF400C7
:1056180093071000239CF4009307B00023A6F4001E
:10562800130710006FF05FCB130101FD23229102D5
:10563800232E310193840500835925002326110266
:105648002324810223202103232C4101130906006E
:10565800232A510123286101232671012324810172
:10566800232291012320A101130A0500EFF05FA373
:1056780003D424009307050013850400B389F94077
:10568800930A4903EFF0DFA13304A4401307E904A8
:1056980093870A0093872700239F07FEE39CE7FE72
:1056A800634A3409930B4A00138B44009389F9FF2A
:1056B800930CAA01138C240013070B0093870B008B
:1056C80003D6070083560700938727001307270090
:1056D800631AD60AE39697FF13068A011387840193
:1056E8009306000083570700835506001307E7FF5A
:1056F800B387D740B387B74093D607012311F70084
:1057080093F616001306E6FFE31EECFC130D1000DB
:1057180013850A00EFF08FB88357C9041304F4FF08
:1057280013850400336DFD002316A905EFF00FB7AC
:10573800E31434F993060400032481028320C10290
:105748008329C101032A8101832A4101032B010115
:10575800832BC100032C8100832C4100032D010001
:1057680093070900138504000329010283244102D9
:10577800130700001306000093050000130101033E
:105788006FF0DFA9130D0000E3E4C6F86FF0DFF453
:105798000357050083572500630607003787000075
:1057A800B3E7E7002399F50003572500B787000002
:1057B8009387F7FF6304F702930765009385050154
:1057C8001305850103D70700938727009385E5FF15
:1057D8002391E500E398A7FE678000009307650022
:1057E8001305A50103D7070093872700631A07024B
:1057F800E39AA7FE1387250193870500938727005F
:10580800239F07FEE31CF7FE83D725013787000097
:105818001307F7FFB3E7E7002399F5006780000057
:10582800138705019387050093872700239F07FEA9
:10583800E31CF7FEB7C7FF7F23A8F50067800000C9
:10584800130101F723286107035B2501B7870000CF
:105858009387F7FF232C410733FA6701131A0A01CC
:10586800232481082322910823202109232E31078C
:1058780023261108232A5107232671072324810789
:1058880023229107135A0A0193040500138905007E
:1058980013040600938906006312FA10EFF08FB024
:1058A800631A0528835A2901B3775A016382472B63
:1058B80013850400EFF04FDB630E052EB75501800A
:1058C800938585CD13050900EFF04FC863060536AB
:1058D800835A2901B78700009387F7FFB3FA570166
:1058E800939A0A0193DA0A016394FA2C13050900C2
:1058F800EFF08FD76310053283D72401B3F7FA008E
:105908006398570B13850400EFF00FD66318050052
:1059180013050900EFF04FD5630C05081385040043
:10592800EFF04FAF9304050013050900EFF08FAEB9
:10593800B384A440B33490009394F40023199400E2
:10594800130724019307040093872700239F07FE6A
:10595800E31CF7FE83572401378700001307F7FF7E
:10596800B3E7E7002319F4008320C1080324810862
:1059780083244108032901088329C107032A8107D1
:10598800832A4107032B0107832BC106032C8106B9
:10599800832C4106130101096780000083DA250181
:1059A80033F757011317070113570701630AF70461
:1059B800138504009305C100EFF0CFA91305090072
:1059C80093058102EFF00FA98354E1000359A10266
:1059D800639C040493070101930641026388D7205E
:1059E80003D7070093872700E30A07FE1305C100C2
:1059F800EFF00FEB0357A102B304A0406F000003C0
:105A080013850500EFF00F9AE30605EC130749012B
:105A1800835709001309290013042400231FF4FEE7
:105A2800E318E9FE6FF05FF413070900930A090011
:105A38009307C10293060104631207026382F61CEE
:105A480003D7070093872700E30A07FE130581029F
:105A5800EFF00FE50357A102B30AA940835781026B
:105A6800138C8903239BE902239AF9021387E9041B
:105A780093070C002390070093872700E31CF7FE89
:105A8800138AC904930B000013094102930C010106
:105A9800130B6104035509001309E9FF6318050C8A
:105AA80003D7C90493070A00B3EBEB0003D7E7FF5A
:105AB8009387E7FF2391E700E39A87FF239C090276
:105AC800E31A99FD1387490393078102930521047B
:105AD800035607009387270013072700239FC7FE55
:105AE800E398F5FEB7C6FFFFB384540193862600FA
:105AF80093850B001305810293870900130700049F
:105B0800B386D40013060000EFF04FF1035781026B
:105B18008357C1009305040013058102B387E7404A
:105B2800B337F000B307F0402314F102EFF05FC67B
:105B38006FF09FE31387440183D704009384240004
:105B480013042400231FF4FEE398E4FE6FF0DFE162
:105B580013050900EFF00F85E31A05EA1385040021
:105B6800EFF08FB0E30805D66FF05FD51306410458
:105B780093058102EFE09FF993050A0013060000E0
:105B88001307C10503D80500835707009385E5FF70
:105B98001307E7FFB3870701B387C70013D60701C9
:105BA8002391F50013761600E31E67FD6FF05FEF93
:105BB80003DB2401B78700009387F7FF33FB6701F6
:105BC800131B0B01135B0B01E314FBDE13850400AD
:105BD800EFF08FA9E31405D48357290193C7F7FF82
:105BE80013971701E31607DC6FF09FD29307440160
:105BF80013042400231F04FEE39C87FE6FF0DFD606
:105C08009307440113042400231F04FEE31CF4FE3D
:105C18006FF09FD5B7550180938585CD1385040016
:105C2800EFF0CF92630A050083D72401B3F7FA0097
:105C3800E38E57F96FF05FFA130704019307040026
:105C480093872700239F07FEE39CE7FEB7C7FF7FE4
:105C58002328F4006FF05FD183572501130101F564
:105C68002324810A93C7F7FF2322910A2320210BBB
:105C7800232E31092326110A232C4109232A5109ED
:105C880023286109232671092324810923229109E4
:105C98002320A109232EB107139717011309050023
:105CA8009389050013040600938406006316070011
:105CB800EFE05FEF6318053883D7290193C7F7FF33
:105CC80013971701630E0708375A018093058ACD89
:105CD80013050900EFF08F8763040510035A2901A3
:105CE80003D72901B78700009387F7FF33FA4701E5
:105CF800B3FAE700631AFA0813050900EFF0CF9624
:105D08006308051063984A0113850900EFF0CF95E1
:105D18006310050E9307440113042400231F04FE97
:105D2800E31CF4FE8320C10A0324810A8324410A68
:105D38000329010A8329C109032A8109832A410900
:105D4800032B0109832BC108032C8108832C4108EC
:105D5800032D0108832DC1071301010B6780000083
:105D680013850900EFE01FE4E30005F613874901F6
:105D780083D709009389290013042400231FF4FE04
:105D8800E398E9FE6FF01FFA6386FA081305090025
:105D98009305C101EFE01FEC93058103138509000A
:105DA800EFE05FEB835BA1030359E10163920B0C06
:105DB8009307C103930D0105638EFD3403D70700D4
:105DC80093872700E30A07FE13058103EFF04FAD21
:105DD800B307A0400356E1012326F1006F00C00974
:105DE80093058ACD13850900EFE05FF6E31805EE09
:105DF800130704019307040093872700239F07FED6
:105E0800E39CE7FEB7C7FF7F2328F4006FF09FF1FC
:105E1800E39E4AF713850900EFF00F85E30805F6BE
:105E280013050900EFE01FDF93040500138509003F
:105E3800EFE05FDEB387A440B337F0009397F70035
:105E48002319F400130724019307040093872700FC
:105E5800239F07FEE39CE7FE835724013787000052
:105E68001307F7FFB3E7E7002319F4006FF09FEB80
:105E78002326710113060900232421019307010237
:105E880093064103631206026380F62A03D70700CC
:105E980093872700E30A07FE1305C101EFF04FA01F
:105EA800B307A9402324F10003278103138D84033A
:105EB80093070D0023AAE4021389E40493872700BB
:105EC800239F07FEE31CF9FE13058103EFE09FB64D
:105ED800035C2102370A0100930D0105931A0C0196
:105EE800B38A8A41130BA103130AFAFF930CE10644
:105EF800930961058357C1030357E103930B0A0014
:105F080093970701B387E70063E8FA00B3D78703DD
:105F1800939B070193DB0B01130641059305C10110
:105F280013850B00EFE09FBE1307C103930781059C
:105F380083D5070003560700938727001307270018
:105F48006390C512E39697FF930700009305C10677
:105F580013860D000357060003D805001306E6FF55
:105F68003307F74033070741935707012311E6002A
:105F780093F717009385E5FFE31E66FD23107D0167
:105F88009307C10303D7270093872700239FE7FEC2
:105F9800E39AB7FF23180104130D2D00E31CA9F59C
:105FA800930500009307C1039306210503D7070053
:105FB80093872700B3E5E500E39AD7FE9397050199
:105FC80093D7074163840700930510009395050153
:105FD80093D50501138744039307810303560700EC
:105FE8009387270013072700239FC7FEE398F6FE31
:105FF8008327C10003278100B74600009386F6FF78
:10600800B38BE7401305810393870400130700044B
:10601800B386DB0013060000EFF04FA0035781039F
:106028008357C1019305040013058103B387E74033
:10603800B337F000B307F040231CF102EFF04FF53F
:106048006FF05FCE13074901835709001309290030
:1060580013042400231FF4FEE318E9FE6FF09FCC1D
:10606800E374B6EE9387FBFF9398070193D8080172
:1060780093070000930541031306C1060357060062
:1060880003D805001306E6FF3307F7403307074137
:10609800935707012311E60093F717009385E5FF4F
:1060A800E31E36FD1307C1039307810583D5070057
:1060B8000356070093872700130727006398C50036
:1060C800E39697FF938B08006FF01FE8E37CB6FE1A
:1060D8009387EBFF939B070193DB0B0113060000EB
:1060E800930541031307C1068357070003D805002A
:1060F8001307E7FFB387C740B387074113D60701E4
:106108002311F700137616009385E5FFE31E37FD8C
:106118006FF09FE39307440113042400231F04FE38
:10612800E39C87FE6FF01FC00357C10183578103AB
:106138006304F700378600002319C40013072401FD
:106148009307040093872700239F07FEE31CF7FEAD
:1061580083572401378700001307F7FFB3E7E700E9
:106168002319F4006FF01FBC130101FD23248102E1
:106178002326110213840500930741001307E10148
:1061880093872700239F07FEE39CE7FE0356E5005D
:106198009317060193D7074163CA0706B78700001C
:1061A8009387F7FF231201003376F600630CF60697
:1061B8009307E5002313C1001307A10083D6E7FF67
:1061C8009387E7FF13072700231FD7FEE318F5FE81
:1061D800631206022314010093050400130541000D
:1061E800EFF00FDB8320C1020324810213010103B6
:1061F80067800000930710009305F0FF1305410026
:106208002314F100EFE01FC86FF01FFD9307F0FFA4
:106218002312F100B78700009387F7FF3376F60063
:10622800E318F6F8930705009306E50003D707007F
:1062380093872700631C0704E39AD7FE13074401DA
:106248009307040093872700239F07FEE31CF7FEAC
:10625800130724019307040093872700239F07FE51
:10626800E31CF7FE83572401378700001307F7FF65
:10627800B3E7E7002319F4008317E500E3D407F632
:1062880013050400EFE05F946FF0DFF513070401D6
:106298009307040093872700239F07FEE31CF7FE5C
:1062A800B7C7FF7F2328F4006FF0DFF383A8C5008A
:1062B800130101E183AE050003AE450003A3850089
:1062C800232E1103832505049308F0FF23201117BB
:1062D800930800092324811E232C411D2326111E07
:1062E8002322911E2320211F232E311D232A511DD5
:1062F8002328611D2326711D2324811D2322911D1E
:106308002320A11D232EB11B2328D103232AC10337
:10631800232C6102232211172320C1002324D1003A
:106328002326E100232C0101130A0500138407002A
:10633800638005020327450493071000B397E7001D
:1063480023A2E50023A4F500EF10505823200A04E7
:10635800930901069385090013050103EFF0DFE0B7
:1063680013850900EFE01F8B032701003335A000D8
:106378002320A40093073000E302F7149307400199
:106388002322F100E318075E8357210703274116EC
:1063980093C7F7FF232AE100139717016318070033
:1063A80013850900EFE01F80E314054093070009F7
:1063B8002322F1161307C107938709001306410723
:1063C80083D607009387270013072700231FD7FECC
:1063D800E398C7FE0356E108232801009317060136
:1063E80093D7074163DE070013161601B7070100AC
:1063F800135616019387F7FF2317C1082328F100C6
:10640800375B0180930D8BCD138C4D0193060000F3
:106418009307810913070C00130DC10A6F00800050
:106428008356070093872700239FD7FE130727006B
:10643800E398A7FF63080614B78700009387F7FF60
:10644800E306F6568317C108E3D8075A9305C10730
:1064580013050C00EFE09F8F63020514E34C050C55
:106468008357E108E39C07628317C108930400007F
:106478001309011663C4070213848D111306C1079B
:10648800930609009305060013050400EFF04FBBBF
:106498008317C1089384F4FFE3D207FE1304010DA8
:1064A800930B810E130704009307C1071306010914
:1064B80083D607009387270013072700231FD7FEDB
:1064C800E398C7FE930600009307810913070C00A1
:1064D8006F0080008356070093872700239FD7FE0D
:1064E80013072700E398A7FF938C8D02138DCD1215
:1064F800B7FAFFFF938D8D116F00C000130D4D018A
:10650800938C4C019305040013050C00EFE01F84E5
:10651800930705009305040013050D006356F00466
:10652800EFE0DF82930705009306090013060400D5
:106538009305040013850C0063C00702EFF04FB009
:1065480013068109930609009305060013850C00BC
:10655800EFF00FAFB384540193D7FA01B387570113
:1065680093DA1740E39CBCF91306810993060900E6
:1065780093050C0013050600EFF00FEE930A411285
:106588006F0000039307C1079306E10803D70700CC
:1065980093872700E31C07EAE39AD7FE93040000D9
:1065A800930A4112130901161304010D930B810E6E
:1065B8009305040013058109EFE0CFE9130781096A
:1065C8009307040083D60700938727001307270043
:1065D800231FD7FEE39877FF930504001305C1072F
:1065E8002318010AEFE00FE79307C10703570400D8
:1065F8001304240093872700239FE7FEE31874FF02
:1066080013058109130609009305C107231A010818
:10661800EFF08F810355C11A6314051C930C4109CF
:106628001304E107130C610B93058BCD1305C10708
:10663800EFE0CFF16306051A1307000093860C00FC
:106648006F00C001131717002390F60013170701F6
:106658009386E6FF135707016384860483D70600F1
:1066680013960701135606419397170063540600C3
:10667800136717009397070193D70701137627002D
:1066880093E51700E30006FC131717002390B600E4
:10669800131707019386E6FF13570701E39086FC5B
:1066A8001307410B9307C10783D607009387270079
:1066B80013072700231FD7FEE39897FF2316010C23
:1066C800130700009306C10C6F00C00113171700D1
:1066D8002390F600131707019386E6FF1357070167
:1066E8006384860583D7060013960701135606416F
:1066F80093971700635406001367170093970701D1
:1067080093D707011376270093E51700E30006FCEB
:10671800131717002390B600131707019386E6FF97
:1067280013570701E39086FD130700009306C10C79
:106738006F00C001131717002390F6001317070105
:106748009386E6FF135707016384860583D70600FF
:1067580013960701135606419397170063540600D2
:10676800136717009397070193D70701137627003C
:1067780093E51700E30006FC131717002390B600F3
:10678800131707019386E6FF13570701E39086FD69
:106798001306000093860C001307C10C83D506006E
:1067A800835707009386E6FF1307E7FFB387B70011
:1067B800B387C70013D607012391F6001376160096
:1067C800E31E87FD13058109130609009305C10718
:1067D800EFE09FE50355C11A9384F4FFE30605E44F
:1067E800832701018326010013073000B337F00027
:1067F800B307F04093F7D700938707022302F112FB
:10680800832741006394E600B38797001307A0022B
:10681800138407006354F7001304A0021307A000B1
:106828006302E54E130505031307E002A302A11254
:106838002303E112E3C2071E930771122328F10014
:10684800130C0000232E910093040C00130C090074
:1068580003290101930C410B930D4109930BE107A7
:10686800130D610B1307000013860D006F00C001A4
:10687800131717002310F600131707011306E6FF76
:10688800135707016304760583570600939507019C
:1068980093D505419397170063D405001367170034
:1068A8009397070193D707019375270013E51700FE
:1068B800E38005FC131717002310A6001317070120
:1068C8001306E6FF13570701E31076FD13870C0044
:1068D8009307C10703D607009387270013072700EC
:1068E800231FC7FEE398B7FF2316010C1307000008
:1068F8001306C10C6F00C001131717002310F60010
:10690800131707011306E6FF135707016304A605CB
:10691800835706009395070193D505419397170070
:1069280063D40500136717009397070193D70701EE
:106938009375270013E51700E38005FC131717006C
:106948002310A600131707011306E6FF13570701C4
:10695800E310A6FD130700001306C10C6F00C00169
:10696800131717002310F600131707011306E6FF85
:10697800135707016304A60583570600939507017B
:1069880093D505419397170063D405001367170043
:106998009397070193D707019375270013E517000D
:1069A800E38005FC131717002310A600131707012F
:1069B8001306E6FF13570701E310A6FD9305000031
:1069C80013860D001307C10C0355060083570700F3
:1069D8001306E6FF1307E7FFB387A700B387B700DF
:1069E80093D507012311F60093F51500E31EA7FDC3
:1069F80013060C009305C10713058109EFE0DFC2F8
:106A08008357C11A33079900938414001386070328
:106A18002300C700E35894E41345F4FF032701015A
:106A28001355F5413375A4008324C10113091500DA
:106A380033092701330CA70013074000635EF704EE
:106A480013075000E380E7008347E9FF1307E9FFD6
:106A580093F7F707634404789306E002130680036C
:106A680093050003638ED7006352F6788347F7FFD8
:106A78002300B7001307F7FF93F7F7076FF09FFEA0
:106A88008347F7FF93068003E3F4F60093071003A8
:106A980093841400A30FF7FEB755018013860400F2
:106AA800938545CD13050C00EF20900383572107EC
:106AB800032741012328911693C7F7FF2322E116E4
:106AC80013971701631E070013850900EFE0CFB97C
:106AD8006310052213850900EFE0CF8C631A0520A7
:106AE8008326C100034741129387140023A0F600B0
:106AF80093870A00630A07029306E002630CD71C17
:106B080003C7170093871700E31A07FE930650047C
:106B180063E6FA006F0040016388570103C7F7FF77
:106B28009387F7FFE31AD7FE2380070093870A00AD
:106B3800930600021306D00203C707006304D700B8
:106B48006316C700938717006FF01FFF13840A00AE
:106B58006F00C00003C70700138406002300E40089
:106B68009306140093871700E31607FE8326010097
:106B7800930720000347F4FF6386F612832741003A
:106B88009386070063D49700938604009307000355
:106B98006316F702B307544163D2F60213060003E3
:106BA8006F00800063DCE6008347E4FFA30F04FE68
:106BB8001304F4FF33075441E386C7FE032701009B
:106BC800930730006302F70A8327810023220A040F
:106BD800938697009307700163F2D70C1307100090
:106BE8009307400093971700138647019305070002
:106BF80013071700E3F8C6FE2322BA0413050A0098
:106C0800EF1040422320AA0493850A00930405004C
:106C1800EF20500A83278101638807003304544119
:106C28003384840023A087008320C11E0324811E8F
:106C38000329011E8329C11D032A811D832A411DA1
:106C4800032B011D832BC11C032C811C832C411C8D
:106C5800032D011C832DC11B138504008324411EB1
:106C68001301011F6780000083274100B384970048
:106C780063C804508327C1000327810083A7070046
:106C8800B307F7002324F1008327810023220A0495
:106C98009386370093077001E3E2D7F49305000069
:106CA8006FF0DFF593070003E310F7F2B3075441E1
:106CB80093061000E3C4F6EE6FF01FF18324810001
:106CC800232291009307A00263D097EC2322F100BE
:106CD8006FF08FEB03C70700E30A07E203C717004B
:106CE80093871700A38FE7FEE31A07FE6FF01FE2F2
:106CF8000327C100B72700009387F7702320F70008
:106D08006FF0DFE213071003A302E1121307E0029A
:106D18002303E11293841400635CF02A93070003B1
:106D2800A303F112930781121304F4FF2328F1003F
:106D38006FF01FB1930C410B13870C009307C10729
:106D48001306010983D60700938727001307270036
:106D5800231FD7FEE398C7FEB74700009387E708CD
:106D68002313F10CB78700009387F7FF232EF10058
:106D7800B7C7FFFF930A41121304010D130E000158
:106D880013838D0C93872700232441032322510367
:106D980093040000938A0C0013090116930C040055
:106DA800930BA10A2320F102130A0E001304030017
:106DB800930609001306810993850A001305040048
:106DC800EFE09FE91307C1049307810983D6070001
:106DD8009387270013072700231FD7FEE398A7FFF1
:106DE8008327C1018355E10533F6F50083270102A6
:106DF8003305F6006350A03A130600093306A6408F
:106E080013870C009307C10483D6070093872700D4
:106E180013072700231FD7FEE39837FF6354C006E4
:106E28009307F00013870C0063DCC702130606FF04
:106E38009356460013871600131717003387EC0084
:106E480093870C0093872700239F07FEE39CE7FEA8
:106E5800130600083306A640939646003306D6402C
:106E6800131616003386CD00835707008356062372
:106E7800B3F7D7002310F7009395050193D5054183
:106E880063C005169307810913870C0003D6070012
:106E98008356070093872700130727006314D60239
:106EA800E396FBFE13870A009307810983D6070040
:106EB8009387270013072700231FD7FEE398A7FF10
:106EC800B3844401130444019387CD12135A1A0062
:106ED800E310F4EE8357610C0357E10813840C00A8
:106EE800032A8102B387E70037C7FFFF938C0A00A4
:106EF800130727F7832A4102B387E7002313F10C0E
:106F08001307C10793870C001306810C83D607006B
:106F18009387270013072700231FD7FEE398C7FE90
:106F280013070000930781096F00800003570C00C6
:106F380093872700239FE7FE130C2C00E398A7FFF5
:106F4800138D8D02371C0000938D8D116F00000189
:106F5800135C1C006300BD29130D4D0193850C00C3
:106F680013850D00EFD09FDE9307050093850C0075
:106F780013050D006340F026EFD05FDDE34AA0FC67
:106F88009306090013860C0093850C0013050D0069
:106F9800EFE09FCC130681099306090093050600CC
:106FA80013050D00EFE0DF89B38484016FF05FFA09
:106FB800930A4112B7550180938505CB13850A00C2
:106FC800B7240000EF20C0319384F4706FF01FAE37
:106FD800130C7112E39207AC232881016FF05F86CE
:106FE8009307C10413870C006F00C0009306E105E6
:106FF800E38AF6E803D6070083560700938727003D
:1070080013072700E304D6FE8357210E0327C10187
:10701800B377F700639EE70013850C00EFD09FB8A5
:10702800E31205E613850C00EFD01FE4E31C05E42A
:107038009305C10E13050C00EFD0DFC19305811035
:1070480013850C00EFD01FC10356C10E0355A110C4
:107058008358E10E1346F6FF131606011356060170
:107068002316C10EB385A84093060500635EB006DB
:1070780083264102130781109307011283550700E5
:107088001307270093862600239FB6FEE318F7FE12
:10709800231E0112130781109306C10E6F00800092
:1070A80003D6060013072700231FC7FE9386260072
:1070B800E318F7FE83274102231001121307C10EBC
:1070C8001306C11383D607009387270013072700E9
:1070D800231FD7FEE398C7FE8356A110B3051541B9
:1070E80023120110138506006386052C2326D1027E
:1070F8009307F0F663C8F5061305C10EEFD09FD8C5
:107108008326C10293050500930701121305411058
:107118000356C10E03578110630AE62E13070000B9
:107128001306070003D70700035805009387E7FFF6
:107138003307C74033070741135607012391E70078
:107148001307A110137616001305E5FFE39CE7FC6F
:107158001306100093070900130700041305811094
:10716800EFE0CF8B93850C0013058110EFE04FE221
:107178006FF05FD1832781009384F7FF6FF05FB4CE
:107188008327C1002302011213840A0023A00700E9
:107198006FF09FAF93870C001307410E938727006A
:1071A800239F07FEE39CE7FE6FF01FCD83270101B5
:1071B800930A4112638A0706B7550180938585CBE8
:1071C80013850A00B7240000EF2080119384F4701F
:1071D8006FF0DF8D930B810E6FF08FBD9307100357
:1071E800230FF9FE938414006FF01F8B9387170009
:1071F8002300F7006FF05F8A930A4112B7550180A8
:10720800938505CD13850A00B7240000EF20400DB3
:107218009384F4706FF09F898357C11A130C61121D
:10722800130971126FF05F81B7550180938545CCC2
:1072380013850A00B7240000EF20800A9384F470B5
:107248006FF0DF86930581091305C107EFE04FD47E
:1072580093058BCD13058109EFD05FAF631605FE4B
:10726800E34C04828347E9FF138727FD1337170090
:107278001347F7FF3307EC0003470700137717009E
:10728800E30C07801307E9FF93F7F7076FF0CFFCCC
:1072980093871700A30FF7FE6FF01F801304010DEB
:1072A800930504001305C107B74C0000EFD09F9A5F
:1072B80093040000930B810E1309C10C930A210D4E
:1072C800938CECFF8357810E93F77700639A070C32
:1072D8001307410B9307040083D607009387270001
:1072E80013072700231FD7FEE39877FF1305410BE9
:1072F8002316010CEFD00FF41305410BEFD08FF3D9
:10730800130600009306090013870B0083D50600B7
:10731800835707009386E6FF1307E7FFB387B70095
:10732800B387C70013D607012391F600137616001A
:10733800E31E57FD8357610B0357810B9387370073
:10734800231BF10A630007021305410BEFD08FEEF0
:107358008357610B0357810B93871700231BF10A8F
:10736800E31407FE8357C10C639C07028357610B24
:1073780063E8FC02130704009307410B83D6070058
:107388009387270013072700231FD7FEE39827FFBB
:107398002314010E9384F4FF930750FDE394F4F251
:1073A8009305C10713050400EFE08FBE130901160A
:1073B8006FF04F8F1307C1109307010F83D8070091
:1073C8000356070093872700130727006398C8020E
:1073D80013066110E394C7FE0357C10E835781104B
:1073E8006302F70693870C001307410E9387270063
:1073F800239F07FEE39CE7FE6FF0DFA86366160D88
:1074080093070112130541106FF09FD01307000076
:107418001303E10E03D80700035605009387E7FF1F
:107428001305E5FF330606013307E6001356070187
:107438002391E70013771600E31E65FC130600008E
:107448006FF05FD113870600639206068317E11079
:1074580063CE0704930601126F0000022390F60022
:1074680013171700131707019386E6FF9307A11058
:1074780013570701E388F6CE83D706001396070152
:1074880013560641939717006354060013671700B5
:107498009397070193D707011376270093E5170001
:1074A800E30E06FA2390B6006FF09FFB1306C11097
:1074B80093070112631207086382C708035706007F
:1074C800130626006FF01FFF0326410213078110E1
:1074D8009307011203550700130727001306260018
:1074E800231FA6FEE318F7FE231E011213068110C0
:1074F8001307C10E1305411003580700130727008F
:1075080013062600231F06FFE318A7FE03274102E0
:10751800231001129308C10E1306C1130358070064
:107528001307270093882800239F08FFE318C7FE46
:10753800231201106FF0DFBD138516002315A1106B
:107548006FF05FC2032785008327C5000326050067
:1075580083264500130101FC130501009305410131
:107568002324E1002326F100232E11022320C10049
:107578002322D100EFE05FBF8357610213050000AB
:1075880093C7F7FF13971701631A07001305410103
:10759800EFD04FE113351500130515008320C10303
:1075A80013010104678000001305050F67800000C0
:1075B8001385811B678000001385811B678000008D
:1075C800130101F923248106138405008395E5003E
:1075D800232291062320210723261106930406005F
:1075E8001389060063CA050413068100EF6040434F
:1075F800634405040327C100B7F700008320C106D0
:10760800B3F7E70037E7FFFFB387E70003248106F6
:1076180093B717002320F9009307004023A0F40034
:107628003715000083244106032901061305058048
:1076380013010107678000008357C4002320090055
:1076480093F70708638407028320C1060324810691
:107658009307000423A0F4000329010683244106AC
:107668001305000013010107678000008320C1068D
:10767800032481069307004023A0F4000329010690
:1076880083244106130500001301010767800000E9
:1076980083D7C500130101FE232C8100232E11007E
:1076A800232A91002328210193F72700138405003A
:1076B800638807029387350423A0F50023A8F50003
:1076C8009307100023AAF5008320C1010324810138
:1076D800832441010329010113010102678000008D
:1076E8009306C1001306810093040500EFF05FEDD7
:1076F800832581001309050013850400EF00400B62
:107708008317C4006308050437470080130707166A
:1077180023AEE402032781008326C10093E707080C
:107728002316F4002320A4002328A400232AE4001D
:1077380063980604B3E727018320C1012316F400E8
:10774800032481018324410103290101130101025A
:107758006780000013F70720E31807F693F7C7FFC1
:1077680093E72700130734042316F4009307100047
:107778002320E4002328E400232AF4006FF0DFF438
:107788008315E40013850400EF60407A6316050052
:107798008317C4006FF01FFA0357C4001377C7FF9D
:1077A800136717009317070193D707416FF09FF8E6
:1077B800130101FD232E3101232611022324810206
:1077C8002322910223202103232C4101232A510142
:1077D8002328610123267101232481012322910199
:1077E8009387B50013076001930905006364F706E2
:1077F8009307000163E2B71EEF00500293040001F3
:107808001306200093078001138901CCB307F90000
:1078180003A44700138787FF6308E42083274400F5
:107828008326C4000326840093F7C7FFB307F40038
:1078380003A747002326D60023A4C6001367170012
:107848001385090023A2E700EF00807D130584005B
:107858006F00401993F487FF63C0071863EEB416EE
:10786800EF00C07B9307701F63FA974493D7940087
:107878006384071A130740006360F73C93D76400DA
:10788800138697031385870393163600138901CC53
:10789800B306D90003A44600938686FF6386860252
:1078A8009305F0006F000001635207320324C400FF
:1078B800638C86008327440093F7C7FF338797407C
:1078C800E3D4E5FE130605000324090193088900A3
:1078D80063081417032544009306F0001375C5FFC9
:1078E800B307954063C2F640232A190123281901DA
:1078F80063DC073C9307F01F63E0A72E937785FFAF
:107908009387870083254900B307F90083A60700FA
:1079180013555500130710003317A7003367B70036
:10792800938587FF2326B4002324D4002322E9006B
:1079380023A0870023A686009357264093051000AE
:10794800B395F5006368B710B3F7E50063940702D1
:10795800939515001376C6FFB3F7E50013064600A6
:10796800639A070093951500B3F7E50013064600E0
:10797800E38A07FE1308F000131336003303690087
:10798800130503008327C500130E06006308F52CB2
:1079980003A747001384070083A7C7001377C7FF0F
:1079A800B30697406348D82CE3C206FE3307E400C9
:1079B80083264700032684001385090093E61600F2
:1079C8002322D7002326F60023A4C700EF00406532
:1079D800130584006F0000019307C00023A0F9007D
:1079E800130500008320C10203248102832441027D
:1079F800032901028329C101032A8101832A410144
:107A0800032B0101832BC100032C8100832C41002F
:107A18001301010367800000930600201306000489
:107A28001305F0036FF09FE603A4C70013062600B2
:107A3800E39687DE0324090193088900E31C14E90F
:107A4800032749009357264093051000B395F50086
:107A5800E37CB7EE03248900832A440013FBCAFFA2
:107A680063689B00B3079B401307F000634CF71251
:107A780083AA012903A701269307F0FF330A6401AB
:107A8800B38A54016304F734B71700009387F700EB
:107A9800B38AFA00B7F7FFFFB3FAFA0093850A0032
:107AA80013850900EF1040779307F0FF930B05004B
:107AB8006306F52863624529138C412F83250C0042
:107AC800B385BA002320BC0093870500630EAA384B
:107AD80083A601261307F0FF6386E63A338A4B41F3
:107AE800B307FA002320FC0093FC7B0063820C3070
:107AF800B7170000B38B9B4193858700938B8B004E
:107B0800B3859541B38A5B019387F7FFB3855541E8
:107B180033FAF50093050A0013850900EF10C06FCA
:107B28009307F0FF630AF53A33057541B30A450137
:107B380083250C002324790193EA1A00B305BA00BF
:107B48002320BC0023A25B01630224359306F000C6
:107B580063F266350327440093074BFF93F787FFCB
:107B6800137717003367F7002322E4001306500049
:107B78003307F4002322C7002324C70063E8F6363E
:107B880083AA4B0013840B0003A7C1286374B700B2
:107B980023A6B12803A781286376B71A23A4B1289E
:107BA8006F00401A13E714002322E400B304940082
:107BB8002324990093E717001385090023A2F400F2
:107BC800EF000046130584006FF0DFE18326C40050
:107BD800032684006FF09FC5935795001307400054
:107BE8006372F71413074001636AF7229386C70587
:107BF8009385B70593963600B306D90083A7060088
:107C0800938686FF6388F61C03A747001377C7FF90
:107C18006376E50083A78700E398F6FE83A6C7008E
:107C2800032749002326D4002324F40023A4860034
:107C380023A687006FF05FD0130740016376F71221
:107C480013074005636AF71E93D7C4001386F70627
:107C58001385E706931636006FF05FC3130E1E00F8
:107C680093773E0013058500638E07108327C500B0
:107C78006FF0DFD10326840093E514002322B400BB
:107C88002326F60023A4C700B3049400232A9900EE
:107C98002328990093E7160023A6140123A41401AE
:107CA80023A2F4003307E400138509002320D7003A
:107CB800EF000037130584006FF0DFD213D63400CD
:107CC800938784006FF05FB43307A40083274700CD
:107CD8001385090093E717002322F700EF004034CB
:107CE800130584006FF01FD013E714002322E4006B
:107CF800B3049400232A99002328990013E7170056
:107D080023A6140123A4140123A2E4003305A4002C
:107D18002320F50013850900EF0080301305840047
:107D28006FF05FCC9357650093869703938587031D
:107D3800939636006FF05FEC630E241103248900DC
:107D4800832A440093FACAFFB3879A4063E69A00ED
:107D58001307F000E348F7E413850900EF00402C0F
:107D6800130500006FF01FC81386C7051385B705F4
:107D7800931636006FF09FB1832783001306F6FF32
:107D88006390671C93773600130383FFE39607FE1F
:107D98000327490093C7F5FFB3F7E7002322F9004B
:107DA80093951500E3E8B7CAE38605CA33F7F500EB
:107DB800631A07009395150033F7F500130E4E006C
:107DC800E30A07FE13060E006FF01FBB938A0A0131
:107DD8006FF0DFCC0325490093D525401307100029
:107DE8003317B7003367A7002322E9006FF09FE33A
:107DF800B3855B01B305B0409395450113DA45019E
:107E080093050A0013850900EF1000419307F0FF5E
:107E1800E31CF5D0130A00006FF09FD1130740054B
:107E28006360F7089357C5009386F7069385E706BE
:107E3800939636006FF05FDC130740156360F70810
:107E480093D7F400138687071385770793163600B0
:107E58006FF0DFA3138C412F83270C00B387FA0040
:107E68002320FC006FF0DFC613174A01E31207C690
:107E780003248900B30A5B0193EA1A002322540100
:107E88006FF09FD023A071276FF01FC613840B00DB
:107E98006FF09FCF9307100023A2FB006FF0DFEB7A
:107EA800130740156362F7069357F5009386870713
:107EB80093857707939636006FF01FD413074055C4
:107EC8006362F70693D724011386D7071385C7077C
:107ED800931636006FF09F9B938C8CFFB38A9A01A0
:107EE800B38A7A41130A00006FF09FC49305840097
:107EF80013850900EFC08FEE0324890083250C0049
:107F0800832A44006FF05FC8130740556364F70283
:107F1800935725019386D7079385C707939636000D
:107F28006FF09FCD9306803F1306F0071305E00717
:107F38006FF0DF959306803F9305E0076FF0DFCB86
:107F4800832749006FF0DFE59377350093F6F50F47
:107F5800638A07029307F6FF630E06021306F0FF13
:107F68006F0080011305150013773500630E0700B5
:107F78009387F7FF6380C70203470500E314D7FE22
:107F88006780000093070600130730006366F70256
:107F9800639607001305000067800000B307F5002B
:107FA8006F00C00013051500E386A7FE0347050010
:107FB800E31AD7FE67800000370701009398850011
:107FC8001307F7FFB3F8E80093F5F50FB3E5B8002A
:107FD80093980501B3E8B8003708FFFEB78580809D
:107FE8001308F8EF938505081303300003270500ED
:107FF80033C7E800330607011347F7FF3377E60076
:108008003377B700E31C07F89387C7FF13054500CC
:10801800E36EF3FCE39407F86FF0DFF76780000086
:10802800678000008327C504130101FF2324810012
:108038002322910023261100232021011304050087
:1080480093840500638E070213952400B387A70065
:1080580003A50700630605040327050023A0E7001E
:1080680023280500232605008320C100032481005E
:1080780083244100032901001301010167800000E6
:108088001306100293054000EF5080512326A404E4
:1080980093070500E31A05FA130500006FF0DFFCEB
:1080A80013091000331999001306590013162600F6
:1080B8009305100013050400EF50804EE30E05FCF5
:1080C80023229500232425016FF09FF96380050280
:1080D80003A745008327C50413172700B387E700C4
:1080E80003A7070023A0E50023A0B70067800000CE
:1080F800130101FE232A910083A40501370301001F
:10810800232C81002328210123263101232E11004D
:1081180023244101138905009309050013840600EF
:1081280013884501930800001303F3FF8327080011
:108138001308480093881800B3F66700B386C60290
:1081480093D70701B387C702B386860013DE0601FB
:1081580033F76600B386C701939706013387E700B4
:10816800232EE8FE13D40601E3C298FC630204023E
:108178008327890063D0F4049387440093972700EA
:10818800B307F90023A287009384140023289900D9
:108198008320C10103248101832441018329C10073
:1081A800032A8100130509000329010113010102B3
:1081B8006780000083254900138509009385150011
:1081C800EFF05FE6130A0500630C050403260901B6
:1081D8009305C9001305C5001306260013162600CB
:1081E800EF5090710327490083A7C904131727008C
:1081F800B387E70003A707002320E90023A027018E
:108208009387440013090A0093972700B307F900DE
:1082180023A2870093841400232899006FF05FF746
:10822800B7560180375501809386C6F213060000C1
:108238009305500B130505F4EF500030130101FEB0
:10824800232C8100232A9100232821012326310190
:10825800232441011388860093079000232E1100E0
:10826800232251013348F8029389060013090500B7
:1082780013840500130A06009304070063D8D70C7B
:108288009307100093050000939717009385150036
:10829800E3CC07FF13050900EFF0DFD893050500CD
:1082A800630A050A930710002328F500232A95007E
:1082B8009307900063D64709930A940093840A00B1
:1082C8003304440183C604001306A0001305090003
:1082D800938606FDEFF0DFE1938414009305050013
:1082E800E39284FE13048AFF33848A0063563A03B8
:1082F800B3894941B3093401834604001306A00039
:1083080013050900938606FDEFF09FDE13041400A1
:1083180093050500E39289FE8320C10103248101AE
:1083280083244101032901018329C100032A810013
:10833800832A4100138505001301010267800000AC
:108348001304A400130A90006FF05FFA930500006D
:108358006FF05FF4B7560180375501809386C6F2F7
:10836800130600009305E00C130505F4EF50C01C3C
:108378003707FFFF3377E500930705001305000073
:10838800631607009397070113050001370700FFDD
:1083980033F7E700631607001305850093978700F6
:1083A800370700F033F7E7006316070013054500A9
:1083B80093974700370700C033F7E70063160700B5
:1083C800130525009397270063C807001397170024
:1083D80013051500635407006780000013050002A9
:1083E80067800000832705001307050093F67700D0
:1083F8006384060293F6170013050000639E0606C1
:1084080093F627006380060893D717002320F70008
:1084180013051000678000009396070193D60601A4
:10842800130500006396060093D7070113050001A2
:1084380093F6F70F639606001305850093D7870018
:1084480093F6F700639606001305450093D7470097
:1084580093F63700639606001305250093D7270087
:1084680093F61700639C060093D7170013051500B1
:108478006396070013050002678000002320F700B9
:108488006780000093D727002320F70013052000FA
:1084980067800000130101FF232481001384050075
:1084A8009305100023261100EFF0DFB763000502E3
:1084B8008320C100232A85000324810013071000AC
:1084C8002328E5001301010167800000B7560180E9
:1084D800375501809386C6F21306000093050014F1
:1084E800130505F4EF504005130101FE232821016F
:1084F8002326310103A9050183290601232A9100B6
:1085080023244101232E1100232C8100138A050006
:1085180093040600634C390113870900938405000E
:1085280093090900130A06001309070083A78400AA
:1085380083A5440033842901B3A78700B385F500D8
:10854800EFF05FAE630C051A13034501931824007E
:10855800B3081301930703006378130123A00700EE
:1085680093874700E3EC17FF13084A01131E2900FD
:10857800938E440193952900330EC801B385BE003C
:10858800637CC80B93875401130F400063FEF514F6
:10859800370601001306F6FF6F00000113084800B4
:1085A80013034300637AC809832F0800B3F4CF008C
:1085B8006394040C93DF0F01E3820FFE032703008B
:1085C8009302030093860E009304070093030000B0
:1085D80083A7060093D904013377C700B3F7C70010
:1085E800B387F70383A44200938242009386460030
:1085F80033F9C400B3873701B38777009393070132
:1086080033E7E30023AEE2FE03D7E6FF93D7070183
:108618003307F703330727013307F700935307019D
:10862800E3E8B6FAB307E30123A0E700130848001C
:1086380013034300E36AC8F7634880006F008001B2
:108648001304F4FF6308040083A7C8FF9388C8FFD6
:10865800E38807FE8320C1012328850003248101C4
:1086680083244101032901018329C100032A8100D0
:1086780013010102678000009303030093820E0038
:108688001309000003A7020083AF0300938343008C
:10869800B376C700B38696029357070133F7CF0026
:1086A80093DF0F0193824200B3879702B386E600F7
:1086B800B386260113D70601B3F6C600B387F701C0
:1086C800B387E70013970701B366D70023AED3FE3D
:1086D80013D90701E3E8B2FAB307E30123A027019E
:1086E800832F08006FF01FED338F9540130FBFFEE7
:1086F800137FCFFF130F4F006FF09FE9B75601802C
:10870800375501809386C6F2130600009305D015ED
:10871800130505F4EF405062130101FE232C81007C
:108728002326310123244101232E1100232A9100FD
:1087380023282101937736001304060093090500C6
:10874800138A05006394070C1354244013090A0084
:108758006308040683A48904638E040C93771400C9
:1087680013090A006390070213541440630A0404AF
:1087780003A5040063080506930405009377140015
:10878800E38407FE13860400930509001385090096
:10879800EFF09FD5630809060327490083A7C9049A
:1087A8001354144013172700B387E70003A70700E3
:1087B8002320E90023A0270113090500E31A04FA7E
:1087C8008320C10103248101832441018329C1003D
:1087D800032A81001305090003290101130101027D
:1087E8006780000013860400938504001385090040
:1087F800EFF09FCF23A0A4002320050093040500D9
:108808006FF0DFF7130905006FF01FF69387F7FF86
:1088180037570180130787F993972700B307F700A5
:1088280003A6070093060000EFF09F8C130A0500CB
:108838006FF09FF19305102713850900EFF09FC58E
:1088480023A4A90493040500232005006FF01FF159
:10885800130101FE2324410103AA050183A7850012
:108868002326310193595640338A4901232C81002C
:10887800232A91002328210123225101232E1100AC
:1088880013091A00938405001304060083A5450004
:10889800930A050063D8270193971700938515005D
:1088A800E3CC27FF13850A00EFF0CFF7630C051020
:1088B800130845016354300393895900939929009B
:1088C80033073501930708009387470023AE07FE57
:1088D800E39CE7FE9389C9FE3308380103A7040126
:1088E800938744011373F401131627003386C700D6
:1088F8006304030A93050002B385654093080800E2
:108908009306000003A70700938848009387470051
:10891800331767003367D70023AEE8FE03A7C7FF06
:10892800B356B700E3E0C7FE13875401930740002E
:10893800636AE600B30796409387B7FE93F7C7FFCD
:10894800938747003308F8002320D8006384060083
:10895800130A090003A7440083A7CA048320C1019E
:1089680013172700B387E70003A70700232845014B
:108978000324810123A0E40023A097000329010117
:10898800832441018329C100032A8100832A4100ED
:10899800130101026780000003A7070093874700BF
:1089A80013084800232EE8FEE3F6C7FA03A70700DA
:1089B8009387470013084800232EE8FEE3EEC7FC20
:1089C8006FF05FF9B7560180375501809386C6F27C
:1089D800130600009305901D130505F4EF40D035EC
:1089E8000327050183A70501130805003305F74090
:1089F8006314F704939727001308480193854501EA
:108A08003307F800B387F5006F0080006376E8024B
:108A18008326C7FF03A6C7FF1307C7FF9387C7FFB0
:108A2800E386C6FEB3B6C6003305D0401375E5FF2E
:108A380013051500678000006780000083A7050103
:108A480003270601130101FF23248100232291003B
:108A58002320210123261100938405001304060016
:108A68003389E7406394E71A9316270093854501F5
:108A780013074601B387D5003307D7006F0080007E
:108A880063FCF51803A6C7FF8326C7FF9387C7FFB4
:108A98001307C7FFE306D6FE6360D61683A5440016
:108AA800EFF04FD86302051A03AE040183220401D4
:108AB800938F4401931E2E001308440193922200C1
:108AC80093034501B708010023262501B38EDF0172
:108AD800B3025800138F030013830F00930700009D
:108AE8009388F8FF0327030083250800130F4F001E
:108AF800B3761701B386F600B3F71501B386F640CF
:108B080093D5050193570701B387B74013D706419B
:108B1800B387E70013970701B3F61601B366D700CA
:108B280013084800232EDFFE1303430093D70741A1
:108B3800E36A58FAB38582409385B5FE130454015D
:108B480093D525001307000063E4820013972500DE
:108B58003387E3001308400063E68200938515001D
:108B680013982500B38F0F01B383030163FEDF055C
:108B7800B70801001388030093850F009388F8FF56
:108B880003A70500130848009385450033761701AD
:108B98003306F6009356064193570701B387D7006B
:108BA8009396070133761601B3E6C600232ED8FE46
:108BB80093D70741E3E6D5FD1387FEFFB30FF741CF
:108BC80013F7CFFF3387E300639A06008327C7FFB5
:108BD800130EFEFF1307C7FFE38A07FE8320C100B9
:108BE800032481002328C5018324410003290100AF
:108BF8001301010167800000938704001309100026
:108C080093040400138407006FF05FE9E34609FE4C
:108C1800130900006FF09FE893050000EFF08FC084
:108C2800630205048320C100032481009307100018
:108C38002328F500232A0500832441000329010085
:108C48001301010167800000B75601803755018084
:108C58009386C6F21306000093050024130505F455
:108C6800EF40900DB7560180375501809386C6F2C4
:108C78001306000093052023130505F4EF40D00BDD
:108C8800B707F07FB3F5B700B707C0FCB385F500A9
:108C98006358B00093070000138507006780000041
:108CA800B305B04093D545419307300163C8B70079
:108CB800B7070800B3D5B7406FF0DFFD1387C5FECF
:108CC8009306E0019305000093071000E3C6E6FC55
:108CD800B7070080B3D7E700138507006780000057
:108CE800130101FE232A910083240501232C81000E
:108CF8001304450193942400B3049400232821010C
:108D080003A9C4FF232631012324410113050900C7
:108D180093890500232E1100EFF08FE51307000259
:108D2800B307A74023A0F9009307A000138AC4FF44
:108D380063D0A708130555FF6370440583A784FF14
:108D480063000504B306A74033D7D7003319A90039
:108D58003369E900138684FF3707F03F3367E9007A
:108D6800B397A7006372C40203A644FFB356D600A4
:108D7800B3E7D7006F0040019307000063140506AE
:108D88003707F03F3367E9008320C10103248101DD
:108D980083244101032901018329C100032A810099
:108DA800138507009305070013010102678000007F
:108DB8009306B000B386A640B707F03F3357D900F3
:108DC8003367F700930700006376440183A784FFA5
:108DD800B3D7D700130555013315A900B367F500BC
:108DE8006FF09FFA3315A9003707F03F3367E500A6
:108DF800930700006FF05FF9130101FD232C410177
:108E0800138A0500930510002322910223202103D1
:108E1800232E31012326110223248102232A510102
:108E2800930406009389060013090700EFF08F9F4B
:108E3800630A051093D74401370710001306F7FF9C
:108E480093965701130405003376960093FAF77F3B
:108E5800638406003366E6002326C10063080A0817
:108E68001305810023244101EFF0CFD70327C10068
:108E7800930705006302050C032681009306000290
:108E8800B386A640B316D700B3E6C6003357A7008B
:108E9800232AD4002326E100B334E000938414008D
:108EA800232CE4002328940063840A06938ADABCFE
:108EB800B38AFA001305500323A05901B307F540FC
:108EC8002320F9008320C102130504000324810232
:108ED80083244102032901028329C101032A810154
:108EE800832A410113010103678000001305C100B3
:108EF800EFF04FCF930710002328F4008327C10019
:108F080093041000232AF40093070502E3900AFA59
:108F1800139724003307E400032507019387E7BC70
:108F280023A0F900EFF0CFC493945400B384A44075
:108F3800232099006FF01FF983268100232AD4008B
:108F48006FF09FF5B7560180375501809386C6F2BA
:108F5800130600009305A030130505F4EF40C05D2B
:108F6800130101FD232021031389050093058100C6
:108F7800232611022324810223229102232E310168
:108F880093090500EFF0DFD593040500138405006D
:108F9800130509009305C100EFF09FD48327090149
:108FA80003A709018326C1003307F74083278100FF
:108FB80013175700B387D740B307F7009306050088
:108FC800635EF00293974701338487001386060097
:108FD800138504009386050093050400EF7010388C
:108FE8008320C10203248102832441020329010250
:108FF8008329C1011301010367800000139747010A
:10900800B385E5406FF09FFC130101FF2320210188
:109018002326110023248100232291009307700145
:109028001309050063D6A70483A7812383A5C12359
:1090380003A4012483A44124138507001306040014
:1090480093860400EF80801F1309F9FF930705003A
:10905800E31409FE8320C100032481008324410016
:10906800032901001385070013010101678000002F
:10907800B757018013193500938787F9338927017A
:10908800832709018320C100032481008325490126
:1090980083244100032901001385070013010101FE
:1090A80067800000832606019385F5FF93D5554018
:1090B80093851500930746019396260093952500FE
:1090C800B386D700B305B50063F8D70213070500C8
:1090D80003A807009387470013074700232E07FFBD
:1090E800E3E8D7FEB387C6409387B7FE93F7C7FF79
:1090F800938747003305F5006378B50013054500ED
:10910800232E05FEE36CB5FE6780000003270501EA
:1091180013D65540930645016352C702931727009B
:10912800B387F60063F2F60403A7C7FF9387C7FF68
:10913800E30A07FE13051000678000009317260056
:10914800B387F600E350E6FE93F5F501E38C05FCE2
:1091580003A60700130510003357B600B315B70070
:10916800E302B6FC6780000013050000678000007A
:10917800130101FF23229100B704008023248100FA
:109188002326110093C4F4FF1304060023200600CD
:10919800B3F6B4003706F07F938705001307050080
:1091A80063DEC604B3E8A600638A080433F6C50084
:1091B80013880500930800006310060283A6C124E3
:1091C80003A68124EF808007130705001388050094
:1091D800B3F6B4009308A0FC93D64641B7071080B5
:1091E8009387F7FF938626C03378F800B386160175
:1091F800B707E03FB367F8002320D4008320C100FD
:109208000324810083244100130507009385070088
:109218001301010167800000130101FF232481006D
:10922800232291001304050013850500232611004D
:1092380023AE0130EF70CFAD9307F0FF630CF5005C
:109248008320C1000324810083244100130101010C
:109258006780000083A7C131E38407FE8320C10033
:109268002320F40003248100832441001301010119
:1092780067800000130101F6930EC108232AF10844
:1092880037030080B707FFFF138E05001343F3FF72
:109298002326D108938787209305810093860E00A3
:1092A800232E1106232AF1002328E108232C010983
:1092B800232E11092324C101232CC101232E61006F
:1092C800232861002322D101EF00003D832781007C
:1092D800238007008320C1071301010A678000006B
:1092E800130E0500130101F603A5C125930E81088D
:1092F800232AF10837030080B707FFFF1343F3FF62
:109308002324C1082326D1089387872013860500C4
:1093180093860E0093058100232E1106232AF1005F
:109328002328E108232C0109232E11092324C10134
:10933800232CC101232E6100232861002322D1019F
:10934800EF00803583278100238007008320C10731
:109358001301010A67800000130101FF2324810023
:10936800138405008395E50023261100EF40907CC7
:1093780063400502832704058320C100B387A70043
:109388002328F404032481001301010167800000ED
:109398008357C40037F7FFFF1307F7FFB3F7E7005A
:1093A8008320C1002316F400032481001301010166
:1093B8006780000013050000678000008397C500E0
:1093C800130101FE232C8100232A91002328210167
:1093D80023263101232E110013F7071013840500EB
:1093E800930405008395E500130906009389060098
:1093F800631E070237F7FFFF1307F7FFB3F7E7000E
:109408002316F400032481018320C10193860900F7
:10941800130609008329C1000329010113850400EB
:1094280083244101130101026F40800A9306200042
:1094380013060000EF40D03E8317C4008315E400F4
:109448006FF05FFB130101FF2324810013840500E3
:109458008395E50023261100EF40903C9307F0FF29
:109468006304F5028357C400371700008320C10046
:10947800B3E7E7002328A4042316F400032481009B
:1094880013010101678000008357C40037F7FFFF0D
:109498001307F7FFB3F7E7008320C1002316F40092
:1094A8000324810013010101678000008395E50012
:1094B8006F40001AB367B50093F737006392070847
:1094C80003A70500B7867F7F9386F6F7B377D700A3
:1094D800B387D700B3E7E700B3E7D7001306F0FF79
:1094E800639EC706130605001308F0FF2320E60055
:1094F80003A745009385450013064600B377D700B8
:10950800B387D700B3E7E700B3E7D700E38007FFE7
:1095180083C7050003C7150083C625002300F6008E
:10952800638A0700A300E600630607002301D6004C
:109538006394060067800000A301060067800000AE
:109548009307050003C70500938717009385150047
:10955800A38FE7FEE31807FE6780000013060500E7
:109568006FF01FFB9377350013070500639C070412
:10957800B7867F7F9386F6F79305F0FF03260700EB
:1095880013074700B377D600B387D700B3E7C70000
:10959800B3E7D700E384B7FE8346C7FF0346D7FF88
:1095A8008347E7FF3307A74063800604630A060280
:1095B8003335F0003305E5001305E5FF678000004B
:1095C800E38806FA834707001307170093763700E6
:1095D800E39807FE3307A7401305F7FF67800000ED
:1095E8001305D7FF678000001305C7FF67800000D9
:1095F800B3E7A50093F7370013070500639807063C
:109608009307300063F4C7063703FFFEB7888080EE
:109618001303F3EF93880808130E300083A60500A0
:10962800B387660013C8F6FFB3F70701B3F717014E
:10963800639E07022320D7001306C6FF13074700BF
:1096480093854500E36CCEFC9385150093071700BE
:109658006304060283C6F5FF1308F6FFA38FD7FE3F
:10966800638E06001387070013060800938515000C
:1096780093071700E31006FE678000003306C70053
:10968800630A080093871700A38F07FEE39CC7FEB1
:109698006780000067800000130101E12326111E86
:1096A8002320211F2324811D2320A11D138C0500A5
:1096B80013090600232AD1002324811E2322911E88
:1096C800232E311D232C411D232A511D2328611DC2
:1096D8002326711D2322911D232EB11B130D050076
:1096E800EFD01FED83270500138507002328F1021B
:1096F800EFF05FE70357CC002328010E232A010E61
:10970800232C010E232E010E137707082326A1020E
:109718006308070003270C01631407006F10C05685
:109728009307C110375701802322F10E9388070051
:109738009307070C37570180232CF100130B0900FE
:109748009307C7232324F10083470B002326010E28
:109758002324010E23200102232A0102232C0102C3
:10976800232E0102232401042326010423260100B9
:109778006384072213040B00930650026384D72CDA
:109788008347140013041400E39A07FEB3046441EA
:10979800630464218326C10E8327810E23A06801F8
:1097A800B38696009387170023A298002326D10E2C
:1097B8002324F10E930670009388880063CCF62862
:1097C8000327C10083470400330797002326E100DD
:1097D8006384071C83441400A303010C13041400BE
:1097E800930DF0FF93090000130A00001309A00568
:1097F800930A9000930BA002938C080013041400A2
:10980800938704FE6364F904032781019397270073
:10981800B387E70083A70700678007009309000064
:10982800938604FD8344040093972900B387370186
:1098380093971700B389F600938604FD1304140068
:10984800E3F2DAFE938704FEE370F9FC93880C00D8
:109858006384041423069114A303010C930A1000D3
:10986800930C1000130BC11423280100930D000062
:109878002324010223220102232E0100937B2A00C4
:1098880063840B00938A2A0013794A088327C10E40
:109898006316090033885941E34C00638346710C11
:1098A800638A06028326810E1306710C23A0C80062
:1098B80093871700130610009386160023A2C8008A
:1098C8002326F10E2324D10E1306700093888800F6
:1098D800634CD64C638A0B028326810E1306810CD7
:1098E80023A0C8009387270013062000938616003C
:1098F80023A2C8002326F10E2324D10E13067000DC
:1099080093888800E34CD66A93060008E300D9429E
:10991800B38D9D41E34EB04D93760A10E39A062C21
:109928000327810EB387970123A068011307170047
:1099380023A298012326F10E2324E10E930670003A
:1099480063C0E65A93888800137A4A0063060A00BF
:10995800B38459416346905A63D4590193890A00E4
:109968000327C100330737012326E100E39C075290
:10997800832701012324010E638807008325010141
:1099880013050D00EFA09FC59308C110130B040029
:1099980083470B00E39007DE8327C10E638407002B
:1099A8006F1050340357CC00137707046304070083
:1099B8006F20803F8320C11E0324811E0325C10020
:1099C8008324411E0329011E8329C11D032A811DE9
:1099D800832A411D032B011D832BC11C032C811CD1
:1099E800832C411C032D011C832DC11B1301011F56
:1099F8006780000013050D00EFD09FBB832745004B
:109A0800138507002326F104EFF0DFB5930705005F
:109A180013050D00938407002324F104EFD05FB9E8
:109A280083278500232EF102638404006F104016FB
:109A3800834404006FF09FDC83440400136A0A0225
:109A48006FF0DFDBB3046441E31664D58347040099
:109A58006FF01FD81306410E93050C0013050D0077
:109A6800EF50C002E31005F49308C1106FF05FD502
:109A780093778A0093880C00638407006F10800A2C
:109A8800832741011305010B232891019387770050
:109A980093F787FF83A5070003A6470093878700EE
:109AA800232AF100EFA090038327010B83280101EB
:109AB8002328F10E8327410B232AF10E8327810BDC
:109AC800232CF10E8327C10B232EF10E1305010F52
:109AD80023281101EFD01FA72326A10C93072000EC
:109AE800832801016314F5006F1080659307100047
:109AF8006314F5006F105007930710066394F40081
:109B08006F20C019930710046394F4006F10D052AB
:109B180093FBF4FD9307F0FF232A71056394FD007E
:109B28006F105021930770046394FB006F20801E10
:109B38000323C10F23244103032E010F832E410F5A
:109B4800032F810F93670A10635403006F20C039F5
:109B5800232C0104138A07002328010093076004BB
:109B68006394FB006F10902B930750042322110578
:109B78006384FB006F10D03313891D00930A010B17
:109B8800930609001308C10D9307010D1307C10CB3
:109B98001306200093850A0013050D002328C10B26
:109BA8002320C105232AD10B2322D103232CE10B27
:109BB8002320E103232E610A232E6100EFC00FEF5B
:109BC8000323C101032F0102832E4102032E010446
:109BD80083284104130B050033092501930C010A5E
:109BE80093850C0013850A00232E11012328C10B2D
:109BF800232AD10B232CE10B232E610A2320010AEF
:109C08002322010A2324010A2326010AEF70503F68
:109C18008328C10113070900630205020327C10D48
:109C2800637E27019306000393071700232EF10C88
:109C38002300D7000327C10DE36827FFB307674157
:109C48002320F1020327C10C93077004232EE1009F
:109C5800032741056314F7006F10501103274105CE
:109C6800930760046314F7006F10D0348327C10191
:109C780003274105930510049387F7FF2326F10C6A
:109C880093F6F40F130600006318B7009386F600E6
:109C980093F6F60F13061000230AD10C9306B002B0
:109CA80063DA07000327C101930710009306D00267
:109CB800B387E740A30AD10C9306900063C4F6006B
:109CC8006F20400F1308310E130508001306A0007B
:109CD800130E300633E7C702930505009386070085
:109CE8001305F5FF13070703A38FE5FEB3C7C702E4
:109CF800E342DEFE9387070313F6F70FA30FC5FEB3
:109D08009387E5FF63E407016F2080399306610DAF
:109D18006F00800003C607002380C60093871700E2
:109D280093861600E39807FF9307510EB387B74051
:109D38001307610DB307F7009306410DB387D740AA
:109D4800232CF102032701028326810393071000C5
:109D5800B30CD70063C4E7006F2000238327C10238
:109D6800B38CFC008327810293CAFCFF93DAFA4183
:109D780013FAF7BF136A0A10B3FA5C01232401022D
:109D880023220102232E0100832781056394070003
:109D98006F1010059307D002A303F10C930D000078
:109DA800938A1A006FF09FAD1306410E93050C00BD
:109DB80013050D00EF40904DE31005108327C10EE9
:109DC8009308C1106FF01FB18326810E938C170082
:109DD800832701021306100023A06801938416004C
:109DE80013898800E358F6369307100023A2F80079
:109DF8002326910F2324910E93077000E3C0974AFE
:109E08008327C1020327010393841400B38CFC0049
:109E18002322F9002320E9002326910F2324910E01
:109E28009307700013098900E3CC97488327010F33
:109E3800138614009305010A2328F10A8327410F8A
:109E48001305010B232EC100232AF10A8327810F52
:109E58002320010A2322010A232CF10A8327C10F98
:109E68002324010A2326010A232EF10AEF70501930
:109E78000326C1018327010293088900930606007F
:109E8800938DF7FFE30C052E13071B00B38CBC0161
:109E98002320E9002322B9012326910F2324C10E90
:109EA8009307700063D4C7006F10800193070901FE
:109EB80093862400138908009388070003268103EA
:109EC8001307410D2320E900B30796012322C90097
:109ED8002326F10E2324D10E13077000E356D7A6CC
:109EE8001306410E93050C0013050D00EF40103AC0
:109EF8006314057C8327C10E9308C1106FF0DFA49B
:109F0800930600010327810E63C496006F10101298
:109F1800B7560180938EC62213090001130A7000F8
:109F2800138B0E006F00C000938404FF63569904DE
:109F3800938707011307170023A0680123A22801AC
:109F48002326F10E2324E10E93888800E35EEAFCC1
:109F58001306410E93050C0013050D00EF40103356
:109F6800631C0574938404FF8327C10E0327810EA5
:109F78009308C110E34E99FA930E0B00B38797002C
:109F88001307170023A0D80123A298002326F10E57
:109F98002324E10E93067000E3D0E69C1306410EDD
:109FA80093050C0013050D00EF40502E6316057045
:109FB8008327C10E6FF05F9A83274101A303010C29
:109FC80093880C0003AB070013894700E3020B4E8C
:109FD8009307F0FF6394FD006F10C01F13860D00F8
:109FE8009305000013050B00232A9101EFD0DFF53C
:109FF8002328A10083284101631405006F10C07550
:10A0080083270101232A210123280100B38C6741FA
:10A018008347710C93CAFCFF93DAFA4123240102A7
:10A0280023220102232E0100B3FA5C01930D0000E4
:10A03800E3860784938A1A006FF05F84032741013F
:10A0480093880C00A303010C83270700130747001C
:10A05800232AE1002306F114930A1000930C100040
:10A06800130BC1146FF05F8083440400136A4A0025
:10A078006FF0CFF88326410193770A0293880C008A
:10A0880003A7060093864600232AD100E3900728F9
:10A0980093770A01638407006F10C01293770A044C
:10A0A800638407006F10803D137A0A2063140A0046
:10A0B8006F1040118327C100130B04002300F70021
:10A0C8006FF01F8D834404009307C006E38EF438B5
:10A0D800136A0A016FF08FF203274101B787FFFF68
:10A0E80093C707832314F10C93074700232AF10031
:10A0F80003290700B7570180938747AF93880C005F
:10A10800232AF102930C0000936B2A009307200086
:10A1180093048007A303010C1307F0FF6386ED2067
:10A128003367990113FAFBF7631E071E63940D2624
:10A138006390071C93FC1B00130B011BE3900C1C82
:10A14800938A0C0063D4BC01938A0D008347710C79
:10A15800232801002324010223220102232E0100C7
:10A16800E39A07EC6FF08FF193880C00136A0A01E9
:10A1780093770A02E38C070683274101138B770044
:10A18800137B8BFF03290B00832C4B0093078B0059
:10A19800232AF100937BFABF930700006FF09FF723
:10A1A8008344040093078006E388F42C136A0A04A6
:10A1B8006FF0CFE493880C00936B0A0193F70B02BE
:10A1C800E38C070483274101138B7700137B8BFFF4
:10A1D80093078B00232AF10003290B00832C4B00E3
:10A1E800930710006FF01FF383440400136A8A007A
:10A1F8006FF0CFE0832741018344040083A907005F
:10A2080093874700232AF10063DA09DEB309304156
:10A21800136A4A006FF08FDE83440400136A1A0041
:10A228006FF0CFDD8347710C83440400639807DC2B
:10A2380093070002A303F10C6FF04FDC8344040082
:10A24800136A0A086FF08FDB8344040013071400B5
:10A25800639474016F10505F938604FD1304070024
:10A26800930D000063EEDAD88344040093972D0021
:10A27800B387B70193971700B38DD700938604FD72
:10A2880013041400E3F2DAFE6FF08FD79307B002DD
:10A2980083440400A303F10C6FF04FD693880C009D
:10A2A800136A0A0193770A026380077A83274101B8
:10A2B800138B7700137B8BFF83274B0003290B003D
:10A2C80013078B00232AE100938C070063C6077AE3
:10A2D8009307F0FF930B0A006384FD02B3679901AB
:10A2E800937BFAF7639E070063920D02138A0B00B3
:10A2F800930D0000930C0000130B011B6FF05FE43B
:10A30800E3960C4093079000E3E227411309090301
:10A31800A307211B138A0B00930C1000130BF11ACF
:10A328006FF01FE2930B0A0013071000E38AE7FCA3
:10A3380013072000638CE706130B011B1397DC013E
:10A3480093777900135939009387070333692701F5
:10A3580093DC3C00A30FFBFE3367990113060B0047
:10A36800130BFBFFE31C07FC93F61B00638A06062E
:10A37800930600036386D7061306E6FF9307011BBF
:10A38800A30FDBFEB38CC740138A0B00130B060028
:10A398006FF01FDB130710006394E7006F101017AE
:10A3A80013072000930B0A00E398E7F8832641037C
:10A3B800130B011B9377F900B387F60003C7070057
:10A3C800135949009397CC0133E9270193DC4C00DA
:10A3D800A30FEBFEB3679901130BFBFFE39C07FC8C
:10A3E8009307011BB38C6741138A0B006FF05FD58D
:10A3F80093065006E3DA969C8326010F9305010A1B
:10A408001305010B2328D10A8326410F23221105A6
:10A418002320F104232AD10A8326810F2320010A4D
:10A428002322010A232CD10A8326C10F2324010ADF
:10A438002326010A232ED10AEF70803C83270104CA
:10A4480083284104631C05380327810EB756018011
:10A458009386C68C23A0D800938717009306100014
:10A468001307170023A2D8002326F10E2324E10E98
:10A478009306700093888800E3CCE6440327C10C58
:10A48800832601026350D766032701038326C1028E
:10A498009388880023ACE8FE0327810EB387D70092
:10A4A80023AED8FE130717002326F10E2324E10E4E
:10A4B8009306700063CCE676032701029304F7FF46
:10A4C800635490C8930600010327810EE3D2964295
:10A4D80013090001930C70006F00C000938404FFFF
:10A4E800E3589940832681009387070113071700D3
:10A4F80023A0D80023A228012326F10E2324E10E4D
:10A5080093888800E3DCECFC1306410E93050C00ED
:10A5180013050D00EF4080576310051A8327C10EFD
:10A528000327810E9308C1106FF05FFB33895941EF
:10A53800635020BF130600018326810E635426074B
:10A54800130E0001930B70006F00C000130909FF80
:10A55800635A2E0503278100938707019386160007
:10A5680023A0E80023A2C8012326F10E2324D10E3C
:10A5780093888800E3DCDBFC1306410E93050C008E
:10A5880013050D00EF40805063180512130E0001EB
:10A59800130909FF8327C10E8326810E9308C11072
:10A5A800E34A2EFB03278100B38727019386160011
:10A5B80023A0E80023A228012326F10E2324D10E8C
:10A5C80013067000938888006354D6B41306410EAE
:10A5D80093050C0013050D00EF40404B631E050C5E
:10A5E800B38D9D418327C10E9308C1106356B0B344
:10A5F800130600018326810E6352B607930B0001F0
:10A60800130970006F00C000938D0DFF63D8BB0560
:10A6180003278100938707019386160023A0E8008B
:10A6280023A278012326F10E2324D10E93888800D3
:10A63800E35CD9FC1306410E93050C0013050D00CD
:10A64800EF40C044631A0506938D0DFF8327C10EA2
:10A658008326810E9308C110E3CCBBFB032781003E
:10A66800B387B7019386160023A0E80023A2B80198
:10A678002326F10E2324D10E130670009388880038
:10A68800635CD6A81306410E93050C0013050D0054
:10A69800EF40C03F631205028327C10E9308C11023
:10A6A8006FF08FA71306410E93050C0013050D00DC
:10A6B800EF40C03D630E05AA832B010163840BAEF6
:10A6C80093850B0013050D00EF905FF16FF08FADD0
:10A6D80037570180130600018326810E930EC72287
:10A6E800635C0609232081042322910413040D00CE
:10A6F80093040C00130E000193027000130C080061
:10A70800138D0E006F00C000130C0CFF635A8E05EA
:10A71800938707019386160023A0A80123A2C801E6
:10A728002326F10E2324D10E93888800E3DED2FC81
:10A738001306410E9385040013050400EF4000350D
:10A74800E3120516130E0001130C0CFF8327C10E2C
:10A758008326810E9308C11093027000E34A8EFB92
:10A7680013080C00930E0D00138C0400130D040045
:10A778008324410403240104B38707019386160048
:10A7880023A0D80123A208012326F10E2324D10EE9
:10A7980013067000938888006352D6901306410E02
:10A7A80093050C0013050D00EF40402EE31605F04D
:10A7B8008327C10E9308C1106FF04F8E1306410E08
:10A7C80093050C0013050D00EF40402CE31605EE31
:10A7D8008327C10E9308C1106FF00F938325C10C16
:10A7E800635CB07E0327C10183260102930407003E
:10A7F80063C2E63C635690028326810EB3879700B6
:10A8080023A068019386160023A298002326F10E40
:10A818002324D10E1306700093888800E34CD64099
:10A8280093C6F4FF0327C10193D6F641B3F4D400CD
:10A83800B3049740634E90480327C10193760A40BA
:10A84800B30DEB00639A064E8324C10C0327010263
:10A8580063C6E40093761A00E38206408326010368
:10A868000327C1021306700023A0D8008326810E97
:10A87800B387E70023A2E800938616002326F10E8B
:10A888002324D10E93888800E344D66A83260102E4
:10A898003307DB00B38496403307B74113890400BC
:10A8A8006354970013090700635620030327810E9A
:10A8B800B387270123A0B8011307170023A2280193
:10A8C8002326F10E2324E10E930670009388880056
:10A8D800E3CAE66A1347F9FF1357F7413377E900EC
:10A8E800B384E440634490006FF00F869306000140
:10A8F8000327810E63DE967E13090001930C700016
:10A908006F00C000938404FF6354997E83268100FE
:10A91800938707011307170023A0D80023A2280153
:10A928002326F10E2324E10E93888800E3DCECFC57
:10A938001306410E93050C0013050D00EF4000159A
:10A94800E31C05D68327C10E0327810E9308C11087
:10A958006FF05FFB93771A00639807C823A2C800BB
:10A968002326910F2324910E9307700063CA9754EE
:10A9780093862600938808016FF04FD46350B0D5B2
:10A98800130700016344B7016F10806B130B70004D
:10A99800930406006F000001938D0DFFE35EB7116D
:10A9A8009384140083278100938C0C012322E900EF
:10A9B8002320F9002326910F2324910E13098900DF
:10A9C800E35C9BFC1306410E93050C0013050D0078
:10A9D800EF40C00BE31205CE832CC10E8324810EF9
:10A9E8001309C110130700016FF01FFB83264101F3
:10A9F80093770A01138746006394071893770A042C
:10AA0800E386071483274101930C0000232AE10001
:10AA180003D907006FF00FF88326410193F70B0164
:10AA2800138746006394071493F70B04E380071019
:10AA380083274101930C0000232AE10003D9070072
:10AA4800930710006FF00FED8326410193770A01F9
:10AA5800138746006392071093770A04E388070A6E
:10AA680083274101232AE10003990700935CF941F8
:10AA780093870C00E3DE0784B3372001B30C9041C1
:10AA8800B38CFC409307D002A303F10C3309204197
:10AA9800930B0A00930710006FF00FE81306410E9E
:10AAA80093050C0013050D00EF30507EE31605C02A
:10AAB800832CC10E8324810E1309C1106FF04FB48B
:10AAC8001306410E93050C0013050D00EF30107CA2
:10AAD800E31405BE832CC10E8324810E1309C11013
:10AAE8006FF0CFB413771A00631407006FE0DFE547
:10AAF8006FF09F9993880C006FF0CFFA93070003CB
:10AB0800A307F11A130BF11A6FF08FE38326C10024
:10AB1800130B040093D7F6412320D7002322F70014
:10AB28006FE01FE70327410183270700130747004A
:10AB3800232AE10083A5070003A6470083A6870010
:10AB480083A7C7002328B10E232AC10E232CD10EB8
:10AB5800232EF10E6FE09FF703A90600232AE100D8
:10AB6800935CF94193870C006FF04FF603A9060038
:10AB7800930C0000232AE100930710006FF08FD98F
:10AB880003A90600930C0000232AE1006FF08FE070
:10AB98008327C10383440400639407006FE01FC642
:10ABA80083C70700639407006FE05FC5136A0A4014
:10ABB8006FE0DFC493840600E34090C46FF05FC683
:10ABC80093880C00930B0A006FF04FDFB757018092
:10ABD800938747AF93880C00232AF10293770A02E0
:10ABE8006380072C83274101138B7700137B8BFF2E
:10ABF80003290B00832C4B0093078B00232AF100B9
:10AC080093771A00638E0700B3679901638A070078
:10AC1800930700032304F10CA304910C136A2A0080
:10AC2800937BFABF930720006FF0CFCE1306410E37
:10AC380093050C0013050D00EF305065E31E05A6C3
:10AC48008327C10E9308C1106FF01F87B757018083
:10AC5800938787B093880C00232AF1026FF01FF8BE
:10AC680093880C006FF0CFD083441400136A0A0253
:10AC7800130414006FE09FB883441400136A0A2079
:10AC8800130414006FE09FB79305000413050D002B
:10AC9800EFC01FB22320AC002328AC0063140500CA
:10ACA8006F10C03C13070004232AEC006FE05FA775
:10ACB80093076000938C0D0063EEB77937570180D6
:10ACC800938A0C00232A2101130BC7B16FE0DFB967
:10ACD800130600018326810E6358966A930C0001BF
:10ACE800930D70006F00C000938404FF63DE9C68BE
:10ACF80003278100938707019386160023A0E800A5
:10AD080023A298012326F10E2324D10E93888800CC
:10AD1800E3DCDDFC1306410E93050C0013050D0062
:10AD2800EF30D056E31A05988327C10E8326810E8B
:10AD38009308C1106FF05FFB03270102832C4102C7
:10AD4800232E41012320810423223105232251038C
:10AD58008329810223246103B30BEB000324C1037D
:10AD6800032A8104832AC104930470001309000193
:10AD7800130B0C0063880C08639809081304F4FF8C
:10AD8800938CFCFF0327810EB387470123A058014A
:10AD98001307170023A248012326F10E2324E10EEE
:10ADA8009388880063C4E414834604003386BB4157
:10ADB800138C06006354D600130C060063568003F8
:10ADC8008326810EB387870123A0B80193861600D6
:10ADD80023A288012326F10E2324D10E63C0D43484
:10ADE80083460400938888001346FCFF1356F641F7
:10ADF8003377CC00338CE640634C8001B38DDD00A3
:10AE0800E39C0CF6638C09729389F9FF6FF09FF746
:10AE18008326810E634889016F008005130C0CFF9F
:10AE280063588905032781009387070193861600D5
:10AE380023A0E80023A228012326F10E2324D10E03
:10AE480093888800E3DCD4FC1306410E93050B00BD
:10AE580013050D00EF309043631C055A130C0CFFCB
:10AE68008327C10E8326810E9308C110E34C89FB0A
:10AE780003278100B38787019386160023A0E80083
:10AE880023A288012326F10E2324D10E63C4D4768D
:10AE98008346040093888800B38DDD006FF05FF669
:10AEA8008326410193770A011387460063840720AC
:10AEB80003A90600930C0000232AE1006FF05FD479
:10AEC8001306410E93050C0013050D00EF30103CDE
:10AED800631405FE8326810E832CC10E930841114D
:10AEE800938616001309C1106FE05FFD1306410E2B
:10AEF80093050B0013050D00EF305039631A055008
:10AF08008327C10E9308C1106FF01FEA130B011BB2
:10AF18009307000023288100232E910013040B00BF
:10AF280023223103130B0C009304090093890C00AE
:10AF380013FA0B40832CC103930AF00F138C0800FB
:10AF4800138907006F0040021306A0009306000053
:10AF58001385040093850900EF50003C6380094C79
:10AF680093040500938905001306A00093060000CA
:10AF78001385040093850900EF50407D13050503F0
:10AF8800A30FA4FE130919001304F4FFE30E0AFA31
:10AF980083C60C00E31AD9FAE30859FB639A0942FD
:10AFA8009307900063E6974293080C009307011BF0
:10AFB800130C0B00130B0400232E91038324C101EF
:10AFC800832941020324010123202103B38C674113
:10AFD800138A0B006FF0CF968326810E37560180B7
:10AFE8001306C68C23A0C800938717001306100009
:10AFF8009386160023A2C8002326F10E2324D10E1F
:10B008001306700093888800634CD6066398052061
:10B018000327010293761A00B3E6E600639406005C
:10B028006FE09F92832601030327C1021306700075
:10B0380023A0D8008326810EB387E70023A2E80067
:10B04800938616002326F10E2324D10E634ED64A8A
:10B0580093888800032701029386160023A06801BD
:10B06800B387E70023A2E8002326F10E2324D10E9C
:10B07800130770006344D7006FE0DF8C6FE05FE672
:10B088001306410E93050C0013050D00EF30102038
:10B09800631405E28325C10C8327C10E9308C110F0
:10B0A8006FF0DFF6832B0101130D0400138C0400ED
:10B0B8006FF0CFE093770A04638C0722832741015E
:10B0C800930C0000232AE10003D907006FF05FB357
:10B0D8001306410E93050C0013050D00EF30101BED
:10B0E800631C05DC8327C10E9308C1106FF00FB9EC
:10B0F80083268100B387970023A2980023A0D80055
:10B10800130717002326F10E2324E10E930670007F
:10B1180063C4E6006FE01F836FE09FDC1306410EF7
:10B1280093050B0013050D00EF3050166312052E22
:10B13800834604008327C10E9308C1106FF0DFCA4D
:10B148008327010F9305010A1305010B2328F10A30
:10B158008327410F2320010A2322010A232AF10A07
:10B168008327810F2324010A2326010A232CF10AAD
:10B178008327C10F232EF10AEF609009832801016C
:10B18800634205528347710C13077004635E972866
:10B1980037570180130B87AE2328010023240102AF
:10B1A80023220102232E0100137AFAF7930A3000B2
:10B1B800930C3000930D0000638407006FE09FE755
:10B1C8006FE0CFEB8327C100130B04002320F700A7
:10B1D8006FE00FFC13050B0023209105EFE08FB8FB
:10B1E8008347710C934AF5FF93DAFA41232A210128
:10B1F800232801002324010223220102232E010017
:10B2080083280104930C0500B37A5501930D0000BF
:10B21800638407006FE01FE26FE04FE683260103B7
:10B228000327C1021306700023A0D8008326810ECD
:10B23800B387E70023A2E800938616002326F10EC1
:10B248002324D10E938888006340D62CE3D405E0EC
:10B25800130600FFB304B040E3D4C5261309000168
:10B26800930C70006F00C000938404FFE35A992484
:10B2780003278100938707019386160023A0E8001F
:10B2880023A228012326F10E2324D10E93888800B7
:10B29800E3DCDCFC1306410E93050C0013050D00DE
:10B2A800EF30C07E631A05C08327C10E8326810E46
:10B2B8009308C1106FF05FFB938614001307890091
:10B2C80083278100B38CBC012322B9012320F90014
:10B2D8002326910F2324D10E93077000E3C2D7BE13
:10B2E8009386160093088700130907006FE01FBDB7
:10B2F80093770A20638E071C83274101930C000073
:10B30800232AE10003C907006FF09F8F93770A2073
:10B318006384071A83274101232AE1000389070070
:10B32800935CF94193870C006FE05FFA93F70B2069
:10B338006388071683274101930C0000232AE10044
:10B3480003C90700930710006FE0DFDC93770A203A
:10B35800638E071283274101930C0000232AE10022
:10B3680003C907006FE01FE38327C10F63C80718ED
:10B378008347710C13077004635C97463757018045
:10B38800130B07AF6FF05FE103278100B3879700C6
:10B398009386160023A0E80023A298002326F10E26
:10B3A8002324D10E13067000938888006356D6C8EC
:10B3B8001306410E93050C0013050D00EF30006DC8
:10B3C800631C05AE8327C10E9308C1106FF0CFC66A
:10B3D800832781048325C104130900003304F44042
:10B3E8001386070013050400EFE08FA083C51C0037
:10B3F8001306A000930600003338B000138504003C
:10B4080093850900B38C0C01EF4010716FF05FB5A4
:10B41800832B0101130C0B006FF04FAA93079000C8
:10B42800E3E097B46FF05FB837570180130B47AE6E
:10B438006FF09FD61306410E93050C0013050D00FF
:10B44800EF30C064631A05A68327C10E9308C110A4
:10B458006FF00FBD930C60006FF05F8683260102CA
:10B468003307DB00B38496403308B74113890400DF
:10B47800635298C6130908006FF0CFC58327C1002F
:10B48800130B04002310F7006FE08FD083274101CE
:10B49800930C0000232AE10003A907006FE09FCF67
:10B4A80083274101930C0000232AE10003A9070028
:10B4B800930710006FE01FC683274101232AE1008C
:10B4C80003A90700935CF94193870C006FE01FE024
:10B4D80083274101930C0000232AE10003A90700F8
:10B4E8006FF00FF21306410E93050C0013050D00C3
:10B4F800EF30C0590357CC006FE00FCB9307D00251
:10B50800A303F10C6FF01FE71306410E93050C001F
:10B5180013050D00EF3080576310059A8325C10C81
:10B528008327C10E8326810E9308C110E3D405B288
:10B538006FF01FD2930D60006FE08FDF03270102C9
:10B54800130C0B00032B8102232E8102032AC10155
:10B55800B306EB000324010483294104832A410232
:10B5680063F4B6AF938D06006FF00FAE0327C101E9
:10B578009307D0FF6344F70063DAED009384E4FF98
:10B5880093F7F4FD232AF1046FE04FEE83270102BD
:10B598000327C1016344F72683278102930C070020
:10B5A80093F71700638607008327C102B30CF700DF
:10B5B8008327810293F70740638607008327C10129
:10B5C800E34AF01293CAFCFF93DAFA41B3FA5C013A
:10B5D8009304700623240102232201026FE0CFFAAC
:10B5E8008347710C930D0000638407006FE09FA4EC
:10B5F8006FE0CFA81306410E93050B0013050D004D
:10B60800EF30C048E31605E0834604008327C10EE7
:10B618009308C110B38DDD006FF08FFE930A010B04
:10B628001308C10D9307010D1307C10C93860D0074
:10B638001306300093850A0013050D002322110517
:10B648002328C10B2320C105232AD10B2322D10390
:10B65800232CE10B2320E103232E610A232E610012
:10B66800EFA0DFC40323C101032F0102832E41028F
:10B67800032E010483284104130B0500930760047B
:10B688003309BB01639AFB6283460B0093070003EF
:10B69800E386F610930C010A8327C10C3309F900DD
:10B6A8006FE00FD49307D002A303F10C6FF0DFAD66
:10B6B800930A010B9307010D1308C10D1307C10C61
:10B6C80093860D001306200093850A0013050D00CC
:10B6D8002328C10B2320C105232AD10B2322D10300
:10B6E800232CE10B2320E103232E610A232E610082
:10B6F800EFA0DFBB930770040323C101032F0102EE
:10B70800832E4102032E010483284104130B0500F4
:10B71800E396FBF68327810293F71700639807588F
:10B72800930770040327C10D232AF1046FE00FD19A
:10B738001306410E93050C0013050D00EF3000357C
:10B74800630405006FE05FF78324C10C8327C10EF3
:10B758009308C1106FF08F938347710C232A21013E
:10B768002324010223220102232E0100938A0D00C3
:10B77800938C0D00930D0000638407006FE09F8B8E
:10B788006FE0CF8F1306410E93050C0013050D00D3
:10B79800EF30C02F630405006FE01FF28324C10C53
:10B7A800032701028327C10E9308C110B3049740F1
:10B7B8006FF04F92832781020327C10193F7170087
:10B7C800B3E7B701E354E0046396077A832CC10119
:10B7D800930460068327810293F70740639E0770EE
:10B7E80093CAFCFF93DAFA41B3FA5C016FF09FDE6B
:10B7F80037570180130BC7AE6FF01F9A83270102DA
:10B808000327C10293047006B38CE7008327C101A4
:10B81800E342F0FCB38CFC40938C1C0093CAFCFF01
:10B8280093DAFA41B3FA5C016FF0DFDAB7560180B8
:10B83800938EC6226FE08FF4930700032304F10C64
:10B848009307800513672A00A304F10C2324E1025F
:10B858009307300623280100130BC11463CEB741A8
:10B868000323C10F93FBF4FD232A7105232C010444
:10B87800032E010F832E410F032F810F136A2A1005
:10B888006342033893071006638EF4549307100439
:10B898006384F4006FE08FAC930A010B13850A00F0
:10B8A800232811052328C10B232AD10B232CE10BB4
:10B8B800232E610AEF80D0411306C10CEFD05F8BB5
:10B8C800138605009305050013850A00EF801021F3
:10B8D8008327010B930C010A130901092328F10896
:10B8E8008327410B1306010893050900232AF10851
:10B8F8008327810B13850C002320C104232CF10816
:10B908008327C10B2320010823220108232EF108D5
:10B91800B707FC3F2326F10823240108EF608023A2
:10B928000328010A032E410A832E810A032FC10A24
:10B9380093850C0013850A002328010B2322010597
:10B94800232AC10B2322C103232CD10B2320D1038B
:10B95800232EE10B232EE1012320010A2322010AD1
:10B968002324010A2326010AEF509069032FC101FD
:10B97800832E0102032E4102032841048328010576
:10B9880063160500930710002326F10CB7570180B2
:10B99800938787B02322F1029386FDFF232E41056A
:10B9A800232291062326B107232AA107232C8107E6
:10B9B800930B0B002320810623243107232811072A
:10B9C800138C0600232E6107130D0800930D0E003B
:10B9D80093840E00130A0F006F00800493850C00F7
:10B9E80013850A002320C102232EF101232CF10B19
:10B9F800232EC10A2328610B232A310B2320010A95
:10BA08002322010A2324010A2326010AEF50505F4A
:10BA1800832FC10103260102130CFCFF6302050EEC
:10BA2800B70703401306090093850C0013850A0025
:10BA3800232EF1082320A10B2322B10B2324910AE2
:10BA48002326410B23280108232A0108232C010857
:10BA5800EF60401013850A00EF800062930505002F
:10BA68001304050013850A008329010B8324410B65
:10BA7800032B810B032AC10BEF8040710327010BB5
:10BA880003260104930509002320E1080327410B3D
:10BA980013850C00232831092322E1080327810B91
:10BAA800232A9108232C61092324E1080327C10BC9
:10BAB800232E41092326E108EF70000A832741025B
:10BAC800032B010A8329410A3387870003470700AC
:10BAD800832F810A0326C10A232871052380EB00DE
:10BAE800232281059307F0FF938B1B00130D0B0096
:10BAF800938D090093840F00130A0600E310FCEEEF
:10BB08008328010793030B00938209003709FE3F3E
:10BB180093850C0013850A0023201103232E81002E
:10BB2800032AC10583244106032401062328710A38
:10BB380023227106232A510A23205106232CF10BB4
:10BB4800232EF105232EC10A2320C1042320010A34
:10BB58002322010A2324010A2326210BEF50105720
:10BB6800832DC106032D4107032C8107032BC10731
:10BB780083298106832801026340A00A83234106A2
:10BB880083220106832FC1050326010493850C0037
:10BB980013850A002328710A232A510A232CF10B42
:10BBA800232EC10A2320010A2322010A2324010A81
:10BBB8002326210BEF50D044832801026318050087
:10BBC8008327C10193FC170063980C048327410461
:10BBD8001306000393861700B386DB0063C80700CB
:10BBE800938B1B00A38FCBFEE39CDBFEB3876B41DB
:10BBF8002320F1026FE00F8523244103232801004D
:10BC0800130A0900B707008033C367009307D002FF
:10BC1800232CF1046FF01FC78327010593860B00BF
:10BC2800232EF10C8327410203C6FBFF83C5F700CF
:10BC38006310B60213050003A38FA6FE8326C10D69
:10BC48009387F6FF232EF10C03C6F6FFE386C5FEA5
:10BC5800930516001305900393F5F50F6306A600E8
:10BC6800A38FB6FE6FF09FF88327410283C5A70014
:10BC7800A38FB6FE6FF09FF793851D0013050D0087
:10BC880023281101EFB0DFB283280101130B05004F
:10BC98006308053E2328A1006FF09FBC93070003AB
:10BCA8002304F10C930780076FF0DFB99307700442
:10BCB8003309BB01232AF104930C010A6FD05FF208
:10BCC80003278100B38797009386160023A0E80016
:10BCD80023A298002326F10E2324D10E1306700008
:10BCE8006358D6B61306410E93050C0013050D00D4
:10BCF800EF20D059630405006FE01F9C8327C10E15
:10BD08008326810E9308C1106FF0CFB4930B0A00FD
:10BD18006FE0CFDF63940D00930D10000323C10F74
:10BD2800032E010F832E410F032F810F13690A1071
:10BD3800E34403EC930A010B1308C10D9307010DAB
:10BD48001307C10C93860D001306200093850A0083
:10BD580013050D00232211052328C10B2320C1053B
:10BD6800232AD10B2322D103232CE10B2320E10327
:10BD7800232E610A232E6100EFA04FD30323C101B4
:10BD880023244103032F0102832E4102032E0104C1
:10BD980083284104130B0500130A09002328010016
:10BDA800232C01046FF01F979307F0FF2326F1005F
:10BDB8006FD05FC09306610D6318060093060003F9
:10BDC800230BD10C9306710D1307011B93870703EF
:10BDD8003386E6402380F6009307D60D232CF10224
:10BDE8006FD05FF6930A010B13850A00232811050B
:10BDF8002328C10B232AD10B232CE10B232E610A04
:10BE0800EF80006D1306C10CEFD08FB613860500C6
:10BE18009305050013850A00EF80404C8327010B2A
:10BE2800930C010A130901092328F1088327410B00
:10BE38001306010893050900232AF1088327810BBB
:10BE480013850C002320C104232CF1088327C10B80
:10BE58002320010823220108232EF108B707FC3FFD
:10BE68002326F10823240108EF50D04E0328010AA5
:10BE7800032E410A832E810A032FC10A93850C00E1
:10BE880013850A002328010B23220105232AC10B4D
:10BE98002322C103232CD10B2320D103232EE10B12
:10BEA800232EE1012320010A2322010A2324010A67
:10BEB8002326010AEF50D014032FC101832E01025B
:10BEC800032E410203284104832801056316050057
:10BED800930710002326F10CB7570180938747AFCB
:10BEE8002322F1026FF05FAB23280100138A0700B9
:10BEF8006FF05FD1930470060326C1039306F00F19
:10BF0800834706006388D7180327C101130500007B
:10BF18009305000063DEE7003307F7408347160008
:10BF2800638407049385150013061600E394D7FE6F
:10BF3800232EC102232EE1002322B1022324A102D1
:10BF48000327810283274102B387E700032781047F
:10BF5800B387E702B38C970193CAFCFF93DAFA41DF
:10BF6800B3FA5C016FD05FE2834706001305150042
:10BF78006FF0DFFB8327C10293046006B30CF70060
:10BF8800B38CBC016FF01F858327810293F71700DC
:10BF9800639407006FD01FDD6FD05FDC930C010A3C
:10BFA80093850C0013850A00232211052328C10B51
:10BFB8002320C105232AD10B2322D103232CE10BF3
:10BFC8002320E103232E610A232E61002320010A86
:10BFD8002322010A2324010A2326010AEF505002D2
:10BFE8000323C101032F0102832E4102032E010402
:10BFF80083284104630205EA93071000B387B74119
:10C008002326F10C3309F9006FD09FBD639A07000E
:10C01800930A100093046006930C10006FF08FDBF6
:10C028008327C10293046006938C1700B38CBC016C
:10C0380093CAFCFF93DAFA41B3FA5C016FF08FD927
:10C04800138708006FF0CFA78327410183AD07004E
:10C058009387470063D40D00930DF0FF83441400C9
:10C06800232AF100130407006FD04FF99307C0008B
:10C078002320FD009307F0FF2326F1006FD09F9344
:10C088000357CC0093670704138707002316FC00A7
:10C098006FD09F9123240102232201026FF05FEAEF
:10C0A80093072000232CF1026FD0DFC983A7450630
:10C0B800130101FD23286101232611022324810293
:10C0C8002322910223202103232E3101232C410115
:10C0D800232A510123267101232481011397270163
:10C0E800130B06006358070A83278600832B060074
:10C0F8001389050093090500930AF0FF6388070870
:10C1080003AC4B0003A40B00135A2C0063060A0669
:10C11800930400006F00C00013044400630C9A04E9
:10C12800832504001306090013850900EF10D004C5
:10C1380093841400E31255FF1305F0FF8320C10216
:10C148000324810223240B0023220B0083244102B1
:10C15800032901028329C101032A8101832A41019C
:10C16800032B0101832BC100032C81001301010360
:10C178006780000083278B00137CCCFFB38787413F
:10C188002324FB00938B8B00E39C07F61305000028
:10C198006FF0DFFAEF10100F6FF05FFA03278600D9
:10C1A800630407006FF09FF02322060013050000C8
:10C1B80067800000130101ED232E3111232C41115A
:10C1C800232671112326111223248112232291126E
:10C1D80023202113232A511123286111232481119B
:10C1E800232291112320A111232EB10F2328D1003E
:10C1F800130A050093890500930B060063060500E2
:10C2080083278503638E075E0397C9009317070189
:10C218009316270193D7070163CA0602B7270000C0
:10C2280083A64906B367F7009397070137E7FFFF2F
:10C2380093D707411307F7FF33F7E6002396F90072
:10C248009397070123A2E90693D7070113F78700FD
:10C258006300074003A70901630C073E93F7A70192
:10C268001307A0006386E740B75701809387C72468
:10C27800375B01809304C104232AF10037590180F8
:10C2880093078B3B138C0B00232091042324010478
:10C2980023220104232C0100232E01002322010262
:10C2A80023200102232601002324F1001309893CDD
:10C2B800938B040083470C006388072613040C0043
:10C2C80013075002638EE7428347140013041400D7
:10C2D800E39A07FEB30C844163088425032781048D
:10C2E8008327410423A08B013387EC009387170031
:10C2F80023A29B012324E1042322F1049306700066
:10C30800938B8B0063D0F602E30A073A1306010405
:10C318009385090013050A00EFF05FD9631A052019
:10C32800938B04000327C100834704003307970158
:10C338002326E100638A071E03471400130C140028
:10C34800A30D0102930AF0FF23220100130B000042
:10C35800930CA005130D90001306A002130C1C00EB
:10C36800930707FE63E8FC0483264101939727009F
:10C37800B387D70083A7070067800700232201003F
:10C38800930707FD8325410003470C00130C1C008D
:10C3980093962500B386B60093961600B387D70008
:10C3A8002322F100930707FDE37EFDFC930707FEB8
:10C3B800E3FCFCFA630A07162306E108A30D010251
:10C3C800930C1000130D10001304C108930A000009
:10C3D800937F2B0063840F00938C2C000327410468
:10C3E800137F4B08832781049306170013860600E2
:10C3F80063180F0083254100B38D9541E342B009CE
:10C408008345B10393868B00638C05021307B10340
:10C418009387170023A0EB001307100023A2EB005B
:10C428002324F1042322C104130770006340C77E4C
:10C4380013070600938B06001306160093868600E2
:10C44800638E0F041307C1039387270023A0EB0013
:10C458001307200023A2EB002324F1042322C104A4
:10C4680013077000E350C700E384072A130601048A
:10C478009385090013050A002324E103EFF01FC385
:10C488006318050A0327410483278104032F8102C7
:10C498009306410513061700938B040093050008C3
:10C4A8006306BF5AB38AAA4163425069B307FD00C5
:10C4B80023A08B0023A2AB012324F1042322C1046F
:10C4C800130770006352C702E38E070A13060104BC
:10C4D8009385090013050A00EFF05FBD631A050490
:10C4E800832781049386040013734B0063080300B9
:10C4F80003274100B30B9741E344700B0324410029
:10C508006354940113840C000327C1003307870088
:10C518002326E1006398076C83470C00232201045B
:10C52800938B0400E39C07D883278104E39A07646C
:10C5380083D7C90093F70704E39207688320C112E1
:10C54800032481120325C100832441120329011207
:10C558008329C111032A8111832A4111032B011157
:10C56800832BC110032C8110832C4110032D011043
:10C57800832DC10F130101136780000013050A0002
:10C58800EFB00F8383274500138507002320F102AE
:10C59800EFC05FFD9307050013050A001384070029
:10C5A8002322F102EFB0CF80832785001306A00273
:10C5B800232EF100E318042A03470C006FF01FDA5A
:10C5C80003470C00136B0B026FF05FD9136B0B0161
:10C5D80093770B02638407168327010193877700FB
:10C5E80093F787FF03A7470003AD070093878700EA
:10C5F8002328F100930C0700634A07161307F0FF7E
:10C60800930D0B006388EA0033679D01937DFBF768
:10C61800E30C070AE3960C1613079000E362A717CA
:10C6280093070D03A307F10E138B0D00130D1000D4
:10C638001304F10E938C0A0063D4AA01930C0D0025
:10C648008347B103B337F000B38CFC006FF05FD8B9
:10C658009385090013050A00EF708FD0E310055683
:10C6680083D7C9001307A00093F7A701E39EE7BE8D
:10C678008397E900E3CA07BE8326010113860B00EE
:10C688009385090013050A00EF0090582326A1009E
:10C698006FF0DFEA136B0B0193770B02638A0706CF
:10C6A800832701019387770093F787FF03AD07007E
:10C6B80083AC4700938787002328F100937DFBBF55
:10C6C80013070000A30D01029306F0FF6384DA0C40
:10C6D800B3669D0113FBFDF76390065A639C0A300D
:10C6E8006318077E13FD1D001304010FE3040DF406
:10C6F80093070003A307F10E1304F10E6FF09FF3E5
:10C70800B30C8441E31C84BD834704006FF09FC2CF
:10C718008326010193770B0113874600E39C0716D4
:10C7280093770B04E388073883270101930C0000F3
:10C738002328E10003DD07006FF05FF8832601017D
:10C7480093770B0113874600E394071093770B0444
:10C75800E3820732832701012328E100039D0700B4
:10C76800935CFD4113870C00E35A07E83337A001B7
:10C77800B30E9041B38CEE401307D002A30DE10233
:10C788009306F0FF330DA041930D0B001307100023
:10C79800E390DAF493061000E30ED7E69306200040
:10C7A8006304D7261304010F9397DC0113777D00E8
:10C7B800135D3D001307070333EDA70193DC3C002D
:10C7C800A30FE4FEB3679D01130604001304F4FFEE
:10C7D800E39C07FC93F71D00638207269307000379
:10C7E800630EF7241306E6FFA30FF4FE9307010F69
:10C7F800338DC740138B0D00130406006FF09FE3C1
:10C80800EF70DFC66FF05FA083270101A30D01025F
:10C8180003A40700938D4700E30004229307F0FF69
:10C82800E388FA1213860A00930500001305040032
:10C83800EFB08FF1E3000536330D85402328B101B1
:10C84800930A00006FF01FDF03270101A30D010207
:10C85800930C100083270700130747002328E100E3
:10C868002306F108130D10001304C1086FF01FB65A
:10C87800832701013787FFFF1347078303AD0700AD
:10C88800938747002328F100B7570180938747AF64
:10C89800231EE102930C0000936D2B00232CF10062
:10C8A800130720006FF01FE203470C009307C00630
:10C8B800E306F716136B0B016FF05FAA03470C0032
:10C8C80093078006E304F714136B0B046FF01FA99A
:10C8D800936D0B0193F70D026384076083270101B1
:10C8E800130710009387770093F787FF03AD0700BE
:10C8F80083AC4700938787002328F1006FF09FDC03
:10C9080003470C00136B0B086FF05FA5832601012A
:10C9180003470C0083A70600938646002328D1000E
:10C928002322F100E3DC07A2B307F0402322F10041
:10C93800136B4B006FF09FA203470C00136B1B0097
:10C948006FF0DFA18347B10303470C00E39807A00A
:10C9580093070002A30DF1026FF05FA003470C00DC
:10C96800136B4B006FF09F9F9307B00203470C00B7
:10C97800A30DF1026FF09F9E03470C0093061C0065
:10C98800E30AC724930707FD138C0600930A0000E7
:10C99800E368FD9C03470C0093962A00B38A56016E
:10C9A800939A1A00B38AFA00930707FD130C1C0028
:10C9B800E372FDFE6FF0DF9A8326010193770B0285
:10C9C80003A70600938646002328D100639A076AC6
:10C9D80093770B01E39C070493770B04E390071408
:10C9E80013730B20E30403048327C1002300F7001B
:10C9F8006FF05F8C93061000E30ED71A93062000A1
:10CA0800930D0B00E310D7DA832681011304010F7D
:10CA18009377FD00B387F60003C70700135D4D0049
:10CA28009397CC0133EDA70193DC4C00A30FE4FEF0
:10CA3800B3679D011304F4FFE39C07FC9307010F00
:10CA4800338D8740138B0D006FF0DFBE83254100C7
:10CA5800B38D9541E358B0A593050001E3D6B5170A
:10CA6800930E0001130F70006F008001130627005A
:10CA7800938B8B0013870600938D0DFF63DCBE0537
:10CA8800938707019306170023A02B0123A2DB013C
:10CA98002324F1042322D104E35ADFFC6380071620
:10CAA800130601049385090013050A00EFF00FE04F
:10CAB800E31005A803274104930E0001938D0DFF91
:10CAC80083278104938B040013061700130F70004B
:10CAD800E3C8BEFB9305060013858B00B387B70137
:10CAE80023A02B0123A2BB012324F1042322B10498
:10CAF80013077000635AB7526386077E1306010452
:10CB08009385090013050A00EFF04FDAE31205A236
:10CB180003274104B38AAA41832781049306410568
:10CB280013061700938B0400E352509993050001F4
:10CB380063D0557B93080001930D70006F0080014E
:10CB480013062700938B8B0013870600938A0AFF2E
:10CB580063DA5805938707019306170023A02B0172
:10CB680023A21B012324F1042322D104E3DADDFCF0
:10CB780063820706130601049385090013050A005A
:10CB8800EFF0CFD2E316059A03274104930800017A
:10CB9800938A0AFF83278104938B040013061700E6
:10CBA800E3CA58FB93858B00B387570123A02B0159
:10CBB80023A25B012324F1042322C104130770007C
:10CBC8006346C72C1306160093868500938B0500D1
:10CBD8006FF0DF8D1306100013070000938B04001D
:10CBE8006FF0DFF6130601049385090013050A00A8
:10CBF800EFF0CFCBE30205926FF09F93130610007E
:10CC080013070000938B04006FF01FE7638C073055
:10CC1800130601049385090013050A002326E1037E
:10CC28002324F103EFF08FC8E31405900327410490
:10CC380083278104032FC102832F810293064105B4
:10CC480013061700938B04006FF08FFF9307C1033F
:10CC58002326F104930720002328F104130610006B
:10CC68009306410513070600938B06001306170069
:10CC780093868B006FF09F82930D0B006FF09FB12E
:10CC8800130600016350B67313860B00930E000160
:10CC9800930B040093027000138409002324F1030A
:10CCA80093890D00930D0C00138C0A00930A0F0052
:10CCB8006F00C001130527001306860013870600BE
:10CCC800938909FF63DE3E059306170083258100DB
:10CCD800938707012322D6012320B6002324F104D9
:10CCE8002322D104E3D8D2FC638607081306010483
:10CCF8009305040013050A00EFF04FBB6316054CBB
:10CD080003274104930E0001938909FF83278104B7
:10CD1800138604001305170093027000E3C63EFB58
:10CD2800832F8102138F0A0093050500930A0C00D4
:10CD3800138C0D00938D09009309040013840B00D4
:10CD4800930B060003278100B387B70123A2BB0119
:10CD580023A0EB002324F1042322B104130770005D
:10CD68006342B71E938B8B0013861500138705004B
:10CD78006FF00FE913070000130510001386040075
:10CD88006FF01FF42322010413734B006302030E98
:10CD980003274100B30B9741635C700D9386040031
:10CDA800130700010326410463527761130D000144
:10CDB800930D70006F00800113052600938686008E
:10CDC80013060700938B0BFF635A7D0583258100AB
:10CDD800938707011307160023A0B60023A2A60114
:10CDE8002324F1042322E104E3D8EDFC638A070637
:10CDF800130601049385090013050A00EFF00FAB31
:10CE0800631805F203264104938B0BFF83278104E3
:10CE18009386040013051600E34A7DFB930505007D
:10CE280003278100B387770123A2760123A0E600B8
:10CE38002324F1042322B104130770006350B7ECD4
:10CE480063880702130601049385090013050A0085
:10CE5800EFF0CFA5631E05EC832781046FF00FEA7E
:10CE68001305100013060000938604006FF09FF569
:10CE7800032441006354940113840C008327C100E8
:10CE8800B38787002326F1006FF00FE96382073428
:10CE9800130601049385090013050A00EFF00FA19A
:10CEA800631805E803264104832781049306410596
:10CEB80013061600938B04006FF04FDF2322010442
:10CEC800938B04006FF00FC6639C0AF4138B0D005C
:10CED800930A0000130D00001304010F6FF08FF583
:10CEE8008326010193F70D01138746006398071401
:10CEF80093F70D046380073A83270101930C000020
:10CF08002328E10003DD0700130710006FF08FFBF3
:10CF1800930641051306100013070000938B0400C5
:10CF28006FF0CFD763800F189307C1032326F1044E
:10CF3800930720002328F10413071000930B4105E1
:10CF48006FF0DFD26382072213060104938509007C
:10CF580013050A002326E1032324F103EFF00F95BC
:10CF6800631805DC0327410483278104032FC102CA
:10CF7800832F8102938B0400130617006FF04FC8AC
:10CF880093F70D402324410323263103138A0C0011
:10CF980093090D00130B0000032DC1011304010FA9
:10CFA800938C07006F0040021306A0009306000050
:10CFB8001385090093050A00EF300036630E0A3026
:10CFC80093090500138A05001306A00093060000C4
:10CFD8001385090093050A00EF3040771305050310
:10CFE800A30FA4FE130B1B001304F4FFE38E0CFA2B
:10CFF80083460D00E39A66FB9307F00FE306FBFAFE
:10D0080063140A189307900063E037199307010F18
:10D01800232EA101032A81028329C102338D87406F
:10D02800138B0D006FF00FE1138615009306850032
:10D0380013870500930B05006FF0CFC62328E10086
:10D0480003AD0600930C0000130710006FF08FE784
:10D0580003AD06002328E100935CFD4113870C0013
:10D068006FF08FD98327C10103470C00638807AE8F
:10D0780083C70700638407AE136B0B406FF00FAED6
:10D088008326C10093D7F6412320D7002322F70037
:10D098006FF04FA203AD0600930C00002328E100B7
:10D0A8006FF0CFE113070000930641051306100047
:10D0B800938B04006FF08FBE930D0B006FF09F8170
:10D0C800B7570180938787B0232CF10093770B0221
:10D0D80063800706832701019387770093F787FF0B
:10D0E80003AD070083AC4700938787002328F1002E
:10D0F80093761B00638E0600B3669D01638A060063
:10D1080093060003230ED102A30EE102136B2B003A
:10D11800937DFBBF130720006FF0CFDAB75701806C
:10D12800938747AF232CF10093770B02E39407FA18
:10D138000326010193770B0193064600638A070AC9
:10D14800032D0600930C00002328D1006FF05FFA2E
:10D1580013050400EFC00FC1130D05002328B1010A
:10D16800930A00006FF00FCD0347B103631A071845
:10D17800E39E0FAC13070000130610009306410549
:10D18800938B04006FF08FB183274102832501023E
:10D19800130B00003304F440138607001305040042
:10D1A800EFC00FC583451D001306A00093060000BD
:10D1B8003337B0001385090093050A00330DED00DD
:10D1C800EF3080156FF0DFDF930904006FF04FB682
:10D1D8001307100093070D00232681042328A105B7
:10D1E8002324A1052322E104930641056FF0CFAF64
:10D1F80093770B046382070683270101930C0000D1
:10D208002328D10003DD07006FF09FEE03471C00C1
:10D21800136B0B20130C1C006FF04F9403471C007A
:10D22800136B0B02130C1C006FF04F938327C10084
:10D238002320F7006FF00F8893076000138D0A0012
:10D2480063EC570B375E0180930C0D002328B10166
:10D258001304CEB16FF08F9793770B206388071074
:10D2680083270101930C00002328D10003CD070078
:10D278006FF01FE893770B20638E070C832701015B
:10D288002328E100038D0700935CFD4113870C0000
:10D298006FF08FB693F70D206382070A8327010189
:10D2A800930C00002328E10003CD070013071000AA
:10D2B8006FF04FC193770B2063880706832701011E
:10D2C800930C00002328E10003CD07006FF00FBF87
:10D2D800938506006FF05F8D93079000E3E237CFE8
:10D2E8006FF0DFD293064105130610001307000004
:10D2F800938B04006FF00F9B130D60006FF09FF489
:10D308009307B1032326F104930710002328F1049F
:10D3180013061000930641056FF08F918327C10013
:10D328002310F7006FE01FF983270101930C000019
:10D338002328E10003AD07006FF04FB883270101F0
:10D34800930C00002328E10003AD07001307100029
:10D358006FF04FB7832701012328E10003AD0700D1
:10D36800935CFD4113870C006FF00FA9832701011F
:10D37800930C00002328D10003AD07006FF05FD79E
:10D38800130601049385090013050A00EFE01FD274
:10D398006FF00F9A138D0A002328B101930A000039
:10D3A8006FF04FA9938506006FF0DF99930516007B
:10D3B8006FF01FA7930D0B006FF08FA69307F0FF78
:10D3C8002326F1006FF08F9713850600930506005A
:10D3D8006FF0CFF08327010183AA070093874700E6
:10D3E80063D40A00930AF0FF03471C002328F100C6
:10D3F800138C06006FE09FF69307050003A5C1256F
:10D408009306060013860500938507006FE09FDAF0
:10D4180083D7C50003AE450603D3E50083A8C5013D
:10D4280003A84502130101B893F7D7FF130700407B
:10D43800232C8146231AF100138405009307010762
:10D4480093058100232A914623282147232E11463C
:10D45800130905002326C107231B6100232211039A
:10D46800232601032324F100232CF1002328E100C3
:10D47800232EE10023200102EFE0DFD3930405000F
:10D48800635C05028357410193F70704638807002B
:10D498008357C40093E707042316F4008320C14789
:10D4A8000324814703290147138504008324414746
:10D4B80013010148678000009305810013050900E6
:10D4C800EF601FC1E30005FC9304F0FF6FF09FFBC2
:10D4D800130101FF138705002324810023229100F3
:10D4E80093050600130405001386060013050700BC
:10D4F8002326110023AE0130EF205FFF9307F0FFD2
:10D50800630CF5008320C1000324810083244100BB
:10D51800130101016780000083A7C131E38407FE7E
:10D528008320C1002320F4000324810083244100C8
:10D53800130101016780000003A7C125130101FF42
:10D548009387060013080600232611008328C700C6
:10D558009306050013870500138607006300080279
:10D56800B75701809387873DB75501809385853EDE
:10D5780013850800EF00C028EF20D0253758018018
:10D58800930788A6130888A66FF01FFE130101FFF2
:10D59800930606001306000023261100EFF0DFF9BA
:10D5A800B385C502130101FF23248100232611003E
:10D5B800EFA00FA013040500630805020326C5FFAA
:10D5C800130740021376C6FF1306C6FF6360C7063B
:10D5D800930630019307050063E2C60223A0070003
:10D5E80023A2070023A407008320C1001305040019
:10D5F8000324810013010101678000002320050036
:10D60800232205009307B00163F0C7042324050013
:10D618002326050093070501E312E6FC23280500ED
:10D6280093078501232A05006FF05FFB930500002F
:10D63800EF301F868320C1001305040003248100F6
:10D648001301010167800000930785006FF01FF93F
:10D65800130101FF232481002322910013040500F4
:10D66800138505002326110023AE0130EF205FE566
:10D678009307F0FF630CF5008320C10003248100A9
:10D6880083244100130101016780000083A7C13191
:10D69800E38407FE8320C1002320F40003248100D3
:10D6A800832441001301010167800000130101FF79
:10D6B8002326110023248100232291002320210105
:10D6C80063800502138405009304050063060500C2
:10D6D80083278503638C070A8317C40063920702B4
:10D6E8008320C10003248100130900008324410022
:10D6F80013050900032901001301010167800000D7
:10D708009305040013850400EF60CFF68327C40255
:10D7180013090500638A07008325C40113850400E3
:10D72800E7800700634C05068357C40093F7070892
:10D73800639E070683250403638C0500930704048E
:10D748006386F50013850400EF605FE9232804026F
:10D75800832544046388050013850400EF601FE8EF
:10D7680023220404EF609FD123160400EF605FD1E9
:10D778008320C1000324810083244100130509008C
:10D78800032901001301010167800000EF601FCE2B
:10D798008317C400E38607F46FF09FF68357C4002D
:10D7A8001309F0FF93F70708E38607F883250401B8
:10D7B80013850400EF609FE26FF0DFF79305050023
:10D7C80003A5C1256FF09FEE130101FC1303C102ED
:10D7D8002326D10293060300232E11002328E102F9
:10D7E800232AF102232C0103232E1103232661008F
:10D7F800EFE05F9C8320C1011301010467800000F2
:10D80800130E0500130101FC03A5C12513038102B2
:10D818002324C1022326D1021386050093060300A0
:10D8280093050E00232E11002328E102232AF1027A
:10D83800232C0103232E110323266100EFE09F9779
:10D848008320C1011301010467800000130101FD59
:10D8580023248102232E310123286101232611026A
:10D868002322910223202103232C4101232A510141
:10D87800130B05009389050013040600EF00807858
:10D88800930710006310F5029387F9FF1307E00F61
:10D89800636AF70013F7F90F2306E1001309100074
:10D8A8006F00C0029306C405138609009305C100E2
:10D8B80013050B00EF20805E9307F0FF13090500A6
:10D8C8006304F50A630E05080347C10093040000CA
:10D8D800130AF0FF930AA0006F0080028327040058
:10D8E800938617002320D4002380E7009384140034
:10D8F8009307C100B387970063F4240703C70700A1
:10D90800832784009387F7FF2324F400E3D807FCD8
:10D9180083268401930507001306040013050B00F2
:10D9280063C4D700E31C57FBEF20C03DE31045FD5F
:10D938001309F0FF8320C1020324810283244102DA
:10D948008329C101032A8101832A4101032B010193
:10D958001305090003290102130101036780000070
:10D96800138909006FF01FFD8357C40093E707046C
:10D978002316F4006FF01FFC8317C60013972701C6
:10D988006340070203274606B7260000B3E7D7001F
:10D99800B72600003367D7002316F6002322E606D1
:10D9A8006FF0DFEA130101FE232C810003A4C125D7
:10D9B800232E110013860500930505006306040055
:10D9C80083278403638007048317C60013972701FE
:10D9D8006340070203274606B7260000B3E7D700CF
:10D9E800B72600003367D7002316F6002322E60681
:10D9F80013050400032481018320C10113010102DE
:10DA08006FF0DFE42324A100130504002326C100DE
:10DA1800EF60DFA50326C100832581006FF0DFFAE0
:10DA2800130101FF1387050023248100232291009D
:10DA380013040500930506001305070023261100AB
:10DA480023AE0130EF201FA89307F0FF630CF50009
:10DA58008320C100032481008324410013010101B4
:10DA68006780000083A7C131E38407FE8320C100DB
:10DA78002320F400032481008324410013010101C1
:10DA88006780000083278600638E073283D7C5002E
:10DA9800130101FD23248102232C4101232A510172
:10DAA800232611022322910223202103232E310150
:10DAB8002328610123267101232481012322910156
:10DAC8002320A10113F78700130A0600930A050013
:10DAD800138405006306070803A705016302070806
:10DAE80013F7270083240A00630C070883274402DE
:10DAF8008325C401370B0080930900001309000037
:10DB0800134B0BC01386090013850A00630209042E
:10DB18009306090063742B0193060B00E780070046
:10DB28006358A02883278A00B389A9003309A9402C
:10DB38003385A7402324AA00630A052083274402CB
:10DB48008325C4011386090013850A00E31209FC22
:10DB580083A9040003A94400938484006FF09FFA0A
:10DB68009305040013850A00EF509FFF631C053AD4
:10DB78008357C40083240A0013F72700E31807F625
:10DB880013F7170063140724832C8400032504006B
:10DB9800370B0080934BEBFF130C000013090000B8
:10DBA800134BFBFF630E090E13F70720630C0724C2
:10DBB800138D0C006362992F13F70748630A07084F
:10DBC800832944018325040113071900939619003A
:10DBD800B386360193D9F601330DB540B389D90020
:10DBE80093D919403307A7011386090063F6E900A2
:10DBF800930907001306070093F707406384072E6D
:10DC08009305060013850A00EF909FBA930C050050
:10DC1800630205308325040113060D00EF00C04D93
:10DC28008357C40093F7F7B793E707082316F40060
:10DC38003385AC01B387A941232894012320A4008C
:10DC4800232A3401930C09002324F400130D09003E
:10DC580013060D0093050C00EF00C05B032784003A
:10DC68008327040093090900B30C9741B387A701E0
:10DC7800232494012320F4001309000003268A00BA
:10DC8800330C3C01B309364123243A016380090C63
:10DC9800832C8400032504008357C400E31609F08D
:10DCA80003AC040003A94400938484006FF09FEF41
:10DCB80083A9440003AC040093848400E38A09FE2A
:10DCC800138609009305A00013050C00EFA0CFA749
:10DCD8006304051213051500330B854193070B00E8
:10DCE800938B090063F43701938B07000325040025
:10DCF800832704018326440163F8A70003298400CD
:10DD0800338926016342790963C8DB1A83274402F1
:10DD18008325C40113060C0013850A00E780070059
:10DD2800130905006356A008330B2B411305100097
:10DD3800630A0B1603268A00330C2C01B389294188
:10DD48003309264123242A01631A09081305000010
:10DD58008320C10203248102832441020329010292
:10DD68008329C101032A8101832A4101032B01016F
:10DD7800832BC100032C8100832C4100032D01005B
:10DD8800130101036780000093050C0013060900C6
:10DD9800EF004048832704009305040013850A0018
:10DDA800B38727012320F400EF608FB2E30E05F656
:10DDB8008317C40093E707042316F4001305F0FF44
:10DDC8006FF01FF91305000067800000130B0000B7
:10DDD80013050000130C000093090000E38A09EC06
:10DDE800E31E05EE138609009305A00013050C0039
:10DDF800EFA08F95E31005EE93871900138B0700AA
:10DE08006FF01FEE8327040163E2A7048327440110
:10DE1800636EF9029306090063F42B0193060B0065
:10DE2800B3C6F602032744028325C40113060C0077
:10DE380013850A00B386F602E70007009309050078
:10DE4800E358A0F6330939416FF05FE393890C007A
:10DE580063749901930909001386090093050C005E
:10DE6800EF00403B8327840003270400B387374132
:10DE7800330737012324F4002320E400E39407FC4C
:10DE88009305040013850A00EF608FA4E31205F2DE
:10DE9800330939416FF09FDE930C0900130D090017
:10DEA8006FF01FDB9305040013850A00EF604FA293
:10DEB800E30205E86FF0DFEF13860B0093050C0013
:10DEC800EF004035832784000326040013890B00E4
:10DED800B3877741330676012324F4002320C40056
:10DEE8006FF09FE413850A00EF00404B930C050088
:10DEF800E31005D48325040113850A00EF600FEEB3
:10DF08008317C4001307C00023A0EA0093F7F7F7AC
:10DF18006FF05FEA1307C0008317C40023A0EA006C
:10DF28006FF05FE91305F0FF6FF09FE2130101FF47
:10DF38002324810023229100130405001385050082
:10DF48002326110023AE0130EF20CFD89307F0FF2E
:10DF5800630CF5008320C100032481008324410061
:10DF6800130101016780000083A7C131E38407FE24
:10DF78008320C1002320F40003248100832441006E
:10DF88001301010167800000130101FF232611001E
:10DF98002324810023229100630C0602B7550180D7
:10DFA8009385C5411305060013040600EF005016BB
:10DFB800B754018063120502138584418320C10090
:10DFC80003248100832441001301010167800000BC
:10DFD800B75401806FF05FFE9385844113050400F8
:10DFE800EF001013E30A05FCB7550180938585A659
:10DFF80013050400EF00D011E30005FC1305000031
:10E008006FF0DFFB03C5011F678000009307050061
:10E0180003A5C12513860500938507006FF0DFF679
:10E02800130101FF13870500232481002322910097
:10E038009305060013040500138606001305070060
:10E048002326110023AE0130EF204FC99307F0FFBC
:10E05800630CF5008320C100032481008324410060
:10E06800130101016780000083A7C131E38407FE23
:10E078008320C1002320F40003248100832441006D
:10E08800130101016780000003A3C11A67000300A0
:10E09800638005026302060463880604834706005A
:10E0A80023A0F500034506003335A0006780000073
:10E0B800130101FF9305C10063040602638A060287
:10E0C8008347060023A0F500034506003335A0006A
:10E0D800130101016780000013050000678000003C
:10E0E800130500006FF0DFFE1305E0FF67800000F6
:10E0F8001305E0FF6FF0DFFDB3C7A50093F7370006
:10E10800B308C500639207069307300063FEC7048F
:10E1180093773500130705006398070613F6C8FFC1
:10E12800930706FE636CF708637CC70293860500B5
:10E138009307070003A806009387470093864600C5
:10E1480023AE07FFE3E8C7FE9307F6FFB387E74070
:10E1580093F7C7FF938747003307F700B385F500A8
:10E16800636817016780000013070500E37C15FF4B
:10E1780083C705001307170093851500A30FF7FE43
:10E18800E36817FF6780000083C6050013071700C0
:10E1980093773700A30FD7FE93851500E38007F820
:10E1A80083C605001307170093773700A30FD7FE20
:10E1B80093851500E39A07FC6FF05FF683A6450088
:10E1C80083A2050083AF850003AFC50083AE0501B8
:10E1D80003AE450103A3850103A8C5012322D70087
:10E1E80083A60502232057002324F7012326E701ED
:10E1F8002328D701232AC701232C6700232E0701D0
:10E208002320D7021307470293854502E368F7FAEC
:10E218006FF09FF163F6A502B387C5006372F5023C
:10E228003307C500630A060E83C6F7FF9387F7FF17
:10E238001307F7FF2300D700E398F5FE6780000077
:10E248009307F00063E8C702930705009306F6FFFB
:10E25800630C060C93861600B386D70003C7050027
:10E268009387170093851500A38FE7FEE398D7FEE1
:10E2780067800000B3E7A50093F737006390070AAB
:10E28800930806FF93F808FF9388080133081501DF
:10E298001387050093070500832607001307070166
:10E2A8009387070123A8D7FE832647FF23AAD7FE13
:10E2B800832687FF23ACD7FE8326C7FF23AED7FE6E
:10E2C800E31CF8FC1377C600B38515011378F60034
:10E2D800630E07041387050093880700130E3000A8
:10E2E8000323070013074700B306E84023A068008C
:10E2F800B386D50093884800E364DEFE1307C8FFA1
:10E308001377C7FF1307470013763600B387E70074
:10E31800B385E5006FF09FF3678000009306F6FF72
:10E32800930705006FF01FF36780000013060800CD
:10E338006FF0DFF1130101FF13870500232481002B
:10E348002322910093050600130405001386060096
:10E35800130507002326110023AE0130EF208F9804
:10E368009307F0FF630CF5008320C10003248100AC
:10E3780083244100130101016780000083A7C13194
:10E38800E38407FE8320C1002320F40003248100D6
:10E39800832441001301010167800000130101FD7E
:10E3A8002320210323261102232481022322910200
:10E3B800232E3101232C4101232A510123286101F5
:10E3C8002326710123248101130906006382052293
:10E3D8001384050093090500EF905FC49304B90006
:10E3E8009307600163FC970E93F484FF138704007E
:10E3F80063CC040E63EA240F8327C4FF930A84FFC7
:10E4080013FAC7FF338B4A01635AEA18938B01CC7E
:10E4180003A68B0083264B00630E662313F6E6FFE4
:10E428003306CB0003264600137616006314061A3B
:10E4380093F6C6FF3306DA00635EE63293F71700F9
:10E4480063940702032C84FF338C8A4183274C0092
:10E4580093F7C7FFB386D700B38B460163DAEB3473
:10E46800B30BFA0063D2EB0C93050900138509007E
:10E47800EF900FB413090500630C05048327C4FF4C
:10E48800130785FF93F7E7FFB387FA006382E73046
:10E498001306CAFF9307400263E6C730130730012B
:10E4A80083260400636CC72693070500130704003E
:10E4B80023A0D7008326470023A2D700032787007D
:10E4C80023A4E7009305040013850900EF600F916A
:10E4D80013850900EF90DFB46F00C00193040001B9
:10E4E80013070001E3FA24F19307C00023A0F90001
:10E4F800130900008320C1020324810283244102FE
:10E508008329C101032A8101832A4101032B0101C7
:10E51800832BC100032C8100130509000329010284
:10E5280013010103678000008327CC0003278C00B8
:10E538001306CAFF930640022326F70023A4E70028
:10E5480013098C00330B7C0163E4C62E930530015C
:10E55800032704009307090063F2C5022324EC0093
:10E56800032744009307B0012326EC0063E2C73079
:10E578000327840093070C011304840023A0E700F9
:10E5880003274400138A0B00930A0C0023A2E70018
:10E59800032784001304090023A4E70083A74A0083
:10E5A80033079A409306F00093F7170063ECE606EA
:10E5B800B367FA0023A2FA0083274B0093E71700FA
:10E5C8002322FB0013850900EF909FA5130904007F
:10E5D8006FF05FF293F71700E39807E8032C84FFC6
:10E5E800338C8A4183274C0093F7C7FF6FF05FE7AE
:10E5F800032481028320C1028324410203290102EA
:10E608008329C101032A8101832A4101032B0101C6
:10E61800832BC100032C810093050600130101031D
:10E628006F900F99B3E7970023A2FA00B3859A0079
:10E638001367170023A2E50083274B009385850005
:10E648001385090093E717002322FB00EF501FF9F9
:10E658006FF05FF793F6C6FF3306DA00938504017F
:10E668006350B60E93F71700E39007E0032C84FF7E
:10E67800338C8A4183274C0093F7C7FFB386D700B2
:10E68800338B4601E34EBBDC8327CC0003278C0089
:10E698001306CAFF930640022326F70023A4E700C7
:10E6A80013098C0063EEC62093053001032704008C
:10E6B8009307090063F2C5022324EC0003274400F2
:10E6C8009307B0012326EC0063E4C72003278400E6
:10E6D80093070C011304840023A0E70003274400D8
:10E6E80023A2E7000327840023A4E70033079C0044
:10E6F800B3079B4023A4EB0093E717002322F700FE
:10E7080083274C001385090093F71700B3E497009B
:10E7180023229C00EF90DF906FF0DFDD2320D500EF
:10E72800832644001307B0012322D5006360C71273
:10E738008326840013078400930785006FF05FD752
:10E74800B38A9A00B307964023A45B0193E71700A6
:10E7580023A2FA008327C4FF1385090013090400C4
:10E7680093F71700B3E49700232E94FEEF905F8B86
:10E778006FF05FD88327CB0003278B00130A0600AE
:10E78800338BCA002326F70023A4E7006FF01FE1AC
:10E798008327C5FF93F7C7FF330AFA00338B4A0173
:10E7A8006FF0DFDF93050400EFF0DFA66FF09FD175
:10E7B8008327CB0003278B001306CAFF930640026A
:10E7C8002326F70023A4E70003278C008327CC0027
:10E7D80013098C00330B7C012326F70023A4E700E0
:10E7E80063E8C60493063001032704009307090071
:10E7F800E3F6C6D82324EC00032744009307B001AE
:10E808002326EC0003278400E3F6C7D62328EC0070
:10E818000327C40093074002232AEC0003270401BE
:10E828006304F60693078C01130404016FF01FD5E7
:10E838009305040013050900EFF0DF9D1304090098
:10E84800138A0B00930A0C006FF05FD5032784002E
:10E858002324E5000327C4002326E50083260401BA
:10E868006302F60413070401930705016FF05FC400
:10E87800832784002328FC008327C400232AFC0064
:10E8880003270401E310D6FA232CEC0003274401E4
:10E8980093070C0213048401232EEC0003270400C1
:10E8A8006FF0DFCD2328D5008326440113078401A8
:10E8B80093078501232AD500832684016FF05FBF63
:10E8C8009305040013050900EFF0DF946FF01FE2D1
:10E8D800832784002328FC008327C400232AFC0004
:10E8E800032704016308D60093078C01130404016D
:10E8F8006FF09FDE232CEC000327440193070C02E2
:10E9080013048401232EEC00032704006FF0DFDCDE
:10E918003367B5009303F0FF1377370063100710D0
:10E92800B7877F7F9387F7F70326050083A605003F
:10E93800B372F6003363F600B382F200B3E262000A
:10E94800639272106316D6080326450083A6450015
:10E95800B372F6003363F600B382F200B3E26200EA
:10E96800639E720C6316D6060326850083A685006F
:10E97800B372F6003363F600B382F200B3E26200CA
:10E988006398720C6316D6040326C50083A6C500D7
:10E99800B372F6003363F600B382F200B3E26200AA
:10E9A8006392720C6316D6020326050183A605013D
:10E9B800B372F6003363F600B382F200B3E262008A
:10E9C800639C720A1305450193854501E30ED6F44D
:10E9D8001317060193970601631EF70013570601E4
:10E9E80093D706013305F7409375F50F6390050239
:10E9F800678000001357070193D707013305F740D5
:10EA08009375F50F63940500678000001377F70F7F
:10EA180093F7F70F3305F7406780000003460500BA
:10EA280083C6050013051500938515006314D600E9
:10EA3800E31606FE3305D64067800000130545003F
:10EA480093854500E31CD6FC130500006780000091
:10EA58001305850093858500E312D6FC1305000095
:10EA6800678000001305C5009385C500E318D6FA32
:10EA78001305000067800000130505019385050153
:10EA8800E31ED6F813050000678000008327860080
:10EA9800130101FD232A5101232611022324810297
:10EAA8002322910223202103232E3101232C41010B
:10EAB800232861012326710123248101930A06007A
:10EAC80063880714130B05008329060003A50500B6
:10EAD80083A48500138405006F00400D8357C4008C
:10EAE80013F70748630A07088326440183250401AE
:10EAF8001307190093941600B386D40093D4F60133
:10EB0800330AB540B384D40093D414403307470183
:10EB18001386040063F6E400930407001306070055
:10EB280093F707406386070A9305060013050B0051
:10EB3800EF801FC8130C0500630A050A832504012A
:10EB480013060A00EFF04FDB8357C40093F7F7B7BB
:10EB580093E707082316F40033054C01338A444130
:10EB6800232A940023244401232884012320A40079
:10EB780093040900130A090013060A0093850B0081
:10EB8800EFF04FE9032784000325040083A78A00D8
:10EB9800B304974033054501232494002320A4009F
:10EBA8003389274123A42A016304090603A94900DC
:10EBB80083AB0900138A040093898900E30809FEDE
:10EBC800E37E99F093040900130A09006FF0DFFA55
:10EBD80013050B00EFF08FFC130C0500E31E05F680
:10EBE8008325040113050B00EF505F9F9307C000B6
:10EBF8002320FB008357C4001305F0FF93E70704A5
:10EC08002316F40023A40A0023A20A006F00C00000
:10EC180023A20A00130500008320C10203248102F5
:10EC280083244102032901028329C101032A8101A6
:10EC3800832A4101032B0101832BC100032C81008E
:10EC4800130101036780000083D7C500130101ED9C
:10EC5800232C4111232861112320A11123261112ED
:10EC6800232481122322911223202113232E3111D0
:10EC7800232A511123267111232481112322911152
:10EC8800232EB10F93F707082326D100138A050016
:10EC9800130B0500130D06006386070083A7050103
:10ECA800E384075EB7570180930AC10493878742BC
:10ECB800B75B0180B754018093090D0023205105EB
:10ECC8002324010423220104232A0100232C010008
:10ECD80023200102232E0100232401002328F10010
:10ECE800938B4B599384445A138D0A0083C70900A8
:10ECF800638C072013840900930650026388D72A7F
:10ED08008347140013041400E39A07FE330C3441BC
:10ED1800630C341F832681048327410423203D018B
:10ED2800B38686019387170023228D012324D104FB
:10ED38002322F10493067000130D8D0063C0F6289A
:10ED48000327810083470400330787012324E10058
:10ED5800638C071A9308F0FF834614009309140084
:10ED6800A30D01022322010013090000130CA005C2
:10ED7800930C90009305A00213840800938919004E
:10ED8800938706FE6368FC04032701019397270015
:10ED9800B387E70083A707006780070023220100E5
:10EDA800938706FD0326410083C60900938919004D
:10EDB800131726003307C70013171700B387E70098
:10EDC8002322F100938706FDE3FEFCFC938706FEF1
:10EDD800E37CFCFA638A06122306D108A30D01021C
:10EDE800130C1000930C10001304C10893080000C2
:10EDF800137F290063040F00130C2C00937E49082D
:10EE0800832781040326410463980E0003274100E9
:10EE1800B30D8741634AB07B0345B10393051600E0
:10EE280093068D00630005041305B103938717004B
:10EE38002320AD00130510002322AD002324F10484
:10EE48002322B10413057000E340B50A930F26008E
:10EE580013050D0113860500138D060093850F0019
:10EE680093060500630C0F021306C103938727005E
:10EE78002320CD00130620002322CD002324F104F3
:10EE88002322B10413077000E342B70A1386050072
:10EE9800138D0600938515009386860013050008D8
:10EEA800638CAE54B38D98416344B063B387FC0060
:10EEB80023208D0023229D012324F1042322B10461
:10EEC800130770006342B76C1373490063080300AB
:10EED80003274100B30C8741E3489009032441000C
:10EEE8006354840113040C0003278100330787004F
:10EEF8002324E100639A076A83C7090023220104D7
:10EF0800138D0A00E39807DE83278104E39E0756E2
:10EF18008357CA0093F70704E394075A8320C11262
:10EF2800032481120325810083244112032901123D
:10EF38008329C111032A8111832A4111032B01114D
:10EF4800832BC110032C8110832C4110032D011039
:10EF5800832DC10F130101136780000013050B00F7
:10EF6800EF800FE58327450013850700232EF10066
:10EF7800EFA04FDF9307050013050B00938D0700E3
:10EF88002320F102EF80CFE2832785009305A002BA
:10EF9800232CF100E3980D1E83C609006FF01FDED5
:10EFA80083C60900136909026FF05FDD330C344131
:10EFB800E31234D7834704006FF09FD91306010486
:10EFC80093050A0013050B00EFF05FACE31205F49C
:10EFD800138D0A006FF0DFD68327C1009308040061
:10EFE800A30D010203A40700938D4700E30404382E
:10EFF8009307F0FFE38EF8261386080093050000B8
:10F008001305040023261101EF801FF48328C10093
:10F01800E3060548B30C85402326B1019308000098
:10F028006F0040090327C100A30D0102130C100053
:10F0380083270700130747002326E1002306F1086A
:10F04800930C10001304C1086FF05FDA937709027C
:10F0580093080400638E070E8327C1009387770007
:10F0680093F787FF83A6470083AC07009387870041
:10F078002326F100138C060063C406109306F0FFE4
:10F08800930D09006388D800B3E68C01937DF9F7E6
:10F09800638E0676E31C0C0093069000E3E8960165
:10F0A80093870C03A307F10E13890D00930C10002E
:10F0B8001304F10E138C080063D49801138C0C0010
:10F0C8008347B103B337F000330CFC006FF05FD215
:10F0D800930804001369090193770902638407748C
:10F0E8008327C1009387770093F787FF83AC0700D6
:10F0F80003AC4700938787002326F100937DF9BF6F
:10F1080093060000A30D01021306F0FF638EC808E2
:10F1180033E68C0113F9FDF76314064A6392082855
:10F12800639A066E93FC1D001304010FE3840CF828
:10F1380093070003A307F10E1304F10E6FF09FF776
:10F14800136909019377090293080400E39607F00D
:10F158000327C1009377090193064700E392070448
:10F1680093770904E38607268327C1002326D10065
:10F17800839C070013DCFC4193060C00E3D006F0E7
:10F18800B3369001B30E8041338CDE409306D00233
:10F19800A30DD1021306F0FFB30C9041930D0900A3
:10F1A80093061000E396C8F613061000E384C6EE33
:10F1B800130620006380C6201304010F9317DC0197
:10F1C80093F67C0093DC3C0093860603B3EC97012E
:10F1D800135C3C00A30FD4FEB3E78C019305040035
:10F1E8001304F4FFE39C07FC93F71D00638E071ECE
:10F1F80093070003638AF61E9385E5FFA30FF4FEC9
:10F208009307010FB38CB74013890D0013840500D1
:10F218006FF05FEA93080400936D090193F70D02FC
:10F22800638807628327C10093061000138977005B
:10F23800137989FF93078900832C0900032C49005F
:10F248002326F1006FF01FEC8327C100B786FFFF6C
:10F2580093C6068383AC0700938747002326F100F3
:10F26800B7570180938747AF231ED1029308040044
:10F27800130C0000936D2900232AF1009306200047
:10F288006FF05FE883C60900136909086FF01FAFC4
:10F2980083C6090013871900E38AB622938706FDFF
:10F2A8009309070013040000E3ECFCAC83C60900D3
:10F2B80013172400B3088700939818003384F800C4
:10F2C800938706FD93891900E3F2FCFE6FF05FABAC
:10F2D80083C60900136949006FF05FAA9307B0025B
:10F2E80083C60900A30DF1026FF05FA90327C100CF
:10F2F80083C6090083270700130747002326E10078
:10F308002322F100E3DC07A6B307F0402322F10033
:10F31800136949006FF09FA683C609001369190095
:10F328006FF0DFA58347B10383C60900E39807A4FC
:10F3380093070002A30DF1026FF05FA483C60900D2
:10F3480093078006638EF67E136909046FF01FA386
:10F358000327C10093770902832607001307470094
:10F368002326E100639C075E93770901639E077E6D
:10F3780093770904E3940710137309206306037E47
:10F38800832781002380F6006FF05F9683C609000B
:10F398009307C006638EF67A136909016FF01F9E02
:10F3A80013061000E384C61013062000930D09000D
:10F3B800E394C6E0832641011304010F93F7FC0090
:10F3C800B387F60003C7070093DC4C009317CC0102
:10F3D800B3EC9701135C4C00A30FE4FEB3E78C0178
:10F3E8001304F4FFE39C07FC9307010FB38C8740D9
:10F3F80013890D006FF01FCC03274100B30D87411F
:10F40800E352B0AB13050001E356B50B232281028A
:10F418009306000113040A00930E7000138A0D006E
:10F42800938D0900938908006F00C000130A0AFF32
:10F4380063DA4605938707011306160023209D000B
:10F448002322DD002324F1042322C104130D8D009F
:10F45800E3DECEFC130601049305040013050B003C
:10F46800EFF0CFE2631E056E93060001130A0AFF50
:10F478008327810403264104138D0A00930E70002C
:10F48800E3CA46FB9388090093890D00930D0A008F
:10F49800130A0400032441021306160013058D0005
:10F4A800B387B70123209D002322BD012324F10443
:10F4B8002322C10413077000634AC764B38D9841BF
:10F4C8009305160093068500130D0500E350B09FC1
:10F4D80013050001635EB57393060001930870007D
:10F4E8006F00C000938D0DFF63DAB605938707019F
:10F4F8001306160023209D002322DD002324F10497
:10F508002322C104130D8D00E3DEC8FC1306010499
:10F5180093050A0013050B00EFF04FD7E31A059E79
:10F5280093060001938D0DFF832781040326410470
:10F53800138D0A0093087000E3CAB6FB9305160002
:10F5480013068D00B387B70123209D002322BD0138
:10F558002324F1042322B104130770006342B73255
:10F56800130D060093851500B387FC0023208D003A
:10F5780023229D012324F1042322B10413077000E0
:10F5880093068600E352B7941306010493050A0014
:10F5980013050B00EFF08FCFE31C0596832781043A
:10F5A80093860A006FF05F921306010493050A0020
:10F5B80013050B00EFF08FCDE30005946FF05F9516
:10F5C800930D09006FF05FBE9306000163DEB60B72
:10F5D80013070D00930F7000130D0C002322E10395
:10F5E800130C09002324D10313090A00138A090004
:10F5F8009309040013840D00938D0C00938C08006C
:10F608006F00C000130404FF63DA860493870701C0
:10F6180013061600232077012322D7002324F104A0
:10F628002322C10413078700E3DECFFC130601047D
:10F638009305090013050B00EFF04FC56316054A43
:10F6480093060001130404FF832781040326410461
:10F6580013870A00930F7000E3CA86FA032F41024A
:10F66800832E810293880C00938C0D00930D040067
:10F678001384090093090A00130A090013090C00EE
:10F68800130C0D00130D0700B387B70113061600FE
:10F6980023207D012322BD012324F1042322C10458
:10F6A80093067000130D8D0063D8C6F61306010487
:10F6B80093050A0013050B00232611032324D10305
:10F6C8002322E103EFF08FBCE31405848327810430
:10F6D800032641048328C102832E8102032F41029D
:10F6E800138D0A006FF04FF31306010493050A0007
:10F6F80013050B00232611032324D1032322E1033E
:10F70800EFF0CFB8E3160580032641048327810470
:10F718008328C102832E8102032F410293064105EB
:10F7280093051600138D0A006FF0CFF3130601043A
:10F7380093050A0013050B00232411032322D10388
:10F74800EFF0CFB4631605FC032641048327810438
:10F7580083288102832E41029306410593051600F2
:10F76800138D0A006FF08FF313060001032741047D
:10F7780063509607930D0001130470006F00C000DA
:10F78800938C0CFF63D69D05938707011307170019
:10F7980023A0760123A2B6012324F1042322E10445
:10F7A80093868600E35EE4FC1306010493050A00D1
:10F7B80013050B00EFF08FAD631C05F4938C0CFF61
:10F7C800832781040327410493860A00E3CE9DFB27
:10F7D800B38797011307170023A0760123A2960188
:10F7E8002324F1042322E1049306700063D8E6EE93
:10F7F8001306010493050A0013050B00EFF00FA987
:10F80800631805F0832781046FF04FEDE39A0888A9
:10F8180013890D0093080000930C00001304010FD6
:10F828006FF05F890327C1009377090193064700AA
:10F838006392071893770904638E07368327C100FC
:10F84800130C00002326D10083DC07006FF01F8B08
:10F858000327C10093F70D0193064700639A071029
:10F8680093F70D04638607388327C100130C000043
:10F878002326D10083DC0700930610006FF09F88D1
:10F888001306010493050A0013050B00EFF00FA0FF
:10F89800631005E883254104832781049306410505
:10F8A80093851500138D0A006FF04FE093F70D4014
:10F8B8002324410323263103130A0C0093890C00E7
:10F8C80013090000832C81011304010F2322110363
:10F8D800138C07006F0040021306A0009306000077
:10F8E8001385090093050A00EF00102363060A3206
:10F8F80093090500138A05001306A000930600006B
:10F908001385090093050A00EF00506413050503E9
:10F91800A30FA4FE130919001304F4FFE30E0CFA55
:10F9280083C60C00E39A26FB9307F00FE306F9FA67
:10F93800631C0A169307900063E837179307010FB3
:10F94800232C910183284102032A81028329C102C1
:10F95800B38C874013890D006FF0CFF50327810022
:10F968009357F74123A0E60023A2F6006FF00FB8E3
:10F978002326D100832C0700130C000093061000E7
:10F988006FF04FF88327810183C60900638807BE9B
:10F9980083C70700638407BE136909406FF00FBE71
:10F9A800832C07002326D10013DCFC4193060C00AE
:10F9B8006FF08FEC832C0700130C00002326D10076
:10F9C8006FF0CFF3B7570180938787B0232AF100F0
:10F9D8009377090293080400638C07068327C10004
:10F9E8009387770093F787FF83AC070003AC470042
:10F9F800938787002326F10013761900630E06000B
:10FA080033E68C01630A060013060003230EC102C5
:10FA1800A30ED10213692900937DF9BF9306200034
:10FA28006FF04FEE93080400930D09006FF00FFF7D
:10FA3800930804006FF04FEAB7570180938747AFE8
:10FA4800232AF1009377090293080400E39807F842
:10FA58000327C1009377090113064700638A070843
:10FA6800832C0700130C00002326C1006FF0DFF879
:10FA780013050400EF901FAF930C05002326B10176
:10FA8800930800006FF00FE393050004EF705FD256
:10FA98002320AA002328AA00630C05249307000446
:10FAA800232AFA006FF00FA0832701028325C101E2
:10FAB800130900003304F4401386070013050400FB
:10FAC800EF901FB383C51C001306A0009306000027
:10FAD8003338B0001385090093050A00B38C0C0174
:10FAE800EF0090036FF0DFE0130A09006FF04FC2D8
:10FAF800937709046382070A8327C100130C000067
:10FB08002326C10083DC07006FF01FEF13060104F2
:10FB180093050A0013050B0023221103EFE01FF7DA
:10FB2800631805BE03264104832781048328410204
:10FB38009306410593051600138D0A006FF08FB6E2
:10FB480083C6190013690920938919006FF00FA360
:10FB580083C6190013690902938919006FF00FA26F
:10FB6800130A04006FF0CFBA8327810023A0F600A0
:10FB78006FF0CF9793076000938C080063F4170128
:10FB8800930C6000375E0180138C0C002326B101B2
:10FB98001304CEB16FF08FA5937709206386070C05
:10FBA8008327C100130C00002326C10083CC070063
:10FBB8006FF09FE493770920638E07088327C100BD
:10FBC800130C00002326D10083CC07006FF00FD35D
:10FBD80093770920638407068327C1002326D10071
:10FBE800838C070013DCFC4193060C006FF0CFC830
:10FBF80093F70D20638807028327C100130C0000C8
:10FC08002326D10083CC0700930610006FF08FCF16
:10FC1800138606006FF01F9393079000E3EA37CD31
:10FC28006FF0DFD18327C100130C00002326D10019
:10FC380083AC0700930610006FF0CFCC8327C10078
:10FC48002326D10083AC070013DCFC4193060C008B
:10FC58006FF08FC28327C100130C00002326D10048
:10FC680083AC07006FF08FC98327C100130C000015
:10FC78002326C10083AC07006FF01FD883278100BB
:10FC88002390F6006FF08F861306010493050A008F
:10FC980013050B00EFE09FDF6FF08FA7938C080030
:10FCA8002326B101930800006FF0CFC0930D09001F
:10FCB8006FF00FBF13850600138605006FF04FFE27
:10FCC8009307F0FF2324F1006FF04FA58327C100AD
:10FCD80003A4070093874700635404001304F0FF4C
:10FCE80083C619002326F100930907006FF00F89D6
:10FCF8009307C0002320FB009307F0FF2324F100A3
:10FD08006FF0CFA1130101FE232C8100232A91005B
:10FD180023282101232E1100232631011309050070
:10FD280093840500130406006306050083278503F2
:10FD3800638807140317C400832684019377870018
:10FD48002324D4009316070193D60601638207087B
:10FD580083270401638E07061396260193F9F40F8F
:10FD680093F4F40F635E0608032704008326440116
:10FD7800B307F74063DED70A83268400130617000B
:10FD88002320C4009386F6FF2324D40023003701E0
:10FD980003274401938717006308F70C8357C400AF
:10FDA80093F71700638607009307A000638EF40A91
:10FDB8008320C10103248101032901018329C10092
:10FDC80013850400832441011301010267800000A8
:10FDD8009305040013050900EF309FD8631E05083A
:10FDE8000317C40093F9F40F83270401931607013E
:10FDF80093D606011396260193F4F40FE34606F60C
:10FE080083264406372600003367C70037E6FFFF1E
:10FE18001306F6FFB3F6C6002316E4000327040012
:10FE28002322D40683264401B307F740E3C6D7F458
:10FE38009305040013050900EF408FA9631E05020E
:10FE48000327040083268400930710001306170075
:10FE58009386F6FF2320C4002324D400230037010F
:10FE680003274401E31CF7F2930504001305090076
:10FE7800EF400FA6E30E05F29304F0FF6FF05FF377
:10FE8800EF40CFDE6FF01FEB9307050003A5C125F8
:10FE980013860500938507006FF0DFE6130101FE66
:10FEA800232C8100232A9100232E110083A7811A75
:10FEB800130405009384060063820502E7800700A7
:10FEC8009307F0FF6306F5028320C1010324810133
:10FED800832441011301010267800000130600001A
:10FEE80093054100E78007009307F0FFE31EF5FC48
:10FEF80023A004009307A0088320C1012320F40055
:10FF08000324810183244101130101026780000059
:10FF1800130101FE232C8100232A9100232E1100B6
:10FF280083A4C12583A7811A13040600630A050266
:10FF38001386050093060400930505001385040045
:10FF4800E78007009307F0FF630AF5028320C101E9
:10FF58000324810183244101130101026780000009
:10FF6800930606009305410013060000138504005C
:10FF7800E78007009307F0FFE31AF5FC232004004D
:10FF88008320C101032481019307A00823A0F40062
:10FF980083244101130101026780000003A3811A31
:10FFA80067000300638405029307F00F63E8C70046
:10FFB8002380C50013051000678000009307A00880
:10FFC8002320F5001305F0FF6780000013050000EB
:10FFD80067800000130101FF13056000232611004C
:10FFE800EF00C02813051000EF008FA8130101FFD0
:08FFF800930500082324810099
:02000004800179
:100000002326110013040500EF700FFB232EA42CF0
:100010006304050293070508232005001305450026
:10002000E31CF5FE130500008320C10003248100BA
:1000300013010101678000001305F0FF6FF0DFFE80
:100040008327C52D63860700130500006780000025
:100050006FF05FFA130101FE232A9100232E110095
:10006000232C81009307F0019304050063EAB70293
:10007000138405008325C52D63840504131424000F
:1000800033848500032504002320C4008320C1019C
:1000900003248101832441011301010267800000D0
:1000A0008320C10103248101930760012320F5000F
:1000B000832441011305F0FF130101026780000052
:1000C0002326C100EFF01FF3930705001305F0FF8F
:1000D000E39E07FA83A5C42D0326C1006FF01FFA23
:1000E000130101FF23229100232611002324810004
:1000F0009307F0019304050063EAB70A8327C52D2F
:10010000138405006384070413972500B387E70071
:1001100003A70700630C070293061000630CD706C1
:100120009306F0FF6308D7041385050023A007009A
:10013000E7000700130500008320C10003248100AD
:10014000832441001301010167800000138504002E
:10015000EF00C01C13060400032481008320C100AB
:100160009305050013850400832441001301010158
:100170006F0080148320C100032481009307600175
:100180002320F50083244100130510001301010111
:10019000678000008320C100032481008324410084
:1001A000130500001301010167800000930760013F
:1001B0002320F5001305F0FF6FF01FF89307F001FF
:1001C00063E6B70A8327C52D130101FE232C910096
:1001D000232E110093040500638C07041397250058
:1001E000B387E70003A70700630A07029306F0FF3F
:1001F0006306D706930610006308D704138505002D
:1002000023A00700E7000700130500008320C101B9
:100210008324810113010102678000008320C10152
:10022000832481011305100013010102678000007F
:100230002326B100EFF01FDC6316050283A7C42D4F
:100240008325C1006FF09FF98320C10183248101C0
:100250001305300013010102678000001305200020
:100260006FF0DFFA1305F0FF6FF05FFA1305F0FF90
:10027000678000009305050003A5C1256FF05FE6C8
:100280009307050003A5C125138605009385070084
:100290006FF05FDC03A5C1258327C52D63860700AA
:1002A00013050000678000006FF0DFD493050500A0
:1002B00003A5C1256FF09FF0130101FF138705000F
:1002C00023248100232291001304050093050600D6
:1002D000130507002326110023AE0130EF008FA97C
:1002E0009307F0FF630CF5008320C1000324810015
:1002F00083244100130101016780000083A7C131FD
:10030000E38407FE8320C1002320F400032481003E
:100310008324410013010101678000006F000FA6D4
:10032000930805009387050013080600138506004F
:100330001383080063940628B75601809386C67617
:1003400063F6C50E370701006378E60C1307F00F5C
:100350003337C700131737003355E600B386A600BE
:1003600083C60600130500023387E600B306E540A6
:10037000630CE500B397D70033D7E8003318D600F5
:10038000B365F7003393D80093580801B3D715032A
:10039000131608011356060113570301B3F615038C
:1003A00013850700B305F6029396060133E7E600CE
:1003B000637EB700330707011385F7FF6368070102
:1003C0006376B7001385E7FF330707013307B740AC
:1003D000B3771703131303011353030133571703A1
:1003E0009397070133E36700B306E602130607009D
:1003F000637CD300330368001306F7FF63660301D1
:100400006374D3001306E7FF131505013365C500B8
:10041000930500006F00400E37050001130700012F
:10042000E36CA6F2130780016FF01FF3631606005A
:10043000130710003358C702370701006370E80C38
:100440001307F00F63740701130580003357A800EA
:10045000B386E60003C70600130600023307A700B1
:10046000B306E6406316E60AB3870741930510001A
:100470009358080113160801135606011357030178
:10048000B3F61703B3D717039396060133E7E600D5
:10049000330EF60213850700637EC7013307070199
:1004A0001385F7FF636807016376C7011385E7FFCC
:1004B000330707013307C741B3771703131303014A
:1004C00013530301335717039397070133E367006F
:1004D000B306E60213060700637CD300330368000B
:1004E0001306F7FF636603016374D3001306E7FF87
:1004F000131505013365C50067800000370700014B
:1005000013050001E364E8F4130580016FF01FF4A4
:100510003318D800B3D5E7003393D800B397D7008A
:1005200033D7E800935808013366F70033F7150313
:100530009317080193D7070113550601B3D5150387
:10054000131707013367A700B386B70213850500A9
:10055000637ED700330707011385F5FF6368070142
:100560006376D7001385E5FF33070701B306D7404D
:1005700033F716031316060113560601B3D61603F6
:1005800013170701B388D702B367C70013870600A4
:1005900063FE1701B38707011387F6FF63E80701BE
:1005A00063F617011387E6FFB3870701931505016B
:1005B000B3871741B3E5E5006FF09FEB63E6D5180D
:1005C0003707010063F4E6041307F00FB335D700D3
:1005D000939535003757018033D5B6001307C7769A
:1005E0003307A70003470700130500023307B700CE
:1005F000B305E5406316E50213051000E3EEF6EEE1
:1006000033B5C800134515006FF01FEF3707000121
:1006100093050001E3E0E6FC930580016FF09FFB8A
:100620003353E600B396B6003363D300135503018A
:10063000B31EB60033D6E700B376A602B397B70071
:1006400033D7E8003368F7009317030193D7070106
:10065000135708013356A6029396060133E7E600C6
:10066000338FC702130E0600637EE701330767006E
:10067000130EF6FF636867006376E701130EE6FF6B
:10068000330767003307E741B376A7023357A70262
:10069000939606013386E7029317080193D7070163
:1006A000B3E7F6009306070063FEC700B387670051
:1006B0009306F7FF63E8670063F6C7009306E7FF5A
:1006C000B387670013150E01370E01003365D5009F
:1006D0009306FEFF3378D500B387C740B3F6DE003C
:1006E0001356050193DE0E013303D802B306D6027A
:1006F000135703013308D8033308D8003307070121
:100700003306D6036374D7003306C6019356070138
:100710003386C60063E6C702E39CC7CEB707010075
:100720009387F7FF3377F700131707013373F3004D
:10073000B398B8003307670093050000E3FEE8DADA
:100740001305F5FF6FF0DFCC9305000013050000E3
:100750006FF09FDA930806001387060093070500E1
:1007600013880500639C0622B75601809386C676DF
:1007700063FCC50C37030100637E660A1303F00FA8
:100780006374C300130780003353E600B38666002A
:1007900003CE0600330EEE00130700023303C741F9
:1007A000630CC701B3956500335EC501B3186600DD
:1007B0003368BE00B317650013D608013377C8024B
:1007C000139508011355050193D607013358C80244
:1007D00013170701B366D7003308050363FA060150
:1007E000B386160163E6160163F40601B3861601AB
:1007F000B386064133F7C6029397070193D70701E3
:10080000B3D6C602B306D50213150701B367F500C8
:1008100063FAD700B387170163E6170163F4D700C3
:10082000B3871701B387D74033D56700930500001E
:10083000678000003703000113070001E36666F4D8
:10084000130780016FF05FF46316060013061000B3
:10085000B35816033706010063F2C80A1306F00FF7
:10086000637416011307800033D6E800B386C60010
:1008700003CE0600330EEE00130700023303C74118
:100880006318C709B385154113D7080113950801EB
:100890001355050113D60701B3F6E502B3D5E502FA
:1008A00093960601B3E6C600B305B50263FAB60037
:1008B000B386160163E6160163F4B600B38616012B
:1008C000B385B640B3F6E5029397070193D70701C6
:1008D000B3D5E502B305B50213950601B367F5007C
:1008E00063FAB700B387170163E6170163F4B70033
:1008F000B3871701B387B7406FF01FF337060001C6
:1009000013070001E3E2C8F6130780016FF0DFF57B
:10091000B398680033D7C501B3176500335EC501CE
:1009200013D50801B376A702B3956500336EBE00F8
:100930009395080193D5050113560E013357A7026D
:1009400093960601B3E6C6003387E50263FAE60034
:10095000B386160163E6160163F4E600B38616015A
:100960003386E640B376A602131E0E01135E0E0117
:100970003356A602939606013386C502B3E5C60137
:1009800063FAC500B385150163E6150163F4C5007C
:10099000B3851501B385C5406FF01FEFE3EAD5E8D5
:1009A0003707010063FCE604130EF00F3337DE0057
:1009B00013173700B758018033D3E6009388C87601
:1009C000B388680003CE0800330EEE001307000260
:1009D0003303C741631EC70363E4B600636AC500FF
:1009E000B307C540B385D5403335F5003388A540FE
:1009F00013850700930508006FF09FE3B708000117
:100A000013070001E3E816FB130780016FF09FFA5C
:100A10003357C601B3966600336FD700B3D7C5010D
:100A200013570F01B3F8E702B39565003358C501BA
:100A30003368B80093150F0193D50501935608014B
:100A40003316660033156500B3D7E70293980801A3
:100A5000B3E6D800B38EF5029388070063FED60193
:100A6000B386E6019388F7FF63E8E60163F6D601F3
:100A70009388E7FFB386E601B386D641B3FEE6026C
:100A80001318080113580801B3D6E602939E0E010D
:100A9000B3EE0E01B385D5029387060063FEBE0058
:100AA000B38EEE019387F6FF63E8EE0163F6BE00B6
:100AB0009387E6FFB38EEE01B385BE40939808019D
:100AC000B70E0100B3E8F8009387FEFF33F8F80093
:100AD0009356060193D80801B377F6003307F8025E
:100AE000B387F8023308D802B388D8023308F80075
:100AF00093560701B386060163F4F600B388D80164
:100B0000B70701009387F7FF13D80601B3F6F60085
:100B1000939606013377F700B30818013387E60090
:100B200063E61501639E1501637CE5003306C7404B
:100B30003337C7003307E701B388E84013070600DF
:100B40003307E5403335E500B3851541B385A5404E
:100B5000B397C5013357670033E5E700B3D56500A8
:100B60006FF01FCD130101FD93D7450123229102A0
:100B700023202103232C4101232861012324810107
:100B80009394C5002326110223248102232E3101D0
:100B9000232A5101232671011397570113090500D8
:100BA000130B0600138C060093D4C40013DAF5016E
:100BB0006304070A93FAF77F9307F07F6380FA10C4
:100BC0009359D50193943400B3E49900B709800098
:100BD000B3E9340113143500938A1AC0930B000053
:100BE00093574C011315CC00139757019354C5002C
:100BF00093F5F77F135CFC01630007109307F07F08
:100C00006382F516139534009357DB0133E5A70093
:100C1000B7048000B3649500931F3B00138515C093
:100C20001306000093972B00B3E7C7009387F7FFE5
:100C30001307E000B3468A01B385AA406360F71644
:100C400037570180939727001307876BB387E70017
:100C500083A7070067800700B3E9A400638E090635
:100C60006380040413850400EF30D03B930755FFE5
:100C70001307C001634CF7029309D001130485FFE9
:100C8000B389F940B3948400B3593901B3E99900A9
:100C9000331489009305D0C0B38AA5406FF01FF4C8
:100CA000EF305038130505026FF05FFC930485FDAB
:100CB000B3199900130400006FF0DFFDB3E9A4003D
:100CC000638409021304050093890400930AF07FEA
:100CD000930B30006FF0DFF013040000930A000064
:100CE000930B10006FF0DFEF13040000930AF07F06
:100CF000930B20006FF0DFEEB3EF640163800F0809
:100D00006382040413850400EF30D031930505009D
:100D1000938755FF1307C001634EF7029306D00176
:100D2000938F85FFB386F6403395F401B356DB000D
:100D3000B3E4A600B31FFB011307D0C03305B740CF
:100D40006FF01FEE13050B00EF30D02D9305050259
:100D50006FF01FFC138585FDB314AB00930F0000EB
:100D60006FF09FFDB3EF640163820F02930F0B00DE
:100D70001305F07F130630006FF0DFEA93040000E4
:100D800013050000130610006FF0DFE99304000064
:100D90001305F07F130620006FF0DFE863E63401EF
:100DA000639C9934636AF4351396F9011357140060
:100DB0009317F40193D919003364E6001395840066
:100DC00093D88F01B3E8A8001355050133D8A902C1
:100DD000939E080193DE0E011357040113938F00B5
:100DE000B3F4A902930F080033860E03939904010C
:100DF00033673701637EC70033071701930FF8FF8E
:100E0000636817016376C700930FE8FF3307170184
:100E10003307C740335EA7021314040113540401BF
:100E20003377A70213060E003388CE03131707018A
:100E30003367E400637E0701330717011306FEFFE3
:100E400063681701637607011306EEFF3307170186
:100E500033040741939F0F0137080100B3EFCF0020
:100E6000130EF8FF13D60F0133F7CF01135F030101
:100E7000337EC301B303EE02B304C6033307EF02AC
:100E8000B302E6033306970013D703013307C70005
:100E900063749700B38202011356070133065600AC
:100EA000B70201009382F2FF33785700131808014C
:100EB000B3F35300330878006368C40093840F00D1
:100EC0006314C40463F20705B387670033B7670090
:100ED000330717013304E4009384FFFF63E68800BF
:100EE0006394880263E267026366C400631E86003F
:100EF00063FC0701B387670033B767003307170147
:100F00009384EFFF3304E400338807413304C44083
:100F1000B3B707013304F440930FF0FF63848812E2
:100F2000B35FA402135708013374A40213860F00A1
:100F3000B387FE031314040133648700637EF40057
:100F4000330414011386FFFF636814016376F40011
:100F50001386EFFF330414013304F4403357A40223
:100F600013180801135808013374A40293070700EB
:100F7000B38EEE021314040133648800637ED4013F
:100F8000330414019307F7FF636814016376D401F7
:100F90009307E7FF33041401131606013366F600C6
:100FA0009317060193D70701135706013308EF0281
:100FB0003304D441330FFF02B38EC703330EC7038C
:100FC00093D70E01330FCF01B387E70163F6C70153
:100FD000370701003308E80013D70701330707017B
:100FE000370801001308F8FF33F507011315050151
:100FF000B3FE0E013305D5016368E4006310E424F9
:10100000930F06006300050433848800930FF6FFF6
:10101000636414036366E4006310E4226370A30254
:101020009317130033B36700B3081301930FE6FF60
:1010300033041401138307006314E40063046500A0
:1010400093EF1F009387F53F6358F01013F77F006D
:101050006300070213F7FF0013064000630AC7008E
:1010600013864F00B33FF601B384F401930F0600DB
:1010700013977400635A0700B70700FF9387F7FFC1
:10108000B3F4F400938705401307E07F6340F70A49
:1010900093DF3F001397D4013367F70113D5340072
:1010A000939747013706F07F1315C5008320C102CF
:1010B00003248102B3F7C7001355C50033E5A70029
:1010C0009396F601B367D5008324410203290102F8
:1010D0008329C101032A8101832A4101032B0101D4
:1010E000832BC100032C81001305070093850700A3
:1010F00013010103678000009385F5FF930700004B
:101100006FF0DFCB93060A0093840900930F04006D
:1011100013860B00930730006308F60E9307100048
:10112000630EF60E93072000E31EF6F01305000091
:10113000130700009307F07F6FF09FF693060C00F3
:101140006FF05FFDB7040800930F000093060000E6
:10115000130630006FF01FFC130510003305F54037
:1011600013078003634CA70A1307F0016344A70623
:101170009385E541B397B40033D7AF00B395BF0073
:10118000B3E7E700B335B000B3E7B70033D5A40049
:1011900013F777006300070213F7F7001306400008
:1011A000630AC70013874700B337F7003305F5001C
:1011B0009307070013178500634807061317D50127
:1011C00093D737003367F7001355350093070000B6
:1011D0006FF01FED130710FEB307F7401306000270
:1011E000B3D7F400130700006306C5009385E543F9
:1011F0003397B400B36FF701B33FF001B3E7F701E2
:10120000130500006FF0DFF8370508001307000032
:101210009307F07F930600006FF09FE8130500002E
:10122000130700006FF09FFA13050000130700007A
:10123000930710006FF0DFE613860F00930F060090
:101240006FF01FE0130101FD93D7450123248102B4
:1012500023229102232E3101232C4101232A510103
:101260009394C50023261102232021032328610122
:1012700023267101139757011304050093090600F3
:10128000938A060093D4C40013DAF5016306070AB3
:1012900013FBF77F9307F07F6302FB109357D50191
:1012A00093943400B3E49700B7078000B3E4F400EC
:1012B00013193500130B1BC0930B000093D74A0181
:1012C0001394CA00139757011354C40013F5F77F02
:1012D00093DAFA01630007109307F07F6300F516B5
:1012E00093D7D9011314340033E48700B707800083
:1012F0003364F400130515C09397390013070000F9
:1013000093962B00B3E6E6003305AB009386F6FF19
:101310001308E00033465A0193051500636CD81496
:1013200037550180939626001305456FB386A600B6
:1013300083A606006780060033E9A400630C090653
:101340006380040413850400EF30C04D130755FF7C
:101350009307C00163CCE7029307D001130985FF0F
:10136000B387E740B3942401B357F400B3E4970084
:1013700033192401130BD0C0330BAB406FF0DFF3F4
:10138000EF30404A130505026FF05FFC930485FDC2
:10139000B3149400130900006FF0DFFD33E9A400DB
:1013A0006302090213090500130BF07F930B300051
:1013B0006FF0DFF093040000130B0000930B10009C
:1013C0006FF0DFEF93040000130BF07F930B20000E
:1013D0006FF0DFEEB3673401638E07066300040429
:1013E00013050400EF300044930655FF9307C00136
:1013F00063CED7021307D001930785FF3307D74089
:101400003314F40033D7E90033648700B397F9004D
:101410001307D0C03305A7406FF05FEE13850900B6
:10142000EF304040130505026FF01FFC130485FDEB
:1014300033948900930700006FF09FFDB367340178
:1014400063820702938709001305F07F13073000BA
:101450006FF01FEB130400001305000013071000CA
:101460006FF01FEA130400001305F07F130720003C
:101470006FF01FE9370F01001307FFFF93560901B3
:1014800013D307013379E900B3F7E700B308230367
:101490003308F902B38FF602B38EF80193580801AE
:1014A000B388D801338E660263F4F801330EEE017F
:1014B00093D20801B3F8E8003378E800135F040121
:1014C000939808013374E400B388080133878602D7
:1014D0003308890233092F03B30EE90013590801B9
:1014E0003309D901B386E6036376E90037070100C3
:1014F000B386E600935E0901B38EDE00B7060100F5
:10150000938FF6FF3379F9013378F80113D704018B
:1015100013190901B3F4F401B383970233090901E4
:10152000B382220133089302B307F702B30FE30239
:101530003303F80013D80301330868006374F8001C
:10154000B38FDF0093570801B7060100B38FF7018F
:101550009387F6FF3378F800B3F7F300B3039402F0
:10156000131808013308F80033048702B3049F02FC
:101570003303EF02B384840013D70301B30497004D
:1015800063F484003303D300B70701009387F7FFA8
:10159000B3F6F40093960601B3F7F300330E5E0042
:1015A000B386F60033392E01B386D6013387260180
:1015B000330E0E0133380E01330FF701B3020F0162
:1015C000B3B6D6013337270133E7E60033B802015B
:1015D00093D40401B33FFF013307970033E80F01B1
:1015E00093179E003307070133076700B3E717011E
:1015F00013179700B337F000135E7E0113D4720106
:10160000B3E7C70193929200931677003364870083
:10161000B3E7570063D4061013D7170093F71700EA
:10162000B367F7001317F401B3E7E700135414008E
:101630009386F53F6358D00E13F7770063000702D7
:1016400013F7F70013054000630AA700138747004C
:10165000B337F7003304F40093070700131774003F
:10166000635A0700370700FF1307F7FF3374E400DE
:10167000938605401307E07F6348D71613D73700DA
:101680009317D401B3E7E7001354340013974601CE
:101690001314C400B706F07F3377D7001354C40087
:1016A000336487001316F6018320C1023367C40038
:1016B0000324810283244102032901028329C101F9
:1016C000032A8101832A4101032B0101832BC100DD
:1016D00013850700930507001301010367800000CD
:1016E00013060A00138404009307090013870B00F4
:1016F00093062000630AD70E93063000630CD70CC4
:1017000093061000E316D7F21304000093070000BD
:101710006F00800813860A006FF09FFD9305050097
:101720006FF01FF1130510003305D5401307800338
:10173000E34CA7FC1307F0016344A7069385E5413A
:101740003317B400B3D6A700B397B7003367D700F9
:10175000B337F000B367F7003354A40013F77700F2
:101760006300070213F7F70093064000630AD700EF
:1017700013874700B337F7003304F40093070700DB
:1017800013178400634A07061317D40193D7370051
:10179000B367F70013543400930600006FF01FEF97
:1017A000130710FE3307D740130800023357E40035
:1017B00093060000630605019385E543B316B40064
:1017C000B3E7F600B337F000B367F7001304000087
:1017D0006FF0DFF837040800930700009306F07FEE
:1017E000130600006FF09FEA130400009307000047
:1017F0009306F07F6FF09FE9130400009307000049
:10180000930610006FF09FE88327C50003AF050023
:1018100083AF450083A2850083A5C50037870000FC
:1018200093D607011307F7FF13980701939E05014D
:1018300013D6F701B3F6E60093D705018328050018
:1018400003234500032E8500130101FF13580801EF
:1018500093DE0E01B3F7E70093D5F5016390E6023E
:1018600033E768003367C7013367070113051000CA
:10187000631A07046398D7046F008000639CE70035
:101880003367FF01336757003367D7011305100033
:10189000631A0702130510006396D7026394E803E6
:1018A0006312F30363105E02631ED8016300B60285
:1018B000639A070033E568003365C50133650501A8
:1018C0003335A000130101016780000013050000FB
:1018D0006FF05FFF832F050003284500032E85006E
:1018E0000325C50083A6C500B78700001356050170
:1018F0009387F7FF1393060113D7060183A2050010
:1019000083A8450083AE85003376F6009315050164
:10191000130101FF93D505011355F501135303017D
:101920003377F70093D6F601631EF600B3E70F0195
:10193000B3E7C701B3E7B7006388070C1305E0FFFF
:101940006F004006631AF700B3E71201B3E7D7014F
:10195000B3E76700E39407FE631A060AB3E70F01D3
:10196000B3E7C701B3E7B70093B71700631A0700DF
:1019700033EF1201336FDF01336F6F00630A0F061D
:10198000639C07006394A6006352C702630E0504BC
:101990001305F0FF6F0000011305F0FF63840600DC
:1019A0001385060013010101678000006356E600FD
:1019B000E31A05FE6FF0DFFDE36AB3FC639E650288
:1019C000E3E6CEFD631EDE03E3E208FD63141801C7
:1019D000E3EEF2FBE36E18FD63141801E3EA5FFC2B
:1019E000130500006FF01FFC130510006FF09FFB44
:1019F000E39807FE6FF09FF9E3EC65FA6FF05FFE86
:101A0000E368DEFB6FF0DFFDE300C7F4E31C07F6DD
:101A1000930700006FF0DFF5832F050003284500D2
:101A2000032E85000325C50083A6C500B7870000E7
:101A3000135605019387F7FF1393060113D7060189
:101A400083A2050083A8450083AE85003376F600A7
:101A500093150501130101FF93D505011355F501F8
:101A6000135303013377F70093D6F601631EF60094
:101A7000B3E70F01B3E7C701B3E7B7006388070C0B
:101A8000130520006F004006631AF700B3E7120148
:101A9000B3E7D701B3E76700E39407FE631A060ACA
:101AA000B3E70F01B3E7C701B3E7B70093B7170078
:101AB000631A070033EF1201336FDF01336F6F00DA
:101AC000630A0F06639C07006394A6006352C70273
:101AD000630E05041305F0FF6F0000011305F0FF0E
:101AE000638406001385060013010101678000006E
:101AF0006356E600E31A05FE6FF0DFFDE36AB3FC10
:101B0000639E6502E3E6CEFD631EDE03E3E208FDAD
:101B100063141801E3EEF2FBE36E18FD6314180181
:101B2000E3EA5FFC130500006FF01FFC13051000D3
:101B30006FF09FFBE39807FE6FF09FF9E3EC65FA07
:101B40006FF05FFEE368DEFB6FF0DFFDE300C7F4DC
:101B5000E31C07F6930700006FF0DFF5130101F4B3
:101B6000232A910A83A4C50083A6050083A7450004
:101B70002324A10003A58500139704012328210B2A
:101B80002326310B0329C600832906002324410B99
:101B90002322510B032A8600832A46003786000041
:101BA000232C810A1357070113D404011306F6FFEF
:101BB00023269106232E110A2320610B232E71095F
:101BC000232C8109232A91092328A1092326B1095D
:101BD0002320D1062322F1062324A1062328D102A3
:101BE000232AF102232CA102232EE1023374C40024
:101BF00093D4F401630804126306C424B7070100F8
